Archive member included       because of file (symbol)

E:/nightly/rwsdk.sky/rwsdk/lib/sky2/librplogo.a(rplogo.obj)
                              obj/sky2/main.o (RpLogoPluginAttach)
E:/nightly/rwsdk.sky/rwsdk/lib/sky2/librtcharse.a(chrprint.obj)
                              obj/sky2/menu.o (RtCharsetBufferFlush)
E:/nightly/rwsdk.sky/rwsdk/lib/sky2/librtcharse.a(rtcharse.obj)
                              obj/sky2/main.o (RtCharsetCreate)
E:/nightly/rwsdk.sky/rwsdk/lib/sky2/librtpng.a(rtpng.obj)
                              obj/sky2/skeleton.o (RtPNGImageRead)
E:/nightly/rwsdk.sky/rwsdk/lib/sky2/librtpng.a(png.obj)
                              E:/nightly/rwsdk.sky/rwsdk/lib/sky2/librtpng.a(rtpng.obj) (png_create_info_struct)
E:/nightly/rwsdk.sky/rwsdk/lib/sky2/librtpng.a(pngerror.obj)
                              E:/nightly/rwsdk.sky/rwsdk/lib/sky2/librtpng.a(rtpng.obj) (png_error)
E:/nightly/rwsdk.sky/rwsdk/lib/sky2/librtpng.a(pngget.obj)
                              E:/nightly/rwsdk.sky/rwsdk/lib/sky2/librtpng.a(rtpng.obj) (png_get_valid)
E:/nightly/rwsdk.sky/rwsdk/lib/sky2/librtpng.a(pngmem.obj)
                              E:/nightly/rwsdk.sky/rwsdk/lib/sky2/librtpng.a(png.obj) (png_malloc)
E:/nightly/rwsdk.sky/rwsdk/lib/sky2/librtpng.a(pngread.obj)
                              E:/nightly/rwsdk.sky/rwsdk/lib/sky2/librtpng.a(rtpng.obj) (png_create_read_struct_2)
E:/nightly/rwsdk.sky/rwsdk/lib/sky2/librtpng.a(pngrio.obj)
                              E:/nightly/rwsdk.sky/rwsdk/lib/sky2/librtpng.a(rtpng.obj) (png_set_read_fn)
E:/nightly/rwsdk.sky/rwsdk/lib/sky2/librtpng.a(pngrtran.obj)
                              E:/nightly/rwsdk.sky/rwsdk/lib/sky2/librtpng.a(pngread.obj) (png_read_transform_info)
E:/nightly/rwsdk.sky/rwsdk/lib/sky2/librtpng.a(pngrutil.obj)
                              E:/nightly/rwsdk.sky/rwsdk/lib/sky2/librtpng.a(pngread.obj) (png_handle_IHDR)
E:/nightly/rwsdk.sky/rwsdk/lib/sky2/librtpng.a(pngset.obj)
                              E:/nightly/rwsdk.sky/rwsdk/lib/sky2/librtpng.a(pngrutil.obj) (png_set_cHRM)
E:/nightly/rwsdk.sky/rwsdk/lib/sky2/librtpng.a(pngtrans.obj)
                              E:/nightly/rwsdk.sky/rwsdk/lib/sky2/librtpng.a(pngrtran.obj) (png_do_strip_filler)
E:/nightly/rwsdk.sky/rwsdk/lib/sky2/librtpng.a(pngwio.obj)
                              E:/nightly/rwsdk.sky/rwsdk/lib/sky2/librtpng.a(rtpng.obj) (png_set_write_fn)
E:/nightly/rwsdk.sky/rwsdk/lib/sky2/librtpng.a(pngwrite.obj)
                              E:/nightly/rwsdk.sky/rwsdk/lib/sky2/librtpng.a(rtpng.obj) (png_write_info)
E:/nightly/rwsdk.sky/rwsdk/lib/sky2/librtpng.a(pngwtran.obj)
                              E:/nightly/rwsdk.sky/rwsdk/lib/sky2/librtpng.a(pngwrite.obj) (png_do_write_transformations)
E:/nightly/rwsdk.sky/rwsdk/lib/sky2/librtpng.a(pngwutil.obj)
                              E:/nightly/rwsdk.sky/rwsdk/lib/sky2/librtpng.a(pngwrite.obj) (png_write_IHDR)
E:/nightly/rwsdk.sky/rwsdk/lib/sky2/librtpng.a(deflate.obj)
                              E:/nightly/rwsdk.sky/rwsdk/lib/sky2/librtpng.a(pngwutil.obj) (deflateInit2_)
E:/nightly/rwsdk.sky/rwsdk/lib/sky2/librtpng.a(trees.obj)
                              E:/nightly/rwsdk.sky/rwsdk/lib/sky2/librtpng.a(deflate.obj) (_dist_code)
E:/nightly/rwsdk.sky/rwsdk/lib/sky2/librtpng.a(zutil.obj)
                              E:/nightly/rwsdk.sky/rwsdk/lib/sky2/librtpng.a(deflate.obj) (z_errmsg)
E:/nightly/rwsdk.sky/rwsdk/lib/sky2/librtpng.a(inflate.obj)
                              E:/nightly/rwsdk.sky/rwsdk/lib/sky2/librtpng.a(pngread.obj) (inflate)
E:/nightly/rwsdk.sky/rwsdk/lib/sky2/librtpng.a(infblock.obj)
                              E:/nightly/rwsdk.sky/rwsdk/lib/sky2/librtpng.a(inflate.obj) (inflate_blocks_new)
E:/nightly/rwsdk.sky/rwsdk/lib/sky2/librtpng.a(inftrees.obj)
                              E:/nightly/rwsdk.sky/rwsdk/lib/sky2/librtpng.a(infblock.obj) (inflate_trees_bits)
E:/nightly/rwsdk.sky/rwsdk/lib/sky2/librtpng.a(infcodes.obj)
                              E:/nightly/rwsdk.sky/rwsdk/lib/sky2/librtpng.a(infblock.obj) (inflate_codes)
E:/nightly/rwsdk.sky/rwsdk/lib/sky2/librtpng.a(infutil.obj)
                              E:/nightly/rwsdk.sky/rwsdk/lib/sky2/librtpng.a(infblock.obj) (inflate_mask)
E:/nightly/rwsdk.sky/rwsdk/lib/sky2/librtpng.a(inffast.obj)
                              E:/nightly/rwsdk.sky/rwsdk/lib/sky2/librtpng.a(infcodes.obj) (inflate_fast)
E:/nightly/rwsdk.sky/rwsdk/lib/sky2/librtpng.a(crc32.obj)
                              E:/nightly/rwsdk.sky/rwsdk/lib/sky2/librtpng.a(png.obj) (crc32)
E:/nightly/rwsdk.sky/rwsdk/lib/sky2/librtpng.a(adler32.obj)
                              E:/nightly/rwsdk.sky/rwsdk/lib/sky2/librtpng.a(deflate.obj) (adler32)
E:/nightly/rwsdk.sky/rwsdk/lib/sky2/librtbmp.a(rtbmp.obj)
                              obj/sky2/skeleton.o (RtBMPImageRead)
E:/nightly/rwsdk.sky/rwsdk/lib/sky2/librwcore.a(babinary.obj)
                              E:/nightly/rwsdk.sky/rwsdk/lib/sky2/librtbmp.a(rtbmp.obj) (RwMemNative32)
E:/nightly/rwsdk.sky/rwsdk/lib/sky2/librwcore.a(bacamera.obj)
                              obj/sky2/camera.o (RwCameraCreate)
E:/nightly/rwsdk.sky/rwsdk/lib/sky2/librwcore.a(badevice.obj)
                              obj/sky2/skyfs.o (RwEngineRegisterPlugin)
E:/nightly/rwsdk.sky/rwsdk/lib/sky2/librwcore.a(baerr.obj)
                              E:/nightly/rwsdk.sky/rwsdk/lib/sky2/librplogo.a(rplogo.obj) (_rwerror)
E:/nightly/rwsdk.sky/rwsdk/lib/sky2/librwcore.a(baframe.obj)
                              obj/sky2/skeleton.o (RwFrameUpdateObjects)
E:/nightly/rwsdk.sky/rwsdk/lib/sky2/librwcore.a(bafsys.obj)
                              E:/nightly/rwsdk.sky/rwsdk/lib/sky2/librwcore.a(badevice.obj) (_rwFileSystemOpen)
E:/nightly/rwsdk.sky/rwsdk/lib/sky2/librwcore.a(baimage.obj)
                              E:/nightly/rwsdk.sky/rwsdk/lib/sky2/librwcore.a(badevice.obj) (_rwImageOpen)
E:/nightly/rwsdk.sky/rwsdk/lib/sky2/librwcore.a(baimmedi.obj)
                              E:/nightly/rwsdk.sky/rwsdk/lib/sky2/librplogo.a(rplogo.obj) (RwIm2DGetNearScreenZ)
E:/nightly/rwsdk.sky/rwsdk/lib/sky2/librwcore.a(baimras.obj)
                              obj/sky2/sky.o (RwImageSetFromRaster)
E:/nightly/rwsdk.sky/rwsdk/lib/sky2/librwcore.a(bamatrix.obj)
                              E:/nightly/rwsdk.sky/rwsdk/lib/sky2/librwcore.a(bacamera.obj) (RwMatrixOptimize)
E:/nightly/rwsdk.sky/rwsdk/lib/sky2/librwcore.a(bamemory.obj)
                              E:/nightly/rwsdk.sky/rwsdk/lib/sky2/librwcore.a(badevice.obj) (_rwFreeListAllocReal)
E:/nightly/rwsdk.sky/rwsdk/lib/sky2/librwcore.a(baraster.obj)
                              E:/nightly/rwsdk.sky/rwsdk/lib/sky2/librwcore.a(badevice.obj) (_rwRasterOpen)
E:/nightly/rwsdk.sky/rwsdk/lib/sky2/librwcore.a(baresamp.obj)
                              E:/nightly/rwsdk.sky/rwsdk/lib/sky2/librplogo.a(rplogo.obj) (RwImageResample)
E:/nightly/rwsdk.sky/rwsdk/lib/sky2/librwcore.a(baresour.obj)
                              E:/nightly/rwsdk.sky/rwsdk/lib/sky2/librwcore.a(badevice.obj) (_rwResourcesOpen)
E:/nightly/rwsdk.sky/rwsdk/lib/sky2/librwcore.a(bastream.obj)
                              E:/nightly/rwsdk.sky/rwsdk/lib/sky2/librtpng.a(rtpng.obj) (RwStreamRead)
E:/nightly/rwsdk.sky/rwsdk/lib/sky2/librwcore.a(basync.obj)
                              E:/nightly/rwsdk.sky/rwsdk/lib/sky2/librwcore.a(bacamera.obj) (_rwFrameSyncDirty)
E:/nightly/rwsdk.sky/rwsdk/lib/sky2/librwcore.a(batextur.obj)
                              obj/sky2/im3d.o (RwTextureRead)
E:/nightly/rwsdk.sky/rwsdk/lib/sky2/librwcore.a(batkreg.obj)
                              E:/nightly/rwsdk.sky/rwsdk/lib/sky2/librwcore.a(badevice.obj) (_rwPluginRegistryOpen)
E:/nightly/rwsdk.sky/rwsdk/lib/sky2/librwcore.a(batypehf.obj)
                              E:/nightly/rwsdk.sky/rwsdk/lib/sky2/librwcore.a(bacamera.obj) (_rwObjectHasFrameSetFrame)
E:/nightly/rwsdk.sky/rwsdk/lib/sky2/librwcore.a(bavector.obj)
                              obj/sky2/skeleton.o (RwV3dNormalize)
E:/nightly/rwsdk.sky/rwsdk/lib/sky2/librwcore.a(resmem.obj)
                              E:/nightly/rwsdk.sky/rwsdk/lib/sky2/librwcore.a(baresour.obj) (_rwResHeapAlloc)
E:/nightly/rwsdk.sky/rwsdk/lib/sky2/librwcore.a(rwstring.obj)
                              E:/nightly/rwsdk.sky/rwsdk/lib/sky2/librwcore.a(badevice.obj) (_rwStringOpen)
E:/nightly/rwsdk.sky/rwsdk/lib/sky2/librwcore.a(baim3d.obj)
                              obj/sky2/linelist.o (RwIm3DRenderIndexedPrimitive)
E:/nightly/rwsdk.sky/rwsdk/lib/sky2/librwcore.a(bapipe.obj)
                              E:/nightly/rwsdk.sky/rwsdk/lib/sky2/librwcore.a(badevice.obj) (_rwRenderPipelineOpen)
E:/nightly/rwsdk.sky/rwsdk/lib/sky2/librwcore.a(nodeClipLine.obj)
                              E:/nightly/rwsdk.sky/rwsdk/lib/sky2/librwcore.a(baim3d.obj) (RxNodeDefinitionGetClipLine)
E:/nightly/rwsdk.sky/rwsdk/lib/sky2/librwcore.a(nodeClipTriangle.obj)
                              E:/nightly/rwsdk.sky/rwsdk/lib/sky2/librwcore.a(baim3d.obj) (RxNodeDefinitionGetClipTriangle)
E:/nightly/rwsdk.sky/rwsdk/lib/sky2/librwcore.a(nodeCullTriangle.obj)
                              E:/nightly/rwsdk.sky/rwsdk/lib/sky2/librwcore.a(baim3d.obj) (RxNodeDefinitionGetCullTriangle)
E:/nightly/rwsdk.sky/rwsdk/lib/sky2/librwcore.a(nodeImmInstance.obj)
                              E:/nightly/rwsdk.sky/rwsdk/lib/sky2/librwcore.a(baim3d.obj) (RxNodeDefinitionGetImmInstance)
E:/nightly/rwsdk.sky/rwsdk/lib/sky2/librwcore.a(nodeImmMangleLineIndices.obj)
                              E:/nightly/rwsdk.sky/rwsdk/lib/sky2/librwcore.a(baim3d.obj) (RxNodeDefinitionGetImmMangleLineIndices)
E:/nightly/rwsdk.sky/rwsdk/lib/sky2/librwcore.a(nodeImmMangleTriangleIndices.obj)
                              E:/nightly/rwsdk.sky/rwsdk/lib/sky2/librwcore.a(baim3d.obj) (RxNodeDefinitionGetImmMangleTriangleIndices)
E:/nightly/rwsdk.sky/rwsdk/lib/sky2/librwcore.a(nodeImmRenderSetup.obj)
                              E:/nightly/rwsdk.sky/rwsdk/lib/sky2/librwcore.a(baim3d.obj) (RxNodeDefinitionGetImmRenderSetup)
E:/nightly/rwsdk.sky/rwsdk/lib/sky2/librwcore.a(nodeImmStash.obj)
                              E:/nightly/rwsdk.sky/rwsdk/lib/sky2/librwcore.a(baim3d.obj) (RxNodeDefinitionGetImmStash)
E:/nightly/rwsdk.sky/rwsdk/lib/sky2/librwcore.a(nodeSubmitLine.obj)
                              E:/nightly/rwsdk.sky/rwsdk/lib/sky2/librwcore.a(baim3d.obj) (RxNodeDefinitionGetSubmitLine)
E:/nightly/rwsdk.sky/rwsdk/lib/sky2/librwcore.a(nodeSubmitTriangle.obj)
                              E:/nightly/rwsdk.sky/rwsdk/lib/sky2/librwcore.a(baim3d.obj) (RxNodeDefinitionGetSubmitTriangle)
E:/nightly/rwsdk.sky/rwsdk/lib/sky2/librwcore.a(nodeTransform.obj)
                              E:/nightly/rwsdk.sky/rwsdk/lib/sky2/librwcore.a(baim3d.obj) (RxNodeDefinitionGetTransform)
E:/nightly/rwsdk.sky/rwsdk/lib/sky2/librwcore.a(p2altmdl.obj)
                              E:/nightly/rwsdk.sky/rwsdk/lib/sky2/librwcore.a(nodeClipLine.obj) (_rxPacketDestroy)
E:/nightly/rwsdk.sky/rwsdk/lib/sky2/librwcore.a(p2clpcom.obj)
                              E:/nightly/rwsdk.sky/rwsdk/lib/sky2/librwcore.a(nodeClipLine.obj) (_rwGeneratePerspClippedVertexZLO)
E:/nightly/rwsdk.sky/rwsdk/lib/sky2/librwcore.a(p2core.obj)
                              E:/nightly/rwsdk.sky/rwsdk/lib/sky2/librwcore.a(p2altmdl.obj) (_rxHeapGlobal)
E:/nightly/rwsdk.sky/rwsdk/lib/sky2/librwcore.a(p2define.obj)
                              E:/nightly/rwsdk.sky/rwsdk/lib/sky2/librwcore.a(baim3d.obj) (RxLockedPipeUnlock)
E:/nightly/rwsdk.sky/rwsdk/lib/sky2/librwcore.a(p2dep.obj)
                              E:/nightly/rwsdk.sky/rwsdk/lib/sky2/librwcore.a(p2define.obj) (_rxChaseDependencies)
E:/nightly/rwsdk.sky/rwsdk/lib/sky2/librwcore.a(p2heap.obj)
                              E:/nightly/rwsdk.sky/rwsdk/lib/sky2/librwcore.a(baim3d.obj) (RxHeapAlloc)
E:/nightly/rwsdk.sky/rwsdk/lib/sky2/librwcore.a(p2renderstate.obj)
                              E:/nightly/rwsdk.sky/rwsdk/lib/sky2/librwcore.a(p2core.obj) (RxRenderStateVectorSetDefaultRenderStateVector)
E:/nightly/rwsdk.sky/rwsdk/lib/sky2/librwcore.a(p2resort.obj)
                              E:/nightly/rwsdk.sky/rwsdk/lib/sky2/librwcore.a(p2dep.obj) (_rx_rxRadixExchangeSort)
E:/nightly/rwsdk.sky/rwsdk/lib/sky2/librwcore.a(p2stdcls.obj)
                              E:/nightly/rwsdk.sky/rwsdk/lib/sky2/librwcore.a(nodeImmInstance.obj) (RxClObjSpace3DVertices)
E:/nightly/rwsdk.sky/rwsdk/lib/sky2/librwcore.a(im3dpipe.obj)
                              E:/nightly/rwsdk.sky/rwsdk/lib/sky2/librwcore.a(baim3d.obj) (_rwIm3DCreatePlatformTransformPipeline)
E:/nightly/rwsdk.sky/rwsdk/lib/sky2/librwcore.a(basky.obj)
                              E:/nightly/rwsdk.sky/rwsdk/lib/sky2/librwcore.a(badevice.obj) (_rwDeviceGetHandle)
E:/nightly/rwsdk.sky/rwsdk/lib/sky2/librwcore.a(baskytran.obj)
                              E:/nightly/rwsdk.sky/rwsdk/lib/sky2/librwcore.a(basky.obj) (matrixASMMult)
E:/nightly/rwsdk.sky/rwsdk/lib/sky2/librwcore.a(skyblit.obj)
                              E:/nightly/rwsdk.sky/rwsdk/lib/sky2/librwcore.a(basky.obj) (_rwSkyRasterClearRect)
E:/nightly/rwsdk.sky/rwsdk/lib/sky2/librwcore.a(skyconv.obj)
                              E:/nightly/rwsdk.sky/rwsdk/lib/sky2/librwcore.a(basky.obj) (_rwSkyImageFindRasterFormat)
E:/nightly/rwsdk.sky/rwsdk/lib/sky2/librwcore.a(skyinst.obj)
                              E:/nightly/rwsdk.sky/rwsdk/lib/sky2/librwcore.a(basky.obj) (skyTransType)
E:/nightly/rwsdk.sky/rwsdk/lib/sky2/librwcore.a(texcache.obj)
                              E:/nightly/rwsdk.sky/rwsdk/lib/sky2/librwcore.a(basky.obj) (skyPrepareUploadRaster)
E:/nightly/rwsdk.sky/rwsdk/lib/sky2/librwcore.a(imrascnv.obj)
                              E:/nightly/rwsdk.sky/rwsdk/lib/sky2/librwcore.a(skyconv.obj) (_rwImageFindAlphaType)
E:/nightly/rwsdk.sky/rwsdk/lib/sky2/librwcore.a(palquant.obj)
                              E:/nightly/rwsdk.sky/rwsdk/lib/sky2/librwcore.a(batextur.obj) (_rwPalQuantAddImage)
E:/nightly/rwsdk.sky/rwsdk/lib/sky2/librwcore.a(osintf.obj)
                              E:/nightly/rwsdk.sky/rwsdk/lib/sky2/librwcore.a(baimage.obj) (_rwpathisabsolute)
E:/nightly/rwsdk.sky/rwsdk/lib/sky2/librwcore.a(babbox.obj)
                              E:/nightly/rwsdk.sky/rwsdk/lib/sky2/librwcore.a(bacamera.obj) (RwBBoxCalculate)
E:/nightly/rwsdk.sky/rwsdk/lib/sky2/librwcore.a(babintex.obj)
                              E:/nightly/rwsdk.sky/rwsdk/lib/sky2/librwcore.a(basky.obj) (_rwStringStreamFindAndRead)
E:/nightly/rwsdk.sky/rwsdk/lib/sky2/librwcore.a(bacolor.obj)
                              E:/nightly/rwsdk.sky/rwsdk/lib/sky2/librwcore.a(badevice.obj) (_rwColorOpen)
E:/nightly/rwsdk.sky/rwsdk/lib/sky2/librwcore.a(batkbin.obj)
                              E:/nightly/rwsdk.sky/rwsdk/lib/sky2/librwcore.a(babintex.obj) (_rwPluginRegistryReadDataChunks)
E:/nightly/rwsdk.sky/rwsdk/lib/sky2/librwcore.a(GenericPRS.obj)
                              E:/nightly/rwsdk.sky/rwsdk/lib/sky2/librwcore.a(skyinst.obj) (vu1GenericPRS)
E:/nightly/rwsdk.sky/rwsdk/lib/sky2/librwcore.a(SegmentsPRL.obj)
                              E:/nightly/rwsdk.sky/rwsdk/lib/sky2/librwcore.a(skyinst.obj) (vu1SegmentsPRL)
E:/nightly/rwsdk.sky/rwsdk/lib/sky2/librwcore.a(SegmentsPRS.obj)
                              E:/nightly/rwsdk.sky/rwsdk/lib/sky2/librwcore.a(skyinst.obj) (vu1SegmentsPRS)
E:/nightly/rwsdk.sky/rwsdk/lib/sky2/librwcore.a(baasm.obj)
                              E:/nightly/rwsdk.sky/rwsdk/lib/sky2/librwcore.a(basky.obj) (gs_set_up)
E:/nightly/rwsdk.sky/rwsdk/lib/sky2/librwcore.a(baim2dll.obj)
                              E:/nightly/rwsdk.sky/rwsdk/lib/sky2/librwcore.a(skyinst.obj) (vu1im2dll)
E:/nightly/rwsdk.sky/rwsdk/lib/sky2/librwcore.a(baim2dtl.obj)
                              E:/nightly/rwsdk.sky/rwsdk/lib/sky2/librwcore.a(skyinst.obj) (vu1im2dtl)
E:/nightly/rwsdk.sky/rwsdk/lib/sky2/librwcore.a(banfim2dll.obj)
                              E:/nightly/rwsdk.sky/rwsdk/lib/sky2/librwcore.a(skyinst.obj) (vu1nfim2dll)
E:/nightly/rwsdk.sky/rwsdk/lib/sky2/librwcore.a(banfim2dtl.obj)
                              E:/nightly/rwsdk.sky/rwsdk/lib/sky2/librwcore.a(skyinst.obj) (vu1nfim2dtl)
E:/nightly/rwsdk.sky/rwsdk/lib/sky2/librwcore.a(badma.obj)
                              E:/nightly/rwsdk.sky/rwsdk/lib/sky2/librwcore.a(basky.obj) (sweMaxFlips)
E:/nightly/rwsdk.sky/rwsdk/lib/sky2/librwcore.a(baevent.obj)
                              E:/nightly/rwsdk.sky/rwsdk/lib/sky2/librwcore.a(basky.obj) (_rwSkyInitConfigSystem)
E:/nightly/rwsdk.sky/rwsdk/lib/sky2/librwcore.a(dmaalloc.obj)
                              E:/nightly/rwsdk.sky/rwsdk/lib/sky2/librwcore.a(badma.obj) (sweCircAllocBlockSize)
E:/usr/local/sce/ee/lib/libgraph.a(graph001.o)
                              E:/nightly/rwsdk.sky/rwsdk/lib/sky2/librwcore.a(basky.obj) (sceGsResetGraph)
E:/usr/local/sce/ee/lib/libgraph.a(graph002.o)
                              E:/nightly/rwsdk.sky/rwsdk/lib/sky2/librwcore.a(baevent.obj) (sceGsResetPath)
E:/usr/local/sce/ee/lib/libgraph.a(graph011.o)
                              E:/nightly/rwsdk.sky/rwsdk/lib/sky2/librwcore.a(basky.obj) (sceGsSyncV)
E:/usr/local/sce/ee/lib/libgraph.a(graph012.o)
                              E:/nightly/rwsdk.sky/rwsdk/lib/sky2/librwcore.a(basky.obj) (sceGsSyncPath)
E:/usr/local/sce/ee/lib/libgraph.a(graph016.o)
                              E:/nightly/rwsdk.sky/rwsdk/lib/sky2/librwcore.a(basky.obj) (sceGsSetDefStoreImage)
E:/usr/local/sce/ee/lib/libgraph.a(graph018.o)
                              E:/nightly/rwsdk.sky/rwsdk/lib/sky2/librwcore.a(basky.obj) (sceGsExecStoreImage)
E:/usr/local/sce/ee/lib/libgraph.a(graph021.o)
                              E:/nightly/rwsdk.sky/rwsdk/lib/sky2/librwcore.a(badma.obj) (sceGsSetHalfOffset)
E:/usr/local/sce/ee/lib/libgraph.a(graph026.o)
                              E:/nightly/rwsdk.sky/rwsdk/lib/sky2/librwcore.a(badma.obj) (sceGsSetHalfOffset2)
E:/usr/local/sce/ee/lib/libgraph.a(graph027.o)
                              E:/nightly/rwsdk.sky/rwsdk/lib/sky2/librwcore.a(basky.obj) (sceGsSetDefDBuffDc)
E:/usr/local/sce/ee/lib/libgraph.a(graph028.o)
                              E:/nightly/rwsdk.sky/rwsdk/lib/sky2/librwcore.a(basky.obj) (sceGsSwapDBuffDc)
E:/usr/local/sce/ee/lib/libgraph.a(graph003.o)
                              E:/usr/local/sce/ee/lib/libgraph.a(graph027.o) (sceGsSetDefDispEnv)
E:/usr/local/sce/ee/lib/libgraph.a(graph004.o)
                              E:/usr/local/sce/ee/lib/libgraph.a(graph028.o) (sceGsPutDispEnv)
E:/usr/local/sce/ee/lib/libgraph.a(graph005.o)
                              E:/usr/local/sce/ee/lib/libgraph.a(graph027.o) (sceGszbufaddr)
E:/usr/local/sce/ee/lib/libgraph.a(graph006.o)
                              E:/usr/local/sce/ee/lib/libgraph.a(graph027.o) (sceGsSetDefDrawEnv)
E:/usr/local/sce/ee/lib/libgraph.a(graph007.o)
                              E:/usr/local/sce/ee/lib/libgraph.a(graph027.o) (sceGsSetDefClear)
E:/usr/local/sce/ee/lib/libgraph.a(graph008.o)
                              E:/usr/local/sce/ee/lib/libgraph.a(graph028.o) (sceGsPutDrawEnv)
E:/usr/local/sce/ee/lib/libgraph.a(graph022.o)
                              E:/usr/local/sce/ee/lib/libgraph.a(graph027.o) (sceGsSetDefDrawEnv2)
E:/usr/local/sce/ee/lib/libdma.a(libdma.o)
                              E:/nightly/rwsdk.sky/rwsdk/lib/sky2/librwcore.a(basky.obj) (sceDmaGetChan)
E:/usr/local/sce/ee/lib/libpad.a(libpad.o)
                              obj/sky2/sky.o (scePadInit)
E:/usr/local/sce/ee/gcc/lib/gcc-lib/ee\2.95.2\../../../../ee\lib\libm.a(sf_ceil.o)
                              obj/sky2/sky.o (ceilf)
E:/usr/local/sce/ee/gcc/lib/gcc-lib/ee\2.95.2\../../../../ee\lib\libm.a(sf_cos.o)
                              E:/nightly/rwsdk.sky/rwsdk/lib/sky2/librwcore.a(bamatrix.obj) (cosf)
E:/usr/local/sce/ee/gcc/lib/gcc-lib/ee\2.95.2\../../../../ee\lib\libm.a(sf_sin.o)
                              E:/nightly/rwsdk.sky/rwsdk/lib/sky2/librwcore.a(bamatrix.obj) (sinf)
E:/usr/local/sce/ee/gcc/lib/gcc-lib/ee\2.95.2\../../../../ee\lib\libm.a(w_pow.o)
                              E:/nightly/rwsdk.sky/rwsdk/lib/sky2/librtpng.a(pngrtran.obj) (pow)
E:/usr/local/sce/ee/gcc/lib/gcc-lib/ee\2.95.2\../../../../ee\lib\libm.a(wf_acos.o)
                              obj/sky2/skeleton.o (acosf)
E:/usr/local/sce/ee/gcc/lib/gcc-lib/ee\2.95.2\../../../../ee\lib\libm.a(wf_atan2.o)
                              E:/nightly/rwsdk.sky/rwsdk/lib/sky2/librwcore.a(bamatrix.obj) (atan2f)
E:/usr/local/sce/ee/gcc/lib/gcc-lib/ee\2.95.2\../../../../ee\lib\libm.a(wf_pow.o)
                              E:/nightly/rwsdk.sky/rwsdk/lib/sky2/librwcore.a(baimage.obj) (powf)
E:/usr/local/sce/ee/gcc/lib/gcc-lib/ee\2.95.2\../../../../ee\lib\libm.a(e_pow.o)
                              E:/usr/local/sce/ee/gcc/lib/gcc-lib/ee\2.95.2\../../../../ee\lib\libm.a(w_pow.o) (__ieee754_pow)
E:/usr/local/sce/ee/gcc/lib/gcc-lib/ee\2.95.2\../../../../ee\lib\libm.a(e_sqrt.o)
                              E:/usr/local/sce/ee/gcc/lib/gcc-lib/ee\2.95.2\../../../../ee\lib\libm.a(e_pow.o) (__ieee754_sqrt)
E:/usr/local/sce/ee/gcc/lib/gcc-lib/ee\2.95.2\../../../../ee\lib\libm.a(ef_acos.o)
                              E:/usr/local/sce/ee/gcc/lib/gcc-lib/ee\2.95.2\../../../../ee\lib\libm.a(wf_acos.o) (__ieee754_acosf)
E:/usr/local/sce/ee/gcc/lib/gcc-lib/ee\2.95.2\../../../../ee\lib\libm.a(ef_atan2.o)
                              E:/usr/local/sce/ee/gcc/lib/gcc-lib/ee\2.95.2\../../../../ee\lib\libm.a(wf_atan2.o) (__ieee754_atan2f)
E:/usr/local/sce/ee/gcc/lib/gcc-lib/ee\2.95.2\../../../../ee\lib\libm.a(ef_pow.o)
                              E:/usr/local/sce/ee/gcc/lib/gcc-lib/ee\2.95.2\../../../../ee\lib\libm.a(wf_pow.o) (__ieee754_powf)
E:/usr/local/sce/ee/gcc/lib/gcc-lib/ee\2.95.2\../../../../ee\lib\libm.a(ef_rem_pio2.o)
                              E:/usr/local/sce/ee/gcc/lib/gcc-lib/ee\2.95.2\../../../../ee\lib\libm.a(sf_cos.o) (__ieee754_rem_pio2f)
E:/usr/local/sce/ee/gcc/lib/gcc-lib/ee\2.95.2\../../../../ee\lib\libm.a(ef_sqrt.o)
                              E:/usr/local/sce/ee/gcc/lib/gcc-lib/ee\2.95.2\../../../../ee\lib\libm.a(ef_acos.o) (__ieee754_sqrtf)
E:/usr/local/sce/ee/gcc/lib/gcc-lib/ee\2.95.2\../../../../ee\lib\libm.a(kf_cos.o)
                              E:/usr/local/sce/ee/gcc/lib/gcc-lib/ee\2.95.2\../../../../ee\lib\libm.a(sf_cos.o) (__kernel_cosf)
E:/usr/local/sce/ee/gcc/lib/gcc-lib/ee\2.95.2\../../../../ee\lib\libm.a(kf_rem_pio2.o)
                              E:/usr/local/sce/ee/gcc/lib/gcc-lib/ee\2.95.2\../../../../ee\lib\libm.a(ef_rem_pio2.o) (__kernel_rem_pio2f)
E:/usr/local/sce/ee/gcc/lib/gcc-lib/ee\2.95.2\../../../../ee\lib\libm.a(kf_sin.o)
                              E:/usr/local/sce/ee/gcc/lib/gcc-lib/ee\2.95.2\../../../../ee\lib\libm.a(sf_cos.o) (__kernel_sinf)
E:/usr/local/sce/ee/gcc/lib/gcc-lib/ee\2.95.2\../../../../ee\lib\libm.a(s_fabs.o)
                              E:/usr/local/sce/ee/gcc/lib/gcc-lib/ee\2.95.2\../../../../ee\lib\libm.a(e_pow.o) (fabs)
E:/usr/local/sce/ee/gcc/lib/gcc-lib/ee\2.95.2\../../../../ee\lib\libm.a(s_finite.o)
                              E:/usr/local/sce/ee/gcc/lib/gcc-lib/ee\2.95.2\../../../../ee\lib\libm.a(w_pow.o) (finite)
E:/usr/local/sce/ee/gcc/lib/gcc-lib/ee\2.95.2\../../../../ee\lib\libm.a(s_infconst.o)
                              E:/usr/local/sce/ee/gcc/lib/gcc-lib/ee\2.95.2\../../../../ee\lib\libm.a(w_pow.o) (__infinity)
E:/usr/local/sce/ee/gcc/lib/gcc-lib/ee\2.95.2\../../../../ee\lib\libm.a(s_isnan.o)
                              E:/usr/local/sce/ee/gcc/lib/gcc-lib/ee\2.95.2\../../../../ee\lib\libm.a(w_pow.o) (isnan)
E:/usr/local/sce/ee/gcc/lib/gcc-lib/ee\2.95.2\../../../../ee\lib\libm.a(s_lib_ver.o)
                              E:/usr/local/sce/ee/gcc/lib/gcc-lib/ee\2.95.2\../../../../ee\lib\libm.a(w_pow.o) (__fdlib_version)
E:/usr/local/sce/ee/gcc/lib/gcc-lib/ee\2.95.2\../../../../ee\lib\libm.a(s_matherr.o)
                              E:/usr/local/sce/ee/gcc/lib/gcc-lib/ee\2.95.2\../../../../ee\lib\libm.a(w_pow.o) (matherr)
E:/usr/local/sce/ee/gcc/lib/gcc-lib/ee\2.95.2\../../../../ee\lib\libm.a(s_rint.o)
                              E:/usr/local/sce/ee/gcc/lib/gcc-lib/ee\2.95.2\../../../../ee\lib\libm.a(w_pow.o) (rint)
E:/usr/local/sce/ee/gcc/lib/gcc-lib/ee\2.95.2\../../../../ee\lib\libm.a(s_scalbn.o)
                              E:/usr/local/sce/ee/gcc/lib/gcc-lib/ee\2.95.2\../../../../ee\lib\libm.a(e_pow.o) (scalbn)
E:/usr/local/sce/ee/gcc/lib/gcc-lib/ee\2.95.2\../../../../ee\lib\libm.a(sf_atan.o)
                              E:/usr/local/sce/ee/gcc/lib/gcc-lib/ee\2.95.2\../../../../ee\lib\libm.a(ef_atan2.o) (atanf)
E:/usr/local/sce/ee/gcc/lib/gcc-lib/ee\2.95.2\../../../../ee\lib\libm.a(sf_fabs.o)
                              E:/usr/local/sce/ee/gcc/lib/gcc-lib/ee\2.95.2\../../../../ee\lib\libm.a(wf_acos.o) (fabsf)
E:/usr/local/sce/ee/gcc/lib/gcc-lib/ee\2.95.2\../../../../ee\lib\libm.a(sf_finite.o)
                              E:/usr/local/sce/ee/gcc/lib/gcc-lib/ee\2.95.2\../../../../ee\lib\libm.a(wf_pow.o) (finitef)
E:/usr/local/sce/ee/gcc/lib/gcc-lib/ee\2.95.2\../../../../ee\lib\libm.a(sf_floor.o)
                              E:/usr/local/sce/ee/gcc/lib/gcc-lib/ee\2.95.2\../../../../ee\lib\libm.a(kf_rem_pio2.o) (floorf)
E:/usr/local/sce/ee/gcc/lib/gcc-lib/ee\2.95.2\../../../../ee\lib\libm.a(sf_isnan.o)
                              E:/usr/local/sce/ee/gcc/lib/gcc-lib/ee\2.95.2\../../../../ee\lib\libm.a(wf_acos.o) (isnanf)
E:/usr/local/sce/ee/gcc/lib/gcc-lib/ee\2.95.2\../../../../ee\lib\libm.a(sf_scalbn.o)
                              E:/usr/local/sce/ee/gcc/lib/gcc-lib/ee\2.95.2\../../../../ee\lib\libm.a(ef_pow.o) (scalbnf)
E:/usr/local/sce/ee/gcc/lib/gcc-lib/ee\2.95.2\../../../../ee\lib\libm.a(s_copysign.o)
                              E:/usr/local/sce/ee/gcc/lib/gcc-lib/ee\2.95.2\../../../../ee\lib\libm.a(s_scalbn.o) (copysign)
E:/usr/local/sce/ee/gcc/lib/gcc-lib/ee\2.95.2\../../../../ee\lib\libm.a(sf_copysign.o)
                              E:/usr/local/sce/ee/gcc/lib/gcc-lib/ee\2.95.2\../../../../ee\lib\libm.a(sf_scalbn.o) (copysignf)
E:/usr/local/sce/ee/gcc/lib/gcc-lib/ee\2.95.2\libgcc.a(__main.o)
                              obj/sky2/sky.o (__main)
E:/usr/local/sce/ee/gcc/lib/gcc-lib/ee\2.95.2\libgcc.a(_ctors.o)
                              E:/usr/local/sce/ee/gcc/lib/gcc-lib/ee\2.95.2\libgcc.a(__main.o) (__CTOR_LIST__)
E:/usr/local/sce/ee/gcc/lib/gcc-lib/ee\2.95.2\libgcc.a(_fixdfdi.o)
                              E:/nightly/rwsdk.sky/rwsdk/lib/sky2/librtpng.a(pngset.obj) (__fixdfdi)
E:/usr/local/sce/ee/gcc/lib/gcc-lib/ee\2.95.2\libgcc.a(_fixunsdfdi.o)
                              E:/nightly/rwsdk.sky/rwsdk/lib/sky2/librtpng.a(pngrtran.obj) (__fixunsdfdi)
E:/usr/local/sce/ee/gcc/lib/gcc-lib/ee\2.95.2\libgcc.a(_floatdidf.o)
                              E:/nightly/rwsdk.sky/rwsdk/lib/sky2/librtpng.a(pngrtran.obj) (__floatdidf)
E:/usr/local/sce/ee/gcc/lib/gcc-lib/ee\2.95.2\libgcc.a(_floatdisf.o)
                              E:/nightly/rwsdk.sky/rwsdk/lib/sky2/librtpng.a(pngget.obj) (__floatdisf)
E:/usr/local/sce/ee/gcc/lib/gcc-lib/ee\2.95.2\libgcc.a(_muldi3.o)
                              E:/nightly/rwsdk.sky/rwsdk/lib/sky2/librtpng.a(pngread.obj) (__muldi3)
E:/usr/local/sce/ee/gcc/lib/gcc-lib/ee\2.95.2\libgcc.a(_udivdi3.o)
                              obj/sky2/sky.o (__udivdi3)
E:/usr/local/sce/ee/gcc/lib/gcc-lib/ee\2.95.2\libgcc.a(_umoddi3.o)
                              E:/nightly/rwsdk.sky/rwsdk/lib/sky2/librtpng.a(pngrtran.obj) (__umoddi3)
E:/usr/local/sce/ee/gcc/lib/gcc-lib/ee\2.95.2\libgcc.a(dp-bit.o)
                              E:/nightly/rwsdk.sky/rwsdk/lib/sky2/librtpng.a(pngrtran.obj) (dpadd)
E:/usr/local/sce/ee/gcc/lib/gcc-lib/ee\2.95.2\libgcc.a(fp-bit.o)
                              E:/usr/local/sce/ee/gcc/lib/gcc-lib/ee\2.95.2\libgcc.a(dp-bit.o) (__make_fp)
E:/usr/local/sce/ee/gcc/lib/gcc-lib/ee\2.95.2\../../../../ee\lib\libc.a(calloc.o)
                              E:/nightly/rwsdk.sky/rwsdk/lib/sky2/librtpng.a(zutil.obj) (calloc)
E:/usr/local/sce/ee/gcc/lib/gcc-lib/ee\2.95.2\../../../../ee\lib\libc.a(callocr.o)
                              E:/usr/local/sce/ee/gcc/lib/gcc-lib/ee\2.95.2\../../../../ee\lib\libc.a(calloc.o) (_calloc_r)
E:/usr/local/sce/ee/gcc/lib/gcc-lib/ee\2.95.2\../../../../ee\lib\libc.a(ctype_.o)
                              obj/sky2/skeleton.o (_ctype_)
E:/usr/local/sce/ee/gcc/lib/gcc-lib/ee\2.95.2\../../../../ee\lib\libc.a(errno.o)
                              E:/usr/local/sce/ee/gcc/lib/gcc-lib/ee\2.95.2\../../../../ee\lib\libm.a(w_pow.o) (__errno)
E:/usr/local/sce/ee/gcc/lib/gcc-lib/ee\2.95.2\../../../../ee\lib\libc.a(fclose.o)
                              E:/nightly/rwsdk.sky/rwsdk/lib/sky2/librwcore.a(bafsys.obj) (fclose)
E:/usr/local/sce/ee/gcc/lib/gcc-lib/ee\2.95.2\../../../../ee\lib\libc.a(feof.o)
                              E:/nightly/rwsdk.sky/rwsdk/lib/sky2/librwcore.a(bafsys.obj) (feof)
E:/usr/local/sce/ee/gcc/lib/gcc-lib/ee\2.95.2\../../../../ee\lib\libc.a(fflush.o)
                              E:/nightly/rwsdk.sky/rwsdk/lib/sky2/librwcore.a(bafsys.obj) (fflush)
E:/usr/local/sce/ee/gcc/lib/gcc-lib/ee\2.95.2\../../../../ee\lib\libc.a(fgets.o)
                              E:/nightly/rwsdk.sky/rwsdk/lib/sky2/librwcore.a(bafsys.obj) (fgets)
E:/usr/local/sce/ee/gcc/lib/gcc-lib/ee\2.95.2\../../../../ee\lib\libc.a(findfp.o)
                              E:/usr/local/sce/ee/gcc/lib/gcc-lib/ee\2.95.2\../../../../ee\lib\libc.a(fclose.o) (__sinit)
E:/usr/local/sce/ee/gcc/lib/gcc-lib/ee\2.95.2\../../../../ee\lib\libc.a(fopen.o)
                              E:/nightly/rwsdk.sky/rwsdk/lib/sky2/librwcore.a(bafsys.obj) (fopen)
E:/usr/local/sce/ee/gcc/lib/gcc-lib/ee\2.95.2\../../../../ee\lib\libc.a(fputs.o)
                              E:/nightly/rwsdk.sky/rwsdk/lib/sky2/librwcore.a(bafsys.obj) (fputs)
E:/usr/local/sce/ee/gcc/lib/gcc-lib/ee\2.95.2\../../../../ee\lib\libc.a(fread.o)
                              E:/nightly/rwsdk.sky/rwsdk/lib/sky2/librwcore.a(bafsys.obj) (fread)
E:/usr/local/sce/ee/gcc/lib/gcc-lib/ee\2.95.2\../../../../ee\lib\libc.a(freer.o)
                              E:/usr/local/sce/ee/gcc/lib/gcc-lib/ee\2.95.2\../../../../ee\lib\libc.a(fclose.o) (_free_r)
E:/usr/local/sce/ee/gcc/lib/gcc-lib/ee\2.95.2\../../../../ee\lib\libc.a(fseek.o)
                              E:/nightly/rwsdk.sky/rwsdk/lib/sky2/librwcore.a(bafsys.obj) (fseek)
E:/usr/local/sce/ee/gcc/lib/gcc-lib/ee\2.95.2\../../../../ee\lib\libc.a(fstatr.o)
                              E:/usr/local/sce/ee/gcc/lib/gcc-lib/ee\2.95.2\../../../../ee\lib\libc.a(fseek.o) (_fstat_r)
E:/usr/local/sce/ee/gcc/lib/gcc-lib/ee\2.95.2\../../../../ee\lib\libc.a(ftell.o)
                              E:/nightly/rwsdk.sky/rwsdk/lib/sky2/librwcore.a(bafsys.obj) (ftell)
E:/usr/local/sce/ee/gcc/lib/gcc-lib/ee\2.95.2\../../../../ee\lib\libc.a(fvwrite.o)
                              E:/usr/local/sce/ee/gcc/lib/gcc-lib/ee\2.95.2\../../../../ee\lib\libc.a(fputs.o) (__sfvwrite)
E:/usr/local/sce/ee/gcc/lib/gcc-lib/ee\2.95.2\../../../../ee\lib\libc.a(fwalk.o)
                              E:/usr/local/sce/ee/gcc/lib/gcc-lib/ee\2.95.2\../../../../ee\lib\libc.a(fflush.o) (_fwalk)
E:/usr/local/sce/ee/gcc/lib/gcc-lib/ee\2.95.2\../../../../ee\lib\libc.a(fwrite.o)
                              E:/nightly/rwsdk.sky/rwsdk/lib/sky2/librwcore.a(bafsys.obj) (fwrite)
E:/usr/local/sce/ee/gcc/lib/gcc-lib/ee\2.95.2\../../../../ee\lib\libc.a(impure.o)
                              E:/usr/local/sce/ee/gcc/lib/gcc-lib/ee\2.95.2\../../../../ee\lib\libc.a(calloc.o) (_impure_ptr)
E:/usr/local/sce/ee/gcc/lib/gcc-lib/ee\2.95.2\../../../../ee\lib\libc.a(makebuf.o)
                              E:/usr/local/sce/ee/gcc/lib/gcc-lib/ee\2.95.2\../../../../ee\lib\libc.a(fseek.o) (__smakebuf)
E:/usr/local/sce/ee/gcc/lib/gcc-lib/ee\2.95.2\../../../../ee\lib\libc.a(malloc.o)
                              obj/sky2/sky.o (malloc)
E:/usr/local/sce/ee/gcc/lib/gcc-lib/ee\2.95.2\../../../../ee\lib\libc.a(mallocr.o)
                              E:/usr/local/sce/ee/gcc/lib/gcc-lib/ee\2.95.2\../../../../ee\lib\libc.a(freer.o) (__malloc_av_)
E:/usr/local/sce/ee/gcc/lib/gcc-lib/ee\2.95.2\../../../../ee\lib\libc.a(memchr.o)
                              E:/usr/local/sce/ee/gcc/lib/gcc-lib/ee\2.95.2\../../../../ee\lib\libc.a(fgets.o) (memchr)
E:/usr/local/sce/ee/gcc/lib/gcc-lib/ee\2.95.2\../../../../ee\lib\libc.a(memcmp.o)
                              E:/nightly/rwsdk.sky/rwsdk/lib/sky2/librtpng.a(png.obj) (memcmp)
E:/usr/local/sce/ee/gcc/lib/gcc-lib/ee\2.95.2\../../../../ee\lib\libc.a(memcpy.o)
                              obj/sky2/sky.o (memcpy)
E:/usr/local/sce/ee/gcc/lib/gcc-lib/ee\2.95.2\../../../../ee\lib\libc.a(memmove.o)
                              E:/usr/local/sce/ee/gcc/lib/gcc-lib/ee\2.95.2\../../../../ee\lib\libc.a(fvwrite.o) (memmove)
E:/usr/local/sce/ee/gcc/lib/gcc-lib/ee\2.95.2\../../../../ee\lib\libc.a(memset.o)
                              obj/sky2/menu.o (memset)
E:/usr/local/sce/ee/gcc/lib/gcc-lib/ee\2.95.2\../../../../ee\lib\libc.a(mlock.o)
                              E:/usr/local/sce/ee/gcc/lib/gcc-lib/ee\2.95.2\../../../../ee\lib\libc.a(freer.o) (__malloc_lock)
E:/usr/local/sce/ee/gcc/lib/gcc-lib/ee\2.95.2\../../../../ee\lib\libc.a(openr.o)
                              E:/usr/local/sce/ee/gcc/lib/gcc-lib/ee\2.95.2\../../../../ee\lib\libc.a(fopen.o) (_open_r)
E:/usr/local/sce/ee/gcc/lib/gcc-lib/ee\2.95.2\../../../../ee\lib\libc.a(printf.o)
                              obj/sky2/sky.o (printf)
E:/usr/local/sce/ee/gcc/lib/gcc-lib/ee\2.95.2\../../../../ee\lib\libc.a(qsort.o)
                              E:/nightly/rwsdk.sky/rwsdk/lib/sky2/librwcore.a(bamemory.obj) (qsort)
E:/usr/local/sce/ee/gcc/lib/gcc-lib/ee\2.95.2\../../../../ee\lib\libc.a(realloc.o)
                              E:/nightly/rwsdk.sky/rwsdk/lib/sky2/librwcore.a(bamemory.obj) (realloc)
E:/usr/local/sce/ee/gcc/lib/gcc-lib/ee\2.95.2\../../../../ee\lib\libc.a(reallocr.o)
                              E:/usr/local/sce/ee/gcc/lib/gcc-lib/ee\2.95.2\../../../../ee\lib\libc.a(realloc.o) (_realloc_r)
E:/usr/local/sce/ee/gcc/lib/gcc-lib/ee\2.95.2\../../../../ee\lib\libc.a(refill.o)
                              E:/usr/local/sce/ee/gcc/lib/gcc-lib/ee\2.95.2\../../../../ee\lib\libc.a(fgets.o) (__srefill)
E:/usr/local/sce/ee/gcc/lib/gcc-lib/ee\2.95.2\../../../../ee\lib\libc.a(sbrkr.o)
                              E:/usr/local/sce/ee/gcc/lib/gcc-lib/ee\2.95.2\../../../../ee\lib\libc.a(freer.o) (_sbrk_r)
E:/usr/local/sce/ee/gcc/lib/gcc-lib/ee\2.95.2\../../../../ee\lib\libc.a(setjmp.o)
                              E:/nightly/rwsdk.sky/rwsdk/lib/sky2/librtpng.a(rtpng.obj) (setjmp)
E:/usr/local/sce/ee/gcc/lib/gcc-lib/ee\2.95.2\../../../../ee\lib\libc.a(sprintf.o)
                              obj/sky2/sky.o (sprintf)
E:/usr/local/sce/ee/gcc/lib/gcc-lib/ee\2.95.2\../../../../ee\lib\libc.a(sscanf.o)
                              E:/nightly/rwsdk.sky/rwsdk/lib/sky2/librwcore.a(rwstring.obj) (sscanf)
E:/usr/local/sce/ee/gcc/lib/gcc-lib/ee\2.95.2\../../../../ee\lib\libc.a(stdio.o)
                              E:/usr/local/sce/ee/gcc/lib/gcc-lib/ee\2.95.2\../../../../ee\lib\libc.a(findfp.o) (__sread)
E:/usr/local/sce/ee/gcc/lib/gcc-lib/ee\2.95.2\../../../../ee\lib\libc.a(strcat.o)
                              obj/sky2/sky.o (strcat)
E:/usr/local/sce/ee/gcc/lib/gcc-lib/ee\2.95.2\../../../../ee\lib\libc.a(strchr.o)
                              obj/sky2/skyfs.o (strchr)
E:/usr/local/sce/ee/gcc/lib/gcc-lib/ee\2.95.2\../../../../ee\lib\libc.a(strcmp.o)
                              obj/sky2/skeleton.o (strcmp)
E:/usr/local/sce/ee/gcc/lib/gcc-lib/ee\2.95.2\../../../../ee\lib\libc.a(strcpy.o)
                              obj/sky2/sky.o (strcpy)
E:/usr/local/sce/ee/gcc/lib/gcc-lib/ee\2.95.2\../../../../ee\lib\libc.a(strdup.o)
                              obj/sky2/sky.o (strdup)
E:/usr/local/sce/ee/gcc/lib/gcc-lib/ee\2.95.2\../../../../ee\lib\libc.a(strdup_r.o)
                              E:/usr/local/sce/ee/gcc/lib/gcc-lib/ee\2.95.2\../../../../ee\lib\libc.a(strdup.o) (_strdup_r)
E:/usr/local/sce/ee/gcc/lib/gcc-lib/ee\2.95.2\../../../../ee\lib\libc.a(strlen.o)
                              obj/sky2/skyfs.o (strlen)
E:/usr/local/sce/ee/gcc/lib/gcc-lib/ee\2.95.2\../../../../ee\lib\libc.a(strncat.o)
                              E:/nightly/rwsdk.sky/rwsdk/lib/sky2/librwcore.a(rwstring.obj) (strncat)
E:/usr/local/sce/ee/gcc/lib/gcc-lib/ee\2.95.2\../../../../ee\lib\libc.a(strncpy.o)
                              obj/sky2/skyfs.o (strncpy)
E:/usr/local/sce/ee/gcc/lib/gcc-lib/ee\2.95.2\../../../../ee\lib\libc.a(strrchr.o)
                              obj/sky2/skyfs.o (strrchr)
E:/usr/local/sce/ee/gcc/lib/gcc-lib/ee\2.95.2\../../../../ee\lib\libc.a(strstr.o)
                              E:/nightly/rwsdk.sky/rwsdk/lib/sky2/librwcore.a(rwstring.obj) (strstr)
E:/usr/local/sce/ee/gcc/lib/gcc-lib/ee\2.95.2\../../../../ee\lib\libc.a(strtod.o)
                              E:/nightly/rwsdk.sky/rwsdk/lib/sky2/librtpng.a(pngrutil.obj) (strtod)
E:/usr/local/sce/ee/gcc/lib/gcc-lib/ee\2.95.2\../../../../ee\lib\libc.a(strtok.o)
                              E:/nightly/rwsdk.sky/rwsdk/lib/sky2/librwcore.a(rwstring.obj) (strtok)
E:/usr/local/sce/ee/gcc/lib/gcc-lib/ee\2.95.2\../../../../ee\lib\libc.a(strtok_r.o)
                              E:/usr/local/sce/ee/gcc/lib/gcc-lib/ee\2.95.2\../../../../ee\lib\libc.a(strtok.o) (strtok_r)
E:/usr/local/sce/ee/gcc/lib/gcc-lib/ee\2.95.2\../../../../ee\lib\libc.a(vfprintf.o)
                              E:/usr/local/sce/ee/gcc/lib/gcc-lib/ee\2.95.2\../../../../ee\lib\libc.a(printf.o) (vfprintf)
E:/usr/local/sce/ee/gcc/lib/gcc-lib/ee\2.95.2\../../../../ee\lib\libc.a(vfscanf.o)
                              E:/usr/local/sce/ee/gcc/lib/gcc-lib/ee\2.95.2\../../../../ee\lib\libc.a(sscanf.o) (__svfscanf)
E:/usr/local/sce/ee/gcc/lib/gcc-lib/ee\2.95.2\../../../../ee\lib\libc.a(vsprintf.o)
                              E:/nightly/rwsdk.sky/rwsdk/lib/sky2/librwcore.a(rwstring.obj) (vsprintf)
E:/usr/local/sce/ee/gcc/lib/gcc-lib/ee\2.95.2\../../../../ee\lib\libc.a(writer.o)
                              E:/usr/local/sce/ee/gcc/lib/gcc-lib/ee\2.95.2\../../../../ee\lib\libc.a(stdio.o) (_write_r)
E:/usr/local/sce/ee/gcc/lib/gcc-lib/ee\2.95.2\../../../../ee\lib\libc.a(wsetup.o)
                              E:/usr/local/sce/ee/gcc/lib/gcc-lib/ee\2.95.2\../../../../ee\lib\libc.a(fvwrite.o) (__swsetup)
E:/usr/local/sce/ee/gcc/lib/gcc-lib/ee\2.95.2\../../../../ee\lib\libc.a(atof.o)
                              E:/usr/local/sce/ee/gcc/lib/gcc-lib/ee\2.95.2\../../../../ee\lib\libc.a(vfscanf.o) (atof)
E:/usr/local/sce/ee/gcc/lib/gcc-lib/ee\2.95.2\../../../../ee\lib\libc.a(closer.o)
                              E:/usr/local/sce/ee/gcc/lib/gcc-lib/ee\2.95.2\../../../../ee\lib\libc.a(stdio.o) (_close_r)
E:/usr/local/sce/ee/gcc/lib/gcc-lib/ee\2.95.2\../../../../ee\lib\libc.a(dtoa.o)
                              E:/usr/local/sce/ee/gcc/lib/gcc-lib/ee\2.95.2\../../../../ee\lib\libc.a(vfprintf.o) (_dtoa_r)
E:/usr/local/sce/ee/gcc/lib/gcc-lib/ee\2.95.2\../../../../ee\lib\libc.a(flags.o)
                              E:/usr/local/sce/ee/gcc/lib/gcc-lib/ee\2.95.2\../../../../ee\lib\libc.a(fopen.o) (__sflags)
E:/usr/local/sce/ee/gcc/lib/gcc-lib/ee\2.95.2\../../../../ee\lib\libc.a(locale.o)
                              E:/usr/local/sce/ee/gcc/lib/gcc-lib/ee\2.95.2\../../../../ee\lib\libc.a(vfprintf.o) (__mb_cur_max)
E:/usr/local/sce/ee/gcc/lib/gcc-lib/ee\2.95.2\../../../../ee\lib\libc.a(lseekr.o)
                              E:/usr/local/sce/ee/gcc/lib/gcc-lib/ee\2.95.2\../../../../ee\lib\libc.a(stdio.o) (_lseek_r)
E:/usr/local/sce/ee/gcc/lib/gcc-lib/ee\2.95.2\../../../../ee\lib\libc.a(mbtowc_r.o)
                              E:/usr/local/sce/ee/gcc/lib/gcc-lib/ee\2.95.2\../../../../ee\lib\libc.a(vfprintf.o) (_mbtowc_r)
E:/usr/local/sce/ee/gcc/lib/gcc-lib/ee\2.95.2\../../../../ee\lib\libc.a(mprec.o)
                              E:/usr/local/sce/ee/gcc/lib/gcc-lib/ee\2.95.2\../../../../ee\lib\libc.a(strtod.o) (_Balloc)
E:/usr/local/sce/ee/gcc/lib/gcc-lib/ee\2.95.2\../../../../ee\lib\libc.a(readr.o)
                              E:/usr/local/sce/ee/gcc/lib/gcc-lib/ee\2.95.2\../../../../ee\lib\libc.a(stdio.o) (_read_r)
E:/usr/local/sce/ee/gcc/lib/gcc-lib/ee\2.95.2\../../../../ee\lib\libc.a(s_isinf.o)
                              E:/usr/local/sce/ee/gcc/lib/gcc-lib/ee\2.95.2\../../../../ee\lib\libc.a(vfprintf.o) (isinf)
E:/usr/local/sce/ee/gcc/lib/gcc-lib/ee\2.95.2\../../../../ee\lib\libc.a(strtol.o)
                              E:/usr/local/sce/ee/gcc/lib/gcc-lib/ee\2.95.2\../../../../ee\lib\libc.a(vfscanf.o) (strtol)
E:/usr/local/sce/ee/gcc/lib/gcc-lib/ee\2.95.2\../../../../ee\lib\libc.a(strtoul.o)
                              E:/usr/local/sce/ee/gcc/lib/gcc-lib/ee\2.95.2\../../../../ee\lib\libc.a(vfscanf.o) (strtoul)
E:/usr/local/sce/ee/gcc/lib/gcc-lib/ee\2.95.2\../../../../ee\lib\libc.a(ungetc.o)
                              E:/usr/local/sce/ee/gcc/lib/gcc-lib/ee\2.95.2\../../../../ee\lib\libc.a(vfscanf.o) (ungetc)
E:/usr/local/sce/ee/lib\libkernl.a(klib.o)
                              E:/usr/local/sce/ee/lib/libgraph.a(graph001.o) (SetGsCrt)
E:/usr/local/sce/ee/lib\libkernl.a(glue.o)
                              E:/usr/local/sce/ee/lib/libgraph.a(graph011.o) (VSync)
E:/usr/local/sce/ee/lib\libkernl.a(cache.o)
                              E:/nightly/rwsdk.sky/rwsdk/lib/sky2/librwcore.a(basky.obj) (SyncDCache)
E:/usr/local/sce/ee/lib\libkernl.a(intr.o)
                              obj/sky2/sky.o (DisableIntc)
E:/usr/local/sce/ee/lib\libkernl.a(tty.o)
                              E:/usr/local/sce/ee/lib\libkernl.a(glue.o) (sceTtyWrite)
E:/usr/local/sce/ee/lib\libkernl.a(kprintf.o)
                              E:/usr/local/sce/ee/lib\libkernl.a(tty.o) (kprintf)
E:/usr/local/sce/ee/lib\libkernl.a(sifrpc.o)
                              obj/sky2/sky.o (sceSifInitRpc)
E:/usr/local/sce/ee/lib\libkernl.a(filestub.o)
                              obj/sky2/skyfs.o (sceOpen)
E:/usr/local/sce/ee/lib\libkernl.a(iopheap.o)
                              obj/sky2/sky.o (sceSifInitIopHeap)
E:/usr/local/sce/ee/lib\libkernl.a(eeloadfile.o)
                              obj/sky2/sky.o (sceSifLoadModule)
E:/usr/local/sce/ee/lib\libkernl.a(diei.o)
                              E:/nightly/rwsdk.sky/rwsdk/lib/sky2/librwcore.a(basky.obj) (DIntr)
E:/usr/local/sce/ee/lib\libkernl.a(initsys.o)
                              crt0.o (_InitSys)
E:/usr/local/sce/ee/lib\libkernl.a(thread.o)
                              E:/usr/local/sce/ee/lib\libkernl.a(initsys.o) (InitThread)
E:/usr/local/sce/ee/lib\libkernl.a(deci2.o)
                              E:/usr/local/sce/ee/lib\libkernl.a(tty.o) (sceDeci2Open)
E:/usr/local/sce/ee/lib\libkernl.a(sifcmd.o)
                              E:/usr/local/sce/ee/lib\libkernl.a(sifrpc.o) (sceSifGetSreg)
E:/usr/local/sce/ee/gcc/lib/gcc-lib/ee\2.95.2\libgcc.a(_divdi3.o)
                              E:/usr/local/sce/ee/lib\libkernl.a(kprintf.o) (__divdi3)
E:/usr/local/sce/ee/gcc/lib/gcc-lib/ee\2.95.2\libgcc.a(_moddi3.o)
                              E:/usr/local/sce/ee/lib\libkernl.a(kprintf.o) (__moddi3)

Allocating common symbols
Common symbol       size              file

errno               0x4               E:/usr/local/sce/ee/gcc/lib/gcc-lib/ee\2.95.2\../../../../ee\lib\libc.a(sbrkr.o)
__CTOR_LIST__       0x8               E:/usr/local/sce/ee/gcc/lib/gcc-lib/ee\2.95.2\libgcc.a(_ctors.o)
__DTOR_LIST__       0x8               E:/usr/local/sce/ee/gcc/lib/gcc-lib/ee\2.95.2\libgcc.a(_ctors.o)

Memory Configuration

Name             Origin             Length             Attributes
*default*        0x0000000000000000 0xffffffffffffffff

Linker script and memory map

LOAD crt0.o
LOAD obj/sky2/main.o
LOAD obj/sky2/im3d.o
LOAD obj/sky2/linelist.o
LOAD obj/sky2/polyline.o
LOAD obj/sky2/trilist.o
LOAD obj/sky2/tristrip.o
LOAD obj/sky2/trifan.o
LOAD obj/sky2/events.o
LOAD obj/sky2/camera.o
LOAD obj/sky2/menu.o
LOAD obj/sky2/skeleton.o
LOAD obj/sky2/sky.o
LOAD obj/sky2/skyfs.o
LOAD E:/nightly/rwsdk.sky/rwsdk/lib/sky2/librplogo.a
LOAD E:/nightly/rwsdk.sky/rwsdk/lib/sky2/librtcharse.a
LOAD E:/nightly/rwsdk.sky/rwsdk/lib/sky2/librtpng.a
LOAD E:/nightly/rwsdk.sky/rwsdk/lib/sky2/librtbmp.a
LOAD E:/nightly/rwsdk.sky/rwsdk/lib/sky2/librwcore.a
LOAD E:/usr/local/sce/ee/lib/libgraph.a
LOAD E:/usr/local/sce/ee/lib/libdma.a
LOAD E:/usr/local/sce/ee/lib/libpad.a
LOAD E:/usr/local/sce/ee/gcc/lib/gcc-lib/ee\2.95.2\../../../../ee\lib\libm.a
LOAD E:/usr/local/sce/ee/gcc/lib/gcc-lib/ee\2.95.2\libgcc.a
LOAD E:/usr/local/sce/ee/gcc/lib/gcc-lib/ee\2.95.2\libgcc.a
                0x0000000000100000                _stack_size=0x100000
                0xffffffffffffffff                _stack=0xffffffffffffffff
                0xffffffffffffffff                _heap_size=0xffffffffffffffff
START GROUP
LOAD E:/usr/local/sce/ee/gcc/lib/gcc-lib/ee\2.95.2\../../../../ee\lib\libc.a
LOAD E:/usr/local/sce/ee/lib\libkernl.a
LOAD E:/usr/local/sce/ee/gcc/lib/gcc-lib/ee\2.95.2\libgcc.a
END GROUP

.text           0x0000000000100000    0x882f0
 crt0.o(.text)
 .text          0x0000000000100000       0xc8 crt0.o
                0x0000000000100008                _start
                0x0000000000100008                ENTRYPOINT
                0x00000000001000b8                _exit
 *(.text)
 .text          0x00000000001000c8      0x5d4 obj/sky2/main.o
                0x0000000000100418                AppEventHandler
 *fill*         0x000000000010069c 0x303ec800000004
 .text          0x00000000001006a0      0x4d4 obj/sky2/im3d.o
                0x0000000000100b18                Im3DTranslateZ
                0x0000000000100800                Im3DInitialize
                0x0000000000100a00                Im3DRotate
                0x00000000001009c8                Im3DTerminate
                0x00000000001006a0                Im3DRender
 *fill*         0x0000000000100b74 0x303ec800000004
 .text          0x0000000000100b78      0x48c obj/sky2/linelist.o
                0x0000000000100bf8                IndexedLineListCreate
                0x0000000000100b78                LineListCreate
                0x0000000000100e98                LineListSetColor
                0x0000000000100f70                LineListRender
                0x0000000000100fb8                IndexedLineListRender
                0x0000000000100c78                IndexedLineListSetColor
 *fill*         0x0000000000101004 0x303ec800000004
 .text          0x0000000000101008      0x664 obj/sky2/polyline.o
                0x0000000000101340                IndexedPolyLineSetColor
                0x00000000001012c0                IndexedPolyLineCreate
                0x0000000000101088                PolyLineSetColor
                0x00000000001015d8                PolyLineRender
                0x0000000000101620                IndexedPolyLineRender
                0x0000000000101008                PolyLineCreate
 *fill*         0x000000000010166c 0x303ec800000004
 .text          0x0000000000101670      0x7a4 obj/sky2/trilist.o
                0x0000000000101ae8                IndexedTriListSetColor
                0x0000000000101a68                IndexedTriListCreate
                0x0000000000101d80                TriListRender
                0x00000000001016f0                TriListSetColor
                0x0000000000101670                TriListCreate
                0x0000000000101dc8                IndexedTriListRender
 *fill*         0x0000000000101e14 0x303ec800000004
 .text          0x0000000000101e18      0x3ac obj/sky2/tristrip.o
                0x0000000000101f18                TriStripSetColor
                0x0000000000101e18                TriStripCreate
                0x0000000000102178                IndexedTriStripRender
                0x0000000000102038                IndexedTriStripSetColor
                0x0000000000101ff0                TriStripRender
                0x0000000000101e98                IndexedTriStripCreate
 *fill*         0x00000000001021c4 0x303ec800000004
 .text          0x00000000001021c8      0x3f4 obj/sky2/trifan.o
                0x00000000001022c8                TriFanSetColor
                0x00000000001021c8                TriFanCreate
                0x0000000000102450                IndexedTriFanSetColor
                0x0000000000102570                IndexedTriFanRender
                0x0000000000102408                TriFanRender
                0x0000000000102248                IndexedTriFanCreate
 *fill*         0x00000000001025bc 0x303ec800000004
 .text          0x00000000001025c0      0x138 obj/sky2/events.o
                0x00000000001026d0                AttachInputDevices
 .text          0x00000000001026f8      0x8e8 obj/sky2/camera.o
                0x00000000001029e0                CameraMove
                0x0000000000102c58                CameraRotate
                0x0000000000102dd8                CameraCreate
                0x0000000000102b78                CameraPan
                0x0000000000102a98                CameraTilt
                0x0000000000102f38                CameraCreateCrossHair
                0x0000000000102d38                CameraDestroy
                0x00000000001026f8                CameraSize
 .text          0x0000000000102fe0     0x2d34 obj/sky2/menu.o
                0x0000000000105a68                MenuSelectEntry
                0x0000000000105bd8                MenuSetRangeReal
                0x0000000000104d98                MenuRender
                0x00000000001052a8                MenuOpen
                0x0000000000105580                MenuAddEntryBoolTransient
                0x0000000000104398                MenuKeyboardShortcutHandler
                0x0000000000103288                MenuToggle
                0x0000000000104500                MenuKeyboardHandler
                0x0000000000105a58                MenuGetStatus
                0x0000000000103a88                MenuRemoveEntry
                0x00000000001059b8                MenuAddSeparator
                0x0000000000105c98                MenuSetStatus
                0x0000000000105650                MenuAddEntryInt
                0x0000000000105ab0                MenuSetRangeInt
                0x00000000001054b0                MenuAddEntryBool
                0x0000000000103e00                MenuMouseHandler
                0x00000000001040e0                MenuPadHandler
                0x0000000000105100                MenuClose
                0x0000000000105908                MenuAddEntryTrigger
                0x00000000001057e8                MenuAddEntryReal
 *fill*         0x0000000000105d14 0x303ec800000004
 .text          0x0000000000105d18     0x14a8 obj/sky2/skeleton.o
                0x0000000000106e78                RsMouseSetVisibility
                0x0000000000106de8                RsKeyFromScanCode
                0x0000000000106ed8                RsRwTerminate
                0x0000000000106348                RsLoadPresetViews
                0x0000000000106e38                RsErrorMessage
                0x0000000000106e18                RsCameraShowRaster
                0x0000000000106be8                RsPadEventHandler
                0x0000000000106fa0                RsSetPresetView
                0x0000000000106bb0                RsMouseEventHandler
                0x0000000000105e70                RsRwInitialize
                0x0000000000106ce0                RsSelectDevice
                0x0000000000106d88                RsPathGetSeparator
                0x0000000000107178                RsGrabScreen
                0x0000000000106e98                RsMouseSetPos
                0x00000000001070f8                RsDestroyPresetViews
                0x0000000000105f50                RsSetModelTexturePath
                0x00000000001070b0                RsGetPresetViewDescription
                0x0000000000106c88                RsRegisterImageLoader
                0x00000000001068a0                RsSavePresetView
                0x0000000000106f40                RsWarningMessage
                0x0000000000106eb8                RsPathnameDestroy
                0x00000000001060f8                RsSetNextPresetView
                0x0000000000106dc8                RsTimer
                0x0000000000106d68                RsAlwaysOnTop
                0x0000000000105d18                RsEventHandler
                0x0000000000106220                RsSetPreviousPresetView
                0x0000000000106f20                RsTerminate
                0x0000000000106d00                RsInputDeviceAttach
                0x0000000000106b78                RsKeyboardEventHandler
                0x0000000000106c20                RsInitialize
                0x0000000000106da8                RsPathnameCreate
                0x0000000000106f80                RsWindowSetText
 .text          0x00000000001071c0     0x16c4 obj/sky2/sky.o
                0x0000000000108410                psPathnameCreate
                0x0000000000108548                psGetMemoryFunctions
                0x0000000000108510                psAlwaysOnTop
                0x0000000000108290                psTimer
                0x0000000000108270                psDebugMessageHandler
                0x0000000000108500                psInitialize
                0x0000000000108508                psTerminate
                0x0000000000108258                psWindowSetText
                0x0000000000108538                psMouseSetVisibility
                0x00000000001084f8                psPathGetSeparator
                0x0000000000108300                psGrabScreen
                0x0000000000108268                psWarningMessage
                0x0000000000107f20                main
                0x00000000001071c0                psSelectDevice
                0x0000000000108518                psCameraShowRaster
                0x0000000000108630                skyOverideIOPPath
                0x00000000001085b0                psNativeTextureSupport
                0x0000000000108540                psMouseSetPos
                0x00000000001085b8                psMicroTimer
                0x0000000000108260                psErrorMessage
                0x0000000000108588                psInstallFileSystem
                0x00000000001084d0                psPathnameDestroy
 *fill*         0x0000000000108884 0x303ec800000004
 .text          0x0000000000108888      0xca0 obj/sky2/skyfs.o
                0x0000000000108d88                SkyInstallFileSystem
 .text          0x0000000000109528      0x998 E:/nightly/rwsdk.sky/rwsdk/lib/sky2/librplogo.a(rplogo.obj)
                0x0000000000109c48                RpLogoPluginAttach
                0x0000000000109cb8                RpLogoSetPosition
                0x0000000000109e00                RpLogoGetRenderingRect
                0x0000000000109dc8                RpLogoGetState
                0x0000000000109d40                RpLogoGetPosition
                0x0000000000109d70                RpLogoSetState
 .text          0x0000000000109ec0      0x98c E:/nightly/rwsdk.sky/rwsdk/lib/sky2/librtcharse.a(chrprint.obj)
                0x000000000010a508                RtCharsetBufferFlush
                0x000000000010a660                RtCharsetPrintBuffered
                0x000000000010a830                RtCharsetPrint
 *fill*         0x000000000010a84c 0x303ec800000004
 .text          0x000000000010a850      0x75c E:/nightly/rwsdk.sky/rwsdk/lib/sky2/librtcharse.a(rtcharse.obj)
                0x000000000010ad90                RtCharsetClose
                0x000000000010aa18                RtCharsetSetColors
                0x000000000010aba8                RtCharsetCreate
                0x000000000010ad00                RtCharsetOpen
                0x000000000010aeb0                RtCharsetDestroy
                0x000000000010af30                _rtCharsetAtariFontGet
                0x000000000010adf0                RtCharsetGetDesc
 *fill*         0x000000000010afac 0x303ec800000004
 .text          0x000000000010afb0      0xae8 E:/nightly/rwsdk.sky/rwsdk/lib/sky2/librtpng.a(rtpng.obj)
                0x000000000010b920                RwImageWritePNG
                0x000000000010b380                RtPNGImageRead
                0x000000000010b978                RwImageReadPNG
                0x000000000010afb0                RtPNGImageWrite
 .text          0x000000000010ba98      0xac8 E:/nightly/rwsdk.sky/rwsdk/lib/sky2/librtpng.a(png.obj)
                0x000000000010c258                png_get_header_ver
                0x000000000010c3b8                png_zfree
                0x000000000010c308                png_zalloc
                0x000000000010c288                png_get_libpng_ver
                0x000000000010bfc0                png_sig_cmp
                0x000000000010bf68                png_set_sig_bytes
                0x000000000010c2a0                png_info_destroy
                0x000000000010c1e0                png_get_io_ptr
                0x000000000010c478                png_handle_as_unknown
                0x000000000010bf60                png_access_version_number
                0x000000000010c128                png_info_init_3
                0x000000000010c248                png_get_copyright
                0x000000000010c270                png_get_header_version
                0x000000000010c090                png_reset_zstream
                0x000000000010c410                png_calculate_crc
                0x000000000010c558                png_mmx_support
                0x000000000010c030                png_check_sig
                0x000000000010c3d8                png_reset_crc
                0x000000000010c0b0                png_create_info_struct
                0x000000000010c100                png_info_init
                0x000000000010c178                png_destroy_info_struct
                0x000000000010ba98                png_free_data
                0x000000000010c1e8                png_data_freer
 .text          0x000000000010c560      0x468 E:/nightly/rwsdk.sky/rwsdk/lib/sky2/librtpng.a(pngerror.obj)
                0x000000000010c758                png_error
                0x000000000010c930                png_warning
                0x000000000010c560                png_chunk_warning
                0x000000000010c750                png_get_error_ptr
                0x000000000010c7a0                png_chunk_error
                0x000000000010c740                png_set_error_fn
 .text          0x000000000010c9c8      0xcd0 E:/nightly/rwsdk.sky/rwsdk/lib/sky2/librtpng.a(pngget.obj)
                0x000000000010d3f8                png_get_sBIT
                0x000000000010cf80                png_get_cHRM_fixed
                0x000000000010cdf8                png_get_bKGD
                0x000000000010d0e8                png_get_hIST
                0x000000000010caf8                png_get_interlace_type
                0x000000000010ccc0                png_get_x_offset_pixels
                0x000000000010d4e0                png_get_sPLT
                0x000000000010ca38                png_get_rowbytes
                0x000000000010d478                png_get_iCCP
                0x000000000010c9e0                png_get_rgb_to_gray_status
                0x000000000010cae0                png_get_filter_type
                0x000000000010d560                png_get_tIME
                0x000000000010cd98                png_get_y_offset_microns
                0x000000000010ca98                png_get_image_height
                0x000000000010d2a8                png_get_pCAL
                0x000000000010ca80                png_get_image_width
                0x000000000010cb80                png_get_x_pixels_per_meter
                0x000000000010d438                png_get_sRGB
                0x000000000010ca68                png_get_channels
                0x000000000010d038                png_get_gAMA
                0x000000000010cd08                png_get_y_offset_pixels
                0x000000000010c9c8                png_get_compression_buffer_size
                0x000000000010ca10                png_get_valid
                0x000000000010cb10                png_get_compression_type
                0x000000000010cd50                png_get_x_offset_microns
                0x000000000010ca50                png_get_rows
                0x000000000010d248                png_get_oFFs
                0x000000000010cab0                png_get_bit_depth
                0x000000000010cac8                png_get_color_type
                0x000000000010d3b0                png_get_PLTE
                0x000000000010cb28                png_get_pixels_per_meter
                0x000000000010d128                png_get_IHDR
                0x000000000010d0a0                png_get_gAMA_fixed
                0x000000000010cde0                png_get_signature
                0x000000000010d508                png_get_text
                0x000000000010d628                png_get_sCAL
                0x000000000010ce38                png_get_cHRM
                0x000000000010d5a0                png_get_tRNS
                0x000000000010d348                png_get_pHYs
                0x000000000010cbc8                png_get_y_pixels_per_meter
                0x000000000010d670                png_get_unknown_chunks
                0x000000000010cc10                png_get_pixel_aspect_ratio
                0x000000000010c9f8                png_get_user_chunk_ptr
 .text          0x000000000010d698      0x348 E:/nightly/rwsdk.sky/rwsdk/lib/sky2/librtpng.a(pngmem.obj)
                0x000000000010d8e8                png_destroy_struct
                0x000000000010d698                png_set_mem_fn
                0x000000000010d7d0                png_free_default
                0x000000000010d908                png_create_struct_2
                0x000000000010d860                png_memset_check
                0x000000000010d6b0                png_malloc
                0x000000000010d8c8                png_create_struct
                0x000000000010d9a0                png_destroy_struct_2
                0x000000000010d7f8                png_memcpy_check
                0x000000000010d730                png_free
                0x000000000010d6a8                png_get_mem_ptr
                0x000000000010d778                png_malloc_default
 .text          0x000000000010d9e0     0x2088 E:/nightly/rwsdk.sky/rwsdk/lib/sky2/librtpng.a(pngread.obj)
                0x000000000010eea8                png_read_destroy
                0x000000000010f9b0                png_set_read_status_fn
                0x000000000010f9b8                png_read_init
                0x000000000010f540                png_create_read_struct
                0x000000000010dca0                png_read_init_3
                0x000000000010f220                png_read_png
                0x000000000010f568                png_start_read_image
                0x000000000010f9e0                png_read_init_2
                0x000000000010de90                png_read_info
                0x000000000010f8a0                png_destroy_read_struct
                0x000000000010f598                png_read_update_info
                0x000000000010f7a0                png_read_image
                0x000000000010e448                png_read_row
                0x000000000010d9e0                png_create_read_struct_2
                0x000000000010f600                png_read_rows
                0x000000000010e9d8                png_read_end
 .text          0x000000000010fa68       0x90 E:/nightly/rwsdk.sky/rwsdk/lib/sky2/librtpng.a(pngrio.obj)
                0x000000000010fa68                png_set_read_fn
                0x000000000010fac0                png_read_data
 .text          0x000000000010faf8     0x6f54 E:/nightly/rwsdk.sky/rwsdk/lib/sky2/librtpng.a(pngrtran.obj)
                0x00000000001123f8                png_do_read_filler
                0x000000000010faf8                png_set_dither
                0x0000000000116320                png_set_gray_1_2_4_to_8
                0x0000000000116960                png_set_read_user_transform_fn
                0x0000000000116650                png_set_strip_alpha
                0x0000000000116760                png_set_strip_16
                0x0000000000115918                png_build_gamma_table
                0x0000000000111cc0                png_do_unshift
                0x0000000000115718                png_do_dither
                0x0000000000112b48                png_do_rgb_to_gray
                0x0000000000116380                png_set_rgb_to_gray
                0x0000000000116368                png_set_gray_to_rgb
                0x0000000000112898                png_do_gray_to_rgb
                0x0000000000116458                png_set_rgb_to_gray_fixed
                0x0000000000111650                png_do_read_transformations
                0x0000000000116840                png_set_crc_action
                0x0000000000116338                png_set_palette_to_rgb
                0x0000000000112058                png_do_read_swap_alpha
                0x00000000001147a0                png_do_gamma
                0x0000000000116308                png_set_expand
                0x00000000001113c0                png_read_transform_info
                0x0000000000115168                png_do_expand
                0x0000000000110570                png_init_read_transformations
                0x0000000000116350                png_set_tRNS_to_alpha
                0x0000000000112268                png_do_read_invert_alpha
                0x0000000000116588                png_build_grayscale_palette
                0x0000000000116978                png_do_chop
                0x0000000000116668                png_set_background
                0x0000000000111aa0                png_do_unpack
                0x0000000000114da0                png_do_expand_palette
                0x0000000000116778                png_set_gamma
                0x0000000000113410                png_do_background
 *fill*         0x0000000000116a4c 0x303ec800000004
 .text          0x0000000000116a50     0x6cc8 E:/nightly/rwsdk.sky/rwsdk/lib/sky2/librtpng.a(pngrutil.obj)
                0x0000000000118680                png_handle_sRGB
                0x000000000011cb50                png_read_finish_row
                0x0000000000116d58                png_handle_IHDR
                0x000000000011d470                png_crc_error
                0x000000000011d2e0                png_get_uint_16
                0x000000000011d678                png_check_chunk_name
                0x000000000011c818                png_read_filter_row
                0x000000000011cf40                png_read_start_row
                0x000000000011a408                png_handle_pHYs
                0x000000000011d2b0                png_get_uint_32
                0x000000000011d518                png_handle_IEND
                0x000000000011a000                png_handle_hIST
                0x00000000001173f0                png_handle_gAMA
                0x000000000011b4f0                png_handle_tIME
                0x0000000000119558                png_handle_tRNS
                0x0000000000116fa8                png_handle_PLTE
                0x000000000011a7a8                png_handle_oFFs
                0x0000000000119b18                png_handle_bKGD
                0x000000000011b0e8                png_handle_sCAL
                0x0000000000118bc0                png_handle_iCCP
                0x000000000011b9e8                png_handle_zTXt
                0x000000000011ab48                png_handle_pCAL
                0x000000000011bc18                png_handle_unknown
                0x000000000011d2f8                png_crc_read
                0x0000000000117820                png_handle_sBIT
                0x000000000011beb8                png_combine_row
                0x000000000011d348                png_crc_finish
                0x00000000001190b8                png_handle_sPLT
                0x0000000000117bf0                png_handle_cHRM
                0x0000000000116a50                png_decompress_chunk
                0x000000000011c280                png_do_read_interlace
                0x000000000011d280                png_get_int_32
                0x000000000011b820                png_handle_tEXt
 .text          0x000000000011d718     0x192c E:/nightly/rwsdk.sky/rwsdk/lib/sky2/librtpng.a(pngset.obj)
                0x000000000011ea20                png_set_sBIT
                0x000000000011e370                png_set_cHRM_fixed
                0x000000000011e530                png_set_gAMA
                0x000000000011efe0                png_set_unknown_chunk_location
                0x000000000011de38                png_set_text
                0x000000000011e5e0                png_set_gAMA_fixed
                0x000000000011e330                png_set_bKGD
                0x000000000011e758                png_set_oFFs
                0x000000000011d940                png_set_IHDR
                0x000000000011ecf0                png_set_keep_unknown_chunks
                0x000000000011ebe8                png_set_tRNS
                0x000000000011e788                png_set_pCAL
                0x000000000011ee80                png_set_unknown_chunks
                0x000000000011e970                png_set_PLTE
                0x000000000011f020                png_set_invalid
                0x000000000011e090                png_set_sPLT
                0x000000000011d718                png_set_cHRM
                0x000000000011ecc0                png_set_sCAL
                0x000000000011ea88                png_set_iCCP
                0x000000000011e290                png_permit_empty_plte
                0x000000000011e228                png_set_compression_buffer_size
                0x000000000011e2b0                png_set_read_user_chunk_fn
                0x000000000011e670                png_set_hIST
                0x000000000011dbd0                png_set_sRGB_gAMA_and_cHRM
                0x000000000011e940                png_set_pHYs
                0x000000000011ea60                png_set_sRGB
                0x000000000011eba0                png_set_tIME
                0x000000000011e2c0                png_set_rows
 *fill*         0x000000000011f044 0x303ec800000004
 .text          0x000000000011f048      0x960 E:/nightly/rwsdk.sky/rwsdk/lib/sky2/librtpng.a(pngtrans.obj)
                0x000000000011f048                png_do_strip_filler
                0x000000000011f608                png_set_filler
                0x000000000011f738                png_set_interlace_handling
                0x000000000011f798                png_do_swap
                0x000000000011f6b0                png_set_packing
                0x000000000011f5d8                png_set_swap_alpha
                0x000000000011f780                png_set_user_transform_info
                0x000000000011f5c0                png_set_bgr
                0x000000000011f688                png_set_swap
                0x000000000011f3d0                png_do_bgr
                0x000000000011f6e0                png_set_packswap
                0x000000000011f768                png_set_invert_mono
                0x000000000011f858                png_do_packswap
                0x000000000011f928                png_do_invert
                0x000000000011f5f0                png_set_invert_alpha
                0x000000000011f790                png_get_user_transform_ptr
                0x000000000011f708                png_set_shift
 .text          0x000000000011f9a8       0xb8 E:/nightly/rwsdk.sky/rwsdk/lib/sky2/librtpng.a(pngwio.obj)
                0x000000000011f9a8                png_set_write_fn
                0x000000000011fa38                png_flush
                0x000000000011fa00                png_write_data
 .text          0x000000000011fa60     0x1c80 E:/nightly/rwsdk.sky/rwsdk/lib/sky2/librtpng.a(pngwrite.obj)
                0x0000000000121460                png_set_write_status_fn
                0x0000000000121328                png_set_compression_level
                0x0000000000120290                png_create_write_struct_2
                0x0000000000121658                png_write_init_2
                0x0000000000121340                png_set_compression_mem_level
                0x00000000001210f8                png_write_rows
                0x0000000000121370                png_set_compression_window_bits
                0x0000000000120fe8                png_set_flush
                0x0000000000120fc0                png_create_write_struct
                0x000000000011fa60                png_write_info_before_PLTE
                0x00000000001205f0                png_write_row
                0x000000000011fce8                png_write_info
                0x00000000001204a0                png_write_init_3
                0x0000000000120090                png_write_end
                0x0000000000121480                png_write_png
                0x00000000001209b8                png_set_filter
                0x0000000000121468                png_set_write_user_transform_fn
                0x0000000000120850                png_write_destroy
                0x00000000001211a0                png_write_image
                0x0000000000121408                png_set_compression_method
                0x0000000000120be0                png_set_filter_heuristics
                0x0000000000121000                png_write_flush
                0x0000000000121358                png_set_compression_strategy
                0x0000000000121250                png_destroy_write_struct
                0x0000000000121630                png_write_init
 .text          0x00000000001216e0      0xb0c E:/nightly/rwsdk.sky/rwsdk/lib/sky2/librtpng.a(pngwtran.obj)
                0x0000000000121850                png_do_pack
                0x0000000000121ff0                png_do_write_invert_alpha
                0x0000000000121a50                png_do_shift
                0x00000000001216e0                png_do_write_transformations
                0x0000000000121df0                png_do_write_swap_alpha
 *fill*         0x00000000001221ec 0x303ec800000004
 .text          0x00000000001221f0     0x4d58 E:/nightly/rwsdk.sky/rwsdk/lib/sky2/librtpng.a(pngwutil.obj)
                0x00000000001269d0                png_write_gAMA_fixed
                0x0000000000122b40                png_write_iCCP
                0x0000000000123e28                png_check_keyword
                0x0000000000126a58                png_write_sRGB
                0x0000000000122528                png_write_IHDR
                0x00000000001240d8                png_write_tEXt
                0x0000000000126700                png_write_chunk_end
                0x0000000000123268                png_write_cHRM
                0x00000000001267a0                png_save_int_32
                0x0000000000123828                png_write_cHRM_fixed
                0x0000000000124b40                png_write_start_row
                0x00000000001242b0                png_write_zTXt
                0x0000000000122950                png_write_PLTE
                0x0000000000123b78                png_write_bKGD
                0x0000000000123128                png_write_sBIT
                0x0000000000126e08                png_write_filtered_row
                0x0000000000122e48                png_write_sPLT
                0x0000000000125380                png_write_find_filter
                0x0000000000126858                png_write_IDAT
                0x00000000001267e0                png_save_uint_16
                0x0000000000126760                png_save_uint_32
                0x00000000001266a0                png_write_chunk_data
                0x0000000000126598                png_write_chunk
                0x00000000001265f8                png_write_chunk_start
                0x0000000000123cb0                png_write_hIST
                0x0000000000124d20                png_write_finish_row
                0x00000000001268c8                png_write_IEND
                0x00000000001245f0                png_write_pCAL
                0x0000000000124988                png_write_sCAL_s
                0x0000000000126c08                png_write_oFFs
                0x0000000000126920                png_write_gAMA
                0x0000000000124fe8                png_do_write_interlace
                0x0000000000126d08                png_write_pHYs
                0x00000000001267f0                png_write_sig
                0x0000000000126ac8                png_write_tRNS
 .text          0x0000000000126f48     0x2458 E:/nightly/rwsdk.sky/rwsdk/lib/sky2/librtpng.a(deflate.obj)
                0x0000000000127368                deflate
                0x0000000000127200                deflateSetDictionary
                0x00000000001292c8                deflateInit_
                0x0000000000126f48                deflateInit2_
                0x0000000000129108                deflateReset
                0x00000000001278d0                deflateCopy
                0x00000000001291b8                deflateParams
                0x0000000000129020                deflateEnd
 .text          0x00000000001293a0     0x24d0 E:/nightly/rwsdk.sky/rwsdk/lib/sky2/librtpng.a(trees.obj)
                0x000000000012a8b8                _tr_flush_block
                0x000000000012b380                _tr_stored_block
                0x000000000012b310                _tr_init
                0x000000000012ad08                _tr_tally
                0x000000000012a5e0                _tr_align
 .text          0x000000000012b870       0x6c E:/nightly/rwsdk.sky/rwsdk/lib/sky2/librtpng.a(zutil.obj)
                0x000000000012b870                zlibVersion
                0x000000000012b8c0                zcfree
                0x000000000012b880                zError
                0x000000000012b8a0                zcalloc
 *fill*         0x000000000012b8dc 0x303ec800000004
 .text          0x000000000012b8e0      0xa40 E:/nightly/rwsdk.sky/rwsdk/lib/sky2/librtpng.a(inflate.obj)
                0x000000000012bab0                inflate
                0x000000000012c2e0                inflateSyncPoint
                0x000000000012c2b8                inflateInit_
                0x000000000012c258                inflateReset
                0x000000000012bfb8                inflateSync
                0x000000000012c188                inflateSetDictionary
                0x000000000012c118                inflateEnd
                0x000000000012b8e0                inflateInit2_
 .text          0x000000000012c320     0x1000 E:/nightly/rwsdk.sky/rwsdk/lib/sky2/librtpng.a(infblock.obj)
                0x000000000012d1f0                inflate_blocks_free
                0x000000000012c428                inflate_blocks
                0x000000000012d140                inflate_blocks_reset
                0x000000000012d310                inflate_blocks_sync_point
                0x000000000012d2c8                inflate_set_dictionary
                0x000000000012c320                inflate_blocks_new
 .text          0x000000000012d320      0xb20 E:/nightly/rwsdk.sky/rwsdk/lib/sky2/librtpng.a(inftrees.obj)
                0x000000000012de10                inflate_trees_fixed
                0x000000000012db20                inflate_trees_bits
                0x000000000012dc20                inflate_trees_dynamic
 .text          0x000000000012de40      0x928 E:/nightly/rwsdk.sky/rwsdk/lib/sky2/librtpng.a(infcodes.obj)
                0x000000000012e6d0                inflate_codes_new
                0x000000000012de40                inflate_codes
                0x000000000012e740                inflate_codes_free
 .text          0x000000000012e768      0x180 E:/nightly/rwsdk.sky/rwsdk/lib/sky2/librtpng.a(infutil.obj)
                0x000000000012e768                inflate_flush
 .text          0x000000000012e8e8      0x5b8 E:/nightly/rwsdk.sky/rwsdk/lib/sky2/librtpng.a(inffast.obj)
                0x000000000012e8e8                inflate_fast
 .text          0x000000000012eea0      0x20c E:/nightly/rwsdk.sky/rwsdk/lib/sky2/librtpng.a(crc32.obj)
                0x000000000012eea0                crc32
                0x000000000012f0a0                get_crc_table
 *fill*         0x000000000012f0ac 0x303ec800000004
 .text          0x000000000012f0b0      0x1e4 E:/nightly/rwsdk.sky/rwsdk/lib/sky2/librtpng.a(adler32.obj)
                0x000000000012f0b0                adler32
 *fill*         0x000000000012f294 0x303ec800000004
 .text          0x000000000012f298     0x12b8 E:/nightly/rwsdk.sky/rwsdk/lib/sky2/librtbmp.a(rtbmp.obj)
                0x000000000012fea0                RtBMPImageRead
                0x00000000001304e0                RtBMPImageWrite
 .text          0x0000000000130550      0x6b4 E:/nightly/rwsdk.sky/rwsdk/lib/sky2/librwcore.a(babinary.obj)
                0x00000000001309f0                RwMemRealToFloat32
                0x0000000000130a40                RwMemFloat32ToReal
                0x00000000001309e0                RwMemNative16
                0x0000000000130980                RwStreamReadInt16
                0x00000000001309e8                RwMemNative32
                0x0000000000130a90                RwStreamReadChunkHeaderInfo
                0x00000000001309d8                RwMemLittleEndian32
                0x0000000000130700                _rwStreamWriteVersionedChunkHeader
                0x0000000000130830                RwStreamWriteInt32
                0x00000000001309d0                RwMemLittleEndian16
                0x0000000000130880                RwStreamReadReal
                0x0000000000130930                RwStreamReadInt32
                0x0000000000130748                RwStreamWriteReal
                0x0000000000130b58                _rwStreamReadChunkHeader
                0x0000000000130598                RwStreamFindChunk
                0x0000000000130858                RwStreamWriteInt16
 *fill*         0x0000000000130c04 0x303ec800000004
 .text          0x0000000000130c08     0x1d00 E:/nightly/rwsdk.sky/rwsdk/lib/sky2/librwcore.a(bacamera.obj)
                0x00000000001325f0                RwCameraGetFarClipPlane
                0x0000000000132300                RwCameraGetViewWindow
                0x0000000000132230                RwCameraSetZRaster
                0x0000000000132680                RwCameraValidatePlugins
                0x0000000000132658                RwCameraGetPluginOffset
                0x00000000001325f8                RwCameraSetFogDistance
                0x00000000001321e8                RwCameraSetFrame
                0x0000000000132188                RwCameraDestroy
                0x0000000000132778                _rwCameraOpen
                0x0000000000132430                RwCameraGetViewMatrix
                0x0000000000132688                RwCameraFrustumTestSphere
                0x0000000000132518                RwCameraSetFarClipPlane
                0x0000000000132158                RwCameraShowRaster
                0x0000000000132228                RwCameraGetRaster
                0x0000000000132308                RwCameraSetProjection
                0x0000000000132290                RwCameraGetViewOffset
                0x0000000000132298                RwCameraSetViewWindow
                0x0000000000132218                RwCameraSetRaster
                0x0000000000132710                _rwCameraClose
                0x0000000000132510                RwCameraGetNearClipPlane
                0x0000000000132428                RwCameraGetProjection
                0x0000000000132240                RwCameraGetZRaster
                0x0000000000132120                RwCameraClear
                0x0000000000132210                RwCameraGetFrame
                0x0000000000132438                RwCameraSetNearClipPlane
                0x0000000000132610                RwCameraRegisterPlugin
                0x0000000000131de0                RwCameraCreate
                0x0000000000132100                RwCameraEndUpdate
                0x0000000000132608                RwCameraGetFogDistance
                0x00000000001320e0                RwCameraBeginUpdate
                0x0000000000131f70                RwCameraClone
                0x0000000000132248                RwCameraSetViewOffset
 .text          0x0000000000132908      0xd04 E:/nightly/rwsdk.sky/rwsdk/lib/sky2/librwcore.a(badevice.obj)
                0x0000000000132ff0                RwEngineClose
                0x0000000000132dd8                RwEngineSetFocus
                0x0000000000132ef0                RwEngineStart
                0x0000000000132ad8                RwEngineGetNumSubSystems
                0x0000000000133340                RwEngineTerm
                0x0000000000132d08                RwEngineGetTextureMemorySize
                0x0000000000132d70                RwEngineGetMaxTextureSize
                0x0000000000132b68                RwEngineSetSubSystem
                0x00000000001334b8                _rwDeviceSystemRequest
                0x00000000001331c0                RwEngineInit
                0x0000000000133390                RwEngineGetSubSystemInfo
                0x0000000000133318                RwEngineGetPluginOffset
                0x0000000000132ca8                RwEngineSetVideoMode
                0x0000000000132c40                RwEngineGetCurrentVideoMode
                0x0000000000133078                RwEngineOpen
                0x0000000000132e38                RwEngineStop
                0x00000000001331b8                RwEngineGetVersion
                0x0000000000132b28                RwEngineGetCurrentSubSystem
                0x0000000000133438                RwEngineGetVideoModeInfo
                0x0000000000132bd8                RwEngineGetNumVideoModes
                0x00000000001332d8                RwEngineRegisterPlugin
                0x00000000001335a8                _rwGetNumEngineInstances
                0x00000000001334a8                RwEngineGetMetrics
 *fill*         0x000000000013360c 0x303ec800000004
 .text          0x0000000000133610      0x12c E:/nightly/rwsdk.sky/rwsdk/lib/sky2/librwcore.a(baerr.obj)
                0x0000000000133698                RwErrorGet
                0x0000000000133610                _rwerror
                0x00000000001336d8                RwErrorSet
                0x0000000000133650                _rwErrorOpen
                0x0000000000133680                _rwErrorClose
 *fill*         0x000000000013373c 0x303ec800000004
 .text          0x0000000000133740     0x1190 E:/nightly/rwsdk.sky/rwsdk/lib/sky2/librwcore.a(baframe.obj)
                0x00000000001341f8                RwFrameInit
                0x0000000000133a68                RwFrameRotate
                0x0000000000133b68                RwFrameTransform
                0x00000000001342c0                RwFrameDestroy
                0x0000000000134108                RwFrameGetLTM
                0x0000000000134400                RwFrameDirty
                0x00000000001344d8                RwFrameGetPluginOffset
                0x0000000000134100                RwFrameGetRoot
                0x0000000000133740                _rwFrameCloneAndLinkClones
                0x0000000000134370                _rwFrameDeInit
                0x0000000000134500                RwFrameValidatePlugins
                0x0000000000134490                RwFrameRegisterPlugin
                0x0000000000133dd0                RwFrameDestroyHierarchy
                0x0000000000134508                _rwFramePurgeClone
                0x0000000000133f00                RwFrameRemoveChild
                0x0000000000133d20                RwFrameCloneHierarchy
                0x0000000000134230                RwFrameDeInit
                0x0000000000134148                RwFrameUpdateObjects
                0x00000000001339e8                RwFrameTranslate
                0x0000000000134598                _rwFrameClose
                0x0000000000134460                RwFrameSetStaticPluginsSize
                0x0000000000133be8                RwFrameOrthoNormalize
                0x0000000000133898                _rwFrameInit
                0x0000000000134410                RwFrameCount
                0x0000000000133c68                RwFrameSetIdentity
                0x0000000000134600                _rwFrameOpen
                0x00000000001341a8                RwFrameCreate
                0x0000000000133970                RwFrameForAllObjects
                0x0000000000133ae8                RwFrameScale
                0x0000000000133e90                RwFrameForAllChildren
                0x0000000000133fe8                RwFrameAddChild
 .text          0x00000000001348d0      0x108 E:/nightly/rwsdk.sky/rwsdk/lib/sky2/librwcore.a(bafsys.obj)
                0x0000000000134968                _rwFileSystemClose
                0x00000000001348d0                _rwFileSystemOpen
                0x0000000000134970                RwOsGetFileInterface
 .text          0x00000000001349d8     0x242c E:/nightly/rwsdk.sky/rwsdk/lib/sky2/librwcore.a(baimage.obj)
                0x0000000000135dd8                RwImageStreamRead
                0x0000000000136928                RwRGBASetFromPixel
                0x0000000000136058                RwImageStreamWrite
                0x00000000001368b0                RwImageSetPixels
                0x0000000000136a90                RwRGBAGammaCorrect
                0x00000000001359b0                RwImageReadMaskedImage
                0x00000000001367c0                RwImageSetPath
                0x0000000000136ae8                RwImageRegisterPlugin
                0x0000000000136c40                _rwImageGammaUnCorrectArrayOfRGBA
                0x0000000000136b60                RwImageFindFileType
                0x0000000000136a78                RwImageGetGamma
                0x0000000000134c70                RwImageResize
                0x00000000001366c8                RwImageWrite
                0x00000000001368e0                RwImageGetDepth
                0x0000000000136368                RwImageCreate
                0x0000000000136960                RwImageSetGamma
                0x0000000000136b90                RwImageStreamGetSize
                0x00000000001368f0                RwImageGetPalette
                0x0000000000136400                RwImageDestroy
                0x0000000000136160                RwImageGammaCorrect
                0x00000000001368e8                RwImageGetPixels
                0x00000000001365c8                RwImageCopy
                0x0000000000135828                RwImageRegisterImageFormat
                0x0000000000136470                RwImageAllocatePixels
                0x0000000000134fa0                RwImageApplyMask
                0x0000000000136bc0                _rwImageGammaCorrectArrayOfRGBA
                0x0000000000136b58                RwImageValidatePlugins
                0x0000000000136578                RwImageFreePixels
                0x00000000001368a0                RwImageSetStride
                0x0000000000136b30                RwImageGetPluginOffset
                0x00000000001368c0                RwImageSetPalette
                0x00000000001367a8                RwImageGetPath
                0x0000000000135700                RwImageRead
                0x0000000000134e90                RwImageMakeMask
                0x00000000001368f8                RwRGBAToPixel
                0x00000000001349d8                _rwImageOpen
                0x00000000001368d8                RwImageGetHeight
                0x00000000001368d0                RwImageGetWidth
                0x0000000000134b40                _rwImageClose
 *fill*         0x0000000000136e04 0x303ec800000004
 .text          0x0000000000136e08      0x144 E:/nightly/rwsdk.sky/rwsdk/lib/sky2/librwcore.a(baimmedi.obj)
                0x0000000000136e28                RwRenderStateGet
                0x0000000000136f28                RwIm2DRenderIndexedPrimitive
                0x0000000000136e18                RwIm2DGetFarScreenZ
                0x0000000000136e50                RwRenderStateSet
                0x0000000000136eb0                RwIm2DRenderLine
                0x0000000000136ed8                RwIm2DRenderTriangle
                0x0000000000136f00                RwIm2DRenderPrimitive
                0x0000000000136e08                RwIm2DGetNearScreenZ
 *fill*         0x0000000000136f4c 0x303ec800000004
 .text          0x0000000000136f50      0x41c E:/nightly/rwsdk.sky/rwsdk/lib/sky2/librwcore.a(baimras.obj)
                0x0000000000136f50                RwImageSetFromRaster
                0x0000000000136fb8                RwRasterSetFromImage
                0x00000000001372c8                RwImageFindRasterFormat
                0x0000000000137020                RwRGBAGetRasterPixel
                0x0000000000137138                RwRasterRead
                0x00000000001371f8                RwRasterReadMaskedRaster
 *fill*         0x000000000013736c 0x303ec800000004
 .text          0x0000000000137370     0x1f98 E:/nightly/rwsdk.sky/rwsdk/lib/sky2/librwcore.a(bamatrix.obj)
                0x0000000000139128                _rwMatrixIdentityError
                0x0000000000138710                RwMatrixScale
                0x0000000000138f48                RwMatrixUpdate
                0x0000000000138b10                RwMatrixDestroy
                0x0000000000138f28                RwMatrixQueryRotate
                0x0000000000138f68                _rwMatrixDeterminant
                0x0000000000138e30                RwMatrixRotate
                0x0000000000138fe8                _rwMatrixNormalError
                0x0000000000138e10                RwMatrixOrthoNormalize
                0x0000000000139090                _rwMatrixOrthogonalError
                0x00000000001391d8                _rwMatrixSetOptimizations
                0x0000000000138c50                RwMatrixTransform
                0x0000000000139228                _rwMatrixOpen
                0x00000000001382e0                RwMatrixRotateOneMinusCosineSine
                0x0000000000138588                RwMatrixInvert
                0x00000000001380d8                RwMatrixOptimize
                0x0000000000138bd0                RwMatrixMultiply
                0x00000000001392a0                _rwMatrixClose
                0x0000000000138b48                RwMatrixCreate
                0x0000000000138950                RwMatrixTranslate
                0x00000000001391f8                _rwMatrixSetMultFn
 .text          0x0000000000139308      0x968 E:/nightly/rwsdk.sky/rwsdk/lib/sky2/librwcore.a(bamemory.obj)
                0x00000000001399d0                RwFreeListPurge
                0x0000000000139b88                _rwMemoryOpen
                0x0000000000139a80                RwFreeListForAllUsed
                0x0000000000139b80                _rwMemoryClose
                0x00000000001397e0                RwFreeListPurgeAllFreeLists
                0x0000000000139908                RwFreeListDestroy
                0x0000000000139648                _rwFreeListAllocReal
                0x00000000001398e8                RwFreeListCreate
                0x00000000001399b8                _rwFreeListFreeReal
                0x00000000001398d8                RwOsGetMemoryInterface
 .text          0x0000000000139c70      0x7e8 E:/nightly/rwsdk.sky/rwsdk/lib/sky2/librwcore.a(baraster.obj)
                0x0000000000139c70                _rwRasterOpen
                0x0000000000139ea0                RwRasterGetOffset
                0x000000000013a2f8                RwRasterLockPalette
                0x000000000013a060                RwRasterPushContext
                0x000000000013a140                RwRasterGetCurrentContext
                0x0000000000139d38                RwRasterCreate
                0x000000000013a278                RwRasterLock
                0x0000000000139e30                RwRasterDestroy
                0x000000000013a0d8                RwRasterPopContext
                0x000000000013a1e0                RwRasterClearRect
                0x000000000013a378                RwRasterRegisterPlugin
                0x000000000013a2b8                RwRasterUnlock
                0x0000000000139f08                RwRasterSubRaster
                0x000000000013a3e8                RwRasterValidatePlugins
                0x000000000013a028                RwRasterRenderScaled
                0x000000000013a330                RwRasterUnlockPalette
                0x000000000013a210                RwRasterShowRaster
                0x0000000000139fa8                RwRasterRenderFast
                0x0000000000139fe8                RwRasterRender
                0x0000000000139eb8                RwRasterGetNumLevels
                0x000000000013a168                RwRasterClear
                0x000000000013a3c0                RwRasterGetPluginOffset
                0x000000000013a3f0                _rwRasterClose
 .text          0x000000000013a458      0x950 E:/nightly/rwsdk.sky/rwsdk/lib/sky2/librwcore.a(baresamp.obj)
                0x000000000013ac78                RwImageCreateResample
                0x000000000013aa68                RwImageResample
 .text          0x000000000013ada8      0x7e4 E:/nightly/rwsdk.sky/rwsdk/lib/sky2/librwcore.a(baresour.obj)
                0x000000000013b348                RwResourcesGetArenaUsage
                0x000000000013b430                _rwResourcesPurge
                0x000000000013b330                RwResourcesGetArenaSize
                0x000000000013b4c0                RwResourcesUseResEntry
                0x000000000013b208                RwResourcesEmptyArena
                0x000000000013b108                RwResourcesSetArenaSize
                0x000000000013b518                _rwResourcesClose
                0x000000000013b388                RwResourcesFreeResEntry
                0x000000000013aed8                _rwResourcesAllocateResEntry
                0x000000000013ada8                _rwResourcesOpen
 *fill*         0x000000000013b58c 0x303ec800000004
 .text          0x000000000013b590      0x9c4 E:/nightly/rwsdk.sky/rwsdk/lib/sky2/librwcore.a(bastream.obj)
                0x000000000013bd80                RwStreamClose
                0x000000000013b9a0                RwStreamWrite
                0x000000000013bf00                _rwStreamModuleClose
                0x000000000013bb90                RwStreamSkip
                0x000000000013bcd8                RwStreamOpen
                0x000000000013be98                _rwStreamModuleOpen
                0x000000000013b800                RwStreamRead
                0x000000000013b590                _rwStreamInitialize
 *fill*         0x000000000013bf54 0x303ec800000004
 .text          0x000000000013bf58      0x494 E:/nightly/rwsdk.sky/rwsdk/lib/sky2/librwcore.a(basync.obj)
                0x000000000013c150                _rwFrameSyncHierarchyLTM
                0x000000000013c0e8                _rwFrameSyncDirty
 *fill*         0x000000000013c3ec 0x303ec800000004
 .text          0x000000000013c3f0     0x23b8 E:/nightly/rwsdk.sky/rwsdk/lib/sky2/librwcore.a(batextur.obj)
                0x000000000013e298                RwTextureSetRaster
                0x000000000013e2f8                RwTextureSetAddressing
                0x000000000013dd10                RwTextureSetAutoMipmapping
                0x000000000013e328                RwTexDictionaryAddTexture
                0x000000000013e618                RwTexDictionaryRegisterPlugin
                0x000000000013e4e0                RwTextureGetDictionary
                0x000000000013dd80                RwTextureSetMipmapNameCallBack
                0x000000000013e5d0                RwTextureRegisterPlugin
                0x000000000013de50                _rwTextureGetAutoMipMapState
                0x000000000013e688                RwTexDictionaryGetPluginOffset
                0x000000000013deb0                RwTextureSetName
                0x000000000013e558                RwTexDictionaryForAllTexDictionaries
                0x000000000013e140                RwTextureCreate
                0x000000000013e1c8                RwTextureAddRef
                0x000000000013d6f0                RwTextureRead
                0x000000000013e6b0                RwTextureValidatePlugins
                0x000000000013e660                RwTextureGetPluginOffset
                0x000000000013e3b8                RwTexDictionaryFindNamedTexture
                0x000000000013e318                RwTextureSetAddressingV
                0x000000000013de68                RwTextureGetReadCallBack
                0x000000000013db10                _rwTextureOpen
                0x000000000013dcf8                RwTextureGetMipmapping
                0x000000000013e4a8                RwTexDictionaryGetCurrent
                0x000000000013e4e8                RwTexDictionaryForAllTextures
                0x000000000013df50                RwTextureSetMaskName
                0x000000000013dd48                RwTextureSetMipmapGenerationCallBack
                0x000000000013dcd8                RwTextureSetMipmapping
                0x000000000013e4c0                RwTexDictionarySetCurrent
                0x000000000013dd68                RwTextureGetMipmapGenerationCallBack
                0x000000000013de80                RwTextureSetReadCallBack
                0x000000000013e2e8                RwTextureSetFilterMode
                0x000000000013dff0                RwTexDictionaryCreate
                0x000000000013d970                _rwTextureClose
                0x000000000013e1e0                RwTextureDestroy
                0x000000000013dea8                RwTextureGetMaskName
                0x000000000013dda0                RwTextureGetMipmapNameCallBack
                0x000000000013ddf8                RwTextureRasterGenerateMipmaps
                0x000000000013ddb8                RwTextureGenerateMipmapName
                0x000000000013dd30                RwTextureGetAutoMipmapping
                0x000000000013e380                RwTexDictionaryRemoveTexture
                0x000000000013dea0                RwTextureGetName
                0x000000000013e6b8                RwTexDictionaryValidatePlugins
                0x000000000013e308                RwTextureSetAddressingU
                0x000000000013de30                _rwTextureSetAutoMipMapState
                0x000000000013e0a0                RwTexDictionaryDestroy
 .text          0x000000000013e7a8      0x458 E:/nightly/rwsdk.sky/rwsdk/lib/sky2/librwcore.a(batkreg.obj)
                0x000000000013eb30                _rwPluginRegistryCopyObject
                0x000000000013e860                _rwPluginRegistryAddPlugin
                0x000000000013e818                _rwPluginRegistrySetStaticPluginsSize
                0x000000000013e7d8                _rwPluginRegistryClose
                0x000000000013ea38                _rwPluginRegistryInitObject
                0x000000000013ead0                _rwPluginRegistryDeInitObject
                0x000000000013e7a8                _rwPluginRegistryOpen
                0x000000000013ea08                _rwPluginRegistryGetPluginOffset
 .text          0x000000000013ec00       0xa0 E:/nightly/rwsdk.sky/rwsdk/lib/sky2/librwcore.a(batypehf.obj)
                0x000000000013ec70                _rwObjectHasFrameReleaseFrame
                0x000000000013ec00                _rwObjectHasFrameSetFrame
 .text          0x000000000013eca0      0x828 E:/nightly/rwsdk.sky/rwsdk/lib/sky2/librwcore.a(bavector.obj)
                0x000000000013efc0                RwV2dLength
                0x000000000013f220                _rwVectorOpen
                0x000000000013f338                _rwVectorSetMultFn
                0x000000000013f0c0                RwV3dTransformVectors
                0x000000000013f1a0                _rwV3dNormalize
                0x000000000013f2a0                _rwVectorClose
                0x000000000013ef90                RwV3dLength
                0x000000000013f0f0                _rwSqrt
                0x000000000013f148                _rwInvSqrt
                0x000000000013eec8                RwV3dNormalize
                0x000000000013f090                RwV3dTransformPoints
                0x000000000013efe0                RwV2dNormalize
 .text          0x000000000013f4c8      0x688 E:/nightly/rwsdk.sky/rwsdk/lib/sky2/librwcore.a(resmem.obj)
                0x000000000013f980                _rwResHeapClose
                0x000000000013f928                _rwResHeapInit
                0x000000000013f9d8                _rwResHeapFree
                0x000000000013fa90                _rwResHeapGetStats
                0x000000000013f4c8                _rwResHeapAlloc
                0x000000000013f988                _rwResHeapCalloc
                0x000000000013f610                _rwResHeapRealloc
 .text          0x000000000013fb50      0x260 E:/nightly/rwsdk.sky/rwsdk/lib/sky2/librwcore.a(rwstring.obj)
                0x000000000013fc40                _rwStringClose
                0x000000000013fb50                _rwStringOpen
 .text          0x000000000013fdb0     0x1198 E:/nightly/rwsdk.sky/rwsdk/lib/sky2/librwcore.a(baim3d.obj)
                0x0000000000140df0                RwIm3DGetRenderPipeline
                0x0000000000140bc8                RwIm3DRenderTriangle
                0x0000000000140dd8                RwIm3DGetTransformPipeline
                0x0000000000140928                _rwIm3DClose
                0x000000000013ff40                RwIm3DRenderPrimitive
                0x0000000000140ce0                RwIm3DGetGenericTransformPipeline
                0x0000000000140ef0                RwIm3DSetTransformPipeline
                0x0000000000140cf8                RwIm3DGetGenericRenderPipeline
                0x00000000001406f0                _rwIm3DOpen
                0x000000000013fdb0                RwIm3DRenderIndexedPrimitive
                0x0000000000140a80                RwIm3DEnd
                0x0000000000140ad0                RwIm3DRenderLine
                0x00000000001400c8                RwIm3DSetRenderPipeline
                0x00000000001409c0                _rwIm3DGetPool
                0x00000000001409d8                RwIm3DTransform
 .text          0x0000000000140f48       0x68 E:/nightly/rwsdk.sky/rwsdk/lib/sky2/librwcore.a(bapipe.obj)
                0x0000000000140f78                _rwRenderPipelineClose
                0x0000000000140f48                _rwRenderPipelineOpen
                0x0000000000140fa8                _rwPipeInitForCamera
                0x0000000000140fa0                _rwPipeAttach
 .text          0x0000000000140fb0     0x1094 E:/nightly/rwsdk.sky/rwsdk/lib/sky2/librwcore.a(nodeClipLine.obj)
                0x0000000000142038                RxNodeDefinitionGetClipLine
 *fill*         0x0000000000142044 0x303ec800000004
 .text          0x0000000000142048     0x1624 E:/nightly/rwsdk.sky/rwsdk/lib/sky2/librwcore.a(nodeClipTriangle.obj)
                0x0000000000143660                RxNodeDefinitionGetClipTriangle
 *fill*         0x000000000014366c 0x303ec800000004
 .text          0x0000000000143670      0x824 E:/nightly/rwsdk.sky/rwsdk/lib/sky2/librwcore.a(nodeCullTriangle.obj)
                0x0000000000143e18                RxNodeDefinitionGetCullTriangle
 *fill*         0x0000000000143e94 0x303ec800000004
 .text          0x0000000000143e98      0x354 E:/nightly/rwsdk.sky/rwsdk/lib/sky2/librwcore.a(nodeImmInstance.obj)
                0x00000000001441e0                RxNodeDefinitionGetImmInstance
 *fill*         0x00000000001441ec 0x303ec800000004
 .text          0x00000000001441f0      0x36c E:/nightly/rwsdk.sky/rwsdk/lib/sky2/librwcore.a(nodeImmMangleLineIndices.obj)
                0x0000000000144550                RxNodeDefinitionGetImmMangleLineIndices
 *fill*         0x000000000014455c 0x303ec800000004
 .text          0x0000000000144560      0x524 E:/nightly/rwsdk.sky/rwsdk/lib/sky2/librwcore.a(nodeImmMangleTriangleIndices.obj)
                0x0000000000144a78                RxNodeDefinitionGetImmMangleTriangleIndices
 *fill*         0x0000000000144a84 0x303ec800000004
 .text          0x0000000000144a88      0x3d4 E:/nightly/rwsdk.sky/rwsdk/lib/sky2/librwcore.a(nodeImmRenderSetup.obj)
                0x0000000000144e50                RxNodeDefinitionGetImmRenderSetup
 *fill*         0x0000000000144e5c 0x303ec800000004
 .text          0x0000000000144e60      0x204 E:/nightly/rwsdk.sky/rwsdk/lib/sky2/librwcore.a(nodeImmStash.obj)
                0x0000000000145058                RxNodeDefinitionGetImmStash
 *fill*         0x0000000000145064 0x303ec800000004
 .text          0x0000000000145068      0x2f4 E:/nightly/rwsdk.sky/rwsdk/lib/sky2/librwcore.a(nodeSubmitLine.obj)
                0x0000000000145350                RxNodeDefinitionGetSubmitLine
 *fill*         0x000000000014535c 0x303ec800000004
 .text          0x0000000000145360      0x2a4 E:/nightly/rwsdk.sky/rwsdk/lib/sky2/librwcore.a(nodeSubmitTriangle.obj)
                0x00000000001455f8                RxNodeDefinitionGetSubmitTriangle
 *fill*         0x0000000000145604 0x303ec800000004
 .text          0x0000000000145608      0xcd4 E:/nightly/rwsdk.sky/rwsdk/lib/sky2/librwcore.a(nodeTransform.obj)
                0x0000000000146288                RxNodeDefinitionGetTransform
 *fill*         0x00000000001462dc 0x303ec800000004
 .text          0x00000000001462e0      0x3a8 E:/nightly/rwsdk.sky/rwsdk/lib/sky2/librwcore.a(p2altmdl.obj)
                0x00000000001465e8                _rxPacketDestroy
                0x00000000001462e0                _rxEmbeddedPacketBetweenPipelines
                0x0000000000146488                _rxEmbeddedPacketBetweenNodes
 .text          0x0000000000146688     0x1cd0 E:/nightly/rwsdk.sky/rwsdk/lib/sky2/librwcore.a(p2clpcom.obj)
                0x00000000001481c0                _rwGenerateParallelXHIClippedVertex
                0x0000000000146688                _rwForAllEdgesWithRxInterpolant
                0x0000000000146d38                _rwGeneratePerspClippedVertexYLO
                0x0000000000148030                _rwGenerateParallelXLOClippedVertex
                0x0000000000147710                _rwGenerateParallelYHIClippedVertex
                0x0000000000147d00                _rwGeneratePerspClippedVertexXLO
                0x0000000000146908                _rwGeneratePerspClippedVertexZLO
                0x0000000000147538                _rwGenerateParallelYLOClippedVertex
                0x00000000001478e8                _rwForAllEdgesWithoutRxInterpolant
                0x0000000000147310                _rwGenerateParallelZHIClippedVertex
                0x0000000000147af8                _rwForAllEdges
                0x0000000000146f08                _rwGeneratePerspClippedVertexYHI
                0x0000000000147b30                _rwForOneEdge
                0x0000000000146b20                _rwGeneratePerspClippedVertexZHI
                0x0000000000147e90                _rwGeneratePerspClippedVertexXHI
                0x00000000001470e8                _rwGenerateParallelZLOClippedVertex
 .text          0x0000000000148358      0x9ec E:/nightly/rwsdk.sky/rwsdk/lib/sky2/librwcore.a(p2core.obj)
                0x00000000001489a0                RxClusterInitializeData
                0x0000000000148490                _rxPipelineDestroy
                0x0000000000148cc8                RxClusterGetAttributes
                0x0000000000148c98                RxPipelineClusterGetCreationAttributes
                0x0000000000148ce0                RxClusterSetAttributes
                0x00000000001486e8                RxPipelineCreate
                0x0000000000148760                RxHeapGetGlobalHeap
                0x0000000000148860                RxClusterSetStride
                0x0000000000148828                RxPacketCreate
                0x0000000000148870                RxClusterSetExternalData
                0x0000000000148cf8                _rwPipelineCheckForTramplingOfNodePrivateSpace
                0x0000000000148650                _rxPipelineOpen
                0x0000000000148ab8                RxClusterDestroyData
                0x0000000000148768                RxPipelineExecute
                0x0000000000148c48                RxPipelineNodeGetPipelineCluster
                0x0000000000148cb0                RxPipelineClusterSetCreationAttributes
                0x0000000000148358                RxClusterLockWrite
                0x0000000000148a38                RxClusterResizeData
                0x00000000001486b8                _rxPipelineClose
                0x0000000000148b08                RxClusterUnlock
                0x0000000000148b10                RxPipelineNodeSendConfigMsg
                0x0000000000148b50                RxPipelineNodeForAllConnectedOutputs
                0x0000000000148908                RxClusterSetData
 *fill*         0x0000000000148d44 0x303ec800000004
 .text          0x0000000000148d48     0x2634 E:/nightly/rwsdk.sky/rwsdk/lib/sky2/librwcore.a(p2define.obj)
                0x000000000014a1f8                RxLockedPipeDeleteNode
                0x0000000000149e70                RxLockedPipeAddFragment
                0x000000000014b060                RxLockedPipeReplaceNode
                0x000000000014aaa0                RxPipelineNodeFindOutputByIndex
                0x000000000014a9f0                RxPipelineNodeFindOutputByName
                0x0000000000149d78                RxPipelineLock
                0x000000000014b298                RxLockedPipeAddPath
                0x000000000014aad8                RxPipelineNodeFindInput
                0x000000000014ae28                RxPipelineClone
                0x000000000014a3a0                RxPipelineInsertDebugNode
                0x000000000014b328                RxLockedPipeDeletePath
                0x000000000014aed8                RxPipelineFindNodeByName
                0x000000000014b030                RxPipelineFindNodeByIndex
                0x000000000014b248                RxLockedPipeGetEntryPoint
                0x000000000014aaf8                RxPipelineNodeCloneDefinition
                0x000000000014ad78                RxPipelineNodeCreateInitData
                0x000000000014ac88                RxPipelineNodeReplaceCluster
                0x000000000014ab98                RxPipelineNodeRequestCluster
                0x000000000014b1d0                RxLockedPipeSetEntryPoint
                0x0000000000149b60                RxLockedPipeUnlock
                0x000000000014ad68                RxPipelineNodeGetInitData
 *fill*         0x000000000014b37c 0x303ec800000004
 .text          0x000000000014b380     0x1b44 E:/nightly/rwsdk.sky/rwsdk/lib/sky2/librwcore.a(p2dep.obj)
                0x000000000014ccb0                _rxChaseDependencies
 *fill*         0x000000000014cec4 0x303ec800000004
 .text          0x000000000014cec8      0xf8c E:/nightly/rwsdk.sky/rwsdk/lib/sky2/librwcore.a(p2heap.obj)
                0x000000000014d548                RxHeapAlloc
                0x000000000014dcc0                RxHeapCreate
                0x000000000014d2f0                RxHeapFree
                0x000000000014d768                RxHeapRealloc
                0x000000000014d920                RxHeapReset
                0x000000000014ddb8                RxHeapDestroy
 *fill*         0x000000000014de54 0x303ec800000004
 .text          0x000000000014de58      0x508 E:/nightly/rwsdk.sky/rwsdk/lib/sky2/librwcore.a(p2renderstate.obj)
                0x000000000014e170                RxRenderStateVectorGetDefaultRenderStateVector
                0x000000000014de58                RxRenderStateVectorSetDefaultRenderStateVector
                0x000000000014dfc8                RxRenderStateVectorLoadDriverState
                0x000000000014e1d0                RxRenderStateVectorCreate
                0x000000000014e310                RxRenderStateVectorDestroy
 .text          0x000000000014e360      0x5a8 E:/nightly/rwsdk.sky/rwsdk/lib/sky2/librwcore.a(p2resort.obj)
                0x000000000014e360                _rx_rxRadixExchangeSort
                0x000000000014e7d8                _rxSelectionSort
 .text          0x000000000014e908       0x20 E:/nightly/rwsdk.sky/rwsdk/lib/sky2/librwcore.a(im3dpipe.obj)
                0x000000000014e920                _rwIm3DDestroyPlatformRenderPipelines
                0x000000000014e908                _rwIm3DCreatePlatformTransformPipeline
                0x000000000014e910                _rwIm3DCreatePlatformRenderPipelines
                0x000000000014e918                _rwIm3DDestroyPlatformTransformPipeline
 .text          0x000000000014e928     0x9010 E:/nightly/rwsdk.sky/rwsdk/lib/sky2/librwcore.a(basky.obj)
                0x0000000000157318                RpSkyGetTrueTLClipper
                0x00000000001573e8                RpSkyGetDrawBufferRaster
                0x000000000014e928                _rwSkySetRenderState
                0x0000000000157220                RpSkyTextureSetMipmapL
                0x0000000000157160                RpSkyTextureGetDefaultMipmapK
                0x0000000000157000                _skyRasterGetTwiddling
                0x000000000014f588                RpSkyRenderStateSet
                0x00000000001573e0                RpSkyGetDisplayBufferRaster
                0x0000000000157098                RpSkySelectDeepZBuffer
                0x0000000000156fc8                RpSkySuspend
                0x0000000000156f58                _rwSkyFindMSB
                0x00000000001573f0                _rpSkyCreateFrameBufferRasters
                0x0000000000156f48                _rwDeviceGetHandle
                0x00000000001572c0                RpSkyTextureGetMipmapL
                0x0000000000157018                _skyRasterSetTwiddling
                0x0000000000157308                RpSkySelectTrueTLClipper
                0x00000000001572f0                RpSkySelectTrueTSClipper
                0x0000000000157040                _rpSkyFrameBufferRastersUpdate
                0x00000000001570d8                RpSkyTextureSetDefaultMipmapK
                0x0000000000156f78                _rwSkyFSAAMode0SetVisibleWidth
                0x0000000000157320                RpSkyRenderStateGet
                0x0000000000157268                RpSkyTextureGetMipmapK
                0x00000000001571a8                RpSkyTextureSetMipmapK
                0x0000000000156c28                RpSkyResume
                0x0000000000157198                RpSkyTextureGetDefaultMipmapL
                0x0000000000157300                RpSkyGetTrueTSClipper
                0x0000000000157140                RpSkyTextureSetDefaultMipmapL
 .text          0x0000000000157938      0x18c E:/nightly/rwsdk.sky/rwsdk/lib/sky2/librwcore.a(baskytran.obj)
                0x00000000001579b0                vectorASMMultPoint
                0x0000000000157938                matrixASMMult
                0x0000000000157a40                vectorASMMultVector
 *fill*         0x0000000000157ac4 0x303ec800000004
 .text          0x0000000000157ac8     0x1f34 E:/nightly/rwsdk.sky/rwsdk/lib/sky2/librwcore.a(skyblit.obj)
                0x0000000000158a90                _rwSkyRasterRender
                0x0000000000158fb8                _rwSkyRasterRenderScaled
                0x0000000000159940                _rwSkyRasterInitiateStop
                0x00000000001598d0                _rwSkyRasterFinaliseStart
                0x00000000001599c8                _rwSkyRasterSetContext
                0x0000000000159550                _rwSkyRasterRenderFast
                0x0000000000159980                _rwSkyRasterClear
                0x0000000000157f98                _rwSkyRasterClearRect
 *fill*         0x00000000001599fc 0x303ec800000004
 .text          0x0000000000159a00     0x1958 E:/nightly/rwsdk.sky/rwsdk/lib/sky2/librwcore.a(skyconv.obj)
                0x000000000015b068                _rwSkyRGBToPixel
                0x000000000015b248                _rwSkyRasterSetImage
                0x000000000015b160                _rwSkyPixelToRGB
                0x0000000000159a00                _rwSkyImageFindRasterFormat
                0x0000000000159b88                _rwSkyImageGetRaster
 .text          0x000000000015b358     0x2e70 E:/nightly/rwsdk.sky/rwsdk/lib/sky2/librwcore.a(skyinst.obj)
                0x000000000015dcc0                _rwSkyPipeSetupForCamera
                0x000000000015dfe0                _rwSkyOverloadPipelines
                0x000000000015b858                openVU1SetupPkt
                0x000000000015e030                _rwSkyUnOverloadPipelines
 .text          0x000000000015e1c8     0x2fa0 E:/nightly/rwsdk.sky/rwsdk/lib/sky2/librwcore.a(texcache.obj)
                0x0000000000160ea8                RpSkyTexGetTex0
                0x0000000000160e00                RpSkyTexCacheDisable
                0x0000000000160f80                RpSkyUploadPixelData
                0x0000000000160f20                RpSkyTexGetMiptbp12
                0x0000000000160f98                skyFillInPktForUpLoadAlignedContiguousRectangle
                0x0000000000160e78                RpSkyTexCacheRasterGetAddr
                0x0000000000160548                RpSkyTexCacheReleaseRaster
                0x0000000000160070                skyTexCacheCloseCache
                0x00000000001609a8                RpSkyTexCacheFlush
                0x0000000000160a58                RpSkyTexCacheRestore
                0x0000000000160ec8                RpSkyTexSetMiptbp1
                0x0000000000160f00                RpSkyTexSetMiptbp12
                0x0000000000160ca0                RpSkyTexCacheAccessSpeculate
                0x000000000015e440                skyPrepareUploadRaster
                0x0000000000160e50                RpSkyTexCacheSetCallBack
                0x0000000000160e90                RpSkyTexSetTex0
                0x0000000000160f88                RpSkyTexCacheUploadRaster
                0x0000000000160ee0                RpSkyTexGetMiptbp1
                0x00000000001606f0                RpSkyTexCacheRasterLock
                0x0000000000160df8                RpSkyTextureCacheSetState
                0x000000000015ff78                skyTexCacheOpenCache
                0x0000000000160e40                RpSkyTexGetSize
                0x0000000000160f50                RpSkyTexCacheValidateRaster
                0x0000000000160f90                skyTexCacheEndFrame
                0x0000000000160198                RpSkyTexCacheAccessRaster
                0x0000000000160d58                RpSkyTexCacheRasterUnlockAll
                0x0000000000160e30                RpSkyTexGetStartAddress
 .text          0x0000000000161168     0x1a24 E:/nightly/rwsdk.sky/rwsdk/lib/sky2/librwcore.a(imrascnv.obj)
                0x0000000000162710                _rwMipmapRasterSetFromImage4444
                0x00000000001616a8                _rwRasterSetFromImage4444
                0x0000000000162590                _rwMipmapRasterSetFromImage888
                0x0000000000161a68                _rwRasterSetFromImage565
                0x0000000000162130                _rwImageSetFromRaster4444
                0x0000000000161c30                _rwRGBAFromImage8
                0x0000000000161fe0                _rwImageSetFromRaster888
                0x0000000000161d20                _rwRGBAFromImage32
                0x0000000000162210                _rwImageSetFromRaster1555
                0x0000000000162a18                _rwMipmapRasterSetFromImage565
                0x0000000000161328                _rwRasterSetFromImage8888
                0x0000000000161dc8                _rwImageFindNearestPaletteColor
                0x00000000001614f0                _rwRasterSetFromImage888
                0x0000000000162890                _rwMipmapRasterSetFromImage1555
                0x0000000000162418                _rwMipmapRasterSetFromImage8888
                0x0000000000161168                _rwImageFindAlphaType
                0x0000000000161880                _rwRasterSetFromImage1555
                0x0000000000161ef8                _rwImageSetFromRaster8888
                0x0000000000162318                _rwImageSetFromRaster565
 *fill*         0x0000000000162b8c 0x303ec800000004
 .text          0x0000000000162b90     0x210c E:/nightly/rwsdk.sky/rwsdk/lib/sky2/librwcore.a(palquant.obj)
                0x0000000000164368                _rwPalQuantMatchImage
                0x0000000000164930                _rwPalQuantInit
                0x0000000000162b90                _rwPalQuantAddImage
                0x0000000000164a38                _rwPalQuantTerm
                0x0000000000163e98                _rwPalQuantResolvePalette
 *fill*         0x0000000000164c9c 0x303ec800000004
 .text          0x0000000000164ca0       0x50 E:/nightly/rwsdk.sky/rwsdk/lib/sky2/librwcore.a(osintf.obj)
                0x0000000000164ce8                _rwgetcurrenttime
                0x0000000000164ca0                _rwpathisabsolute
 .text          0x0000000000164cf0      0x260 E:/nightly/rwsdk.sky/rwsdk/lib/sky2/librwcore.a(babbox.obj)
                0x0000000000164cf0                RwBBoxCalculate
                0x0000000000164eb8                RwBBoxContainsPoint
                0x0000000000164de0                RwBBoxInitialize
                0x0000000000164e18                RwBBoxAddPoint
 .text          0x0000000000164f50     0x1120 E:/nightly/rwsdk.sky/rwsdk/lib/sky2/librwcore.a(babintex.obj)
                0x0000000000164f50                _rwStringStreamFindAndRead
                0x0000000000165df8                RwTexDictionaryRegisterPluginStream
                0x0000000000165888                RwTexDictionaryStreamRead
                0x0000000000165d20                RwTextureChunkInfoRead
                0x0000000000165500                RwTextureStreamRead
                0x0000000000165e58                RwTexDictionaryStreamGetSize
                0x0000000000165c18                RwTextureRegisterPluginStream
                0x0000000000165e30                RwTexDictionarySetStreamAlwaysCallBack
                0x00000000001652b8                RwTextureStreamWrite
                0x0000000000165c50                RwTextureSetStreamAlwaysCallBack
                0x0000000000165b20                _rwStringDestroy
                0x0000000000165b80                _rwStringStreamWrite
                0x0000000000165c78                RwTextureStreamGetSize
                0x0000000000165740                RwTexDictionaryStreamWrite
                0x0000000000165b48                _rwStringStreamGetSize
 .text          0x0000000000166070       0x2c E:/nightly/rwsdk.sky/rwsdk/lib/sky2/librwcore.a(bacolor.obj)
                0x0000000000166088                _rwColorClose
                0x0000000000166070                _rwColorOpen
 *fill*         0x000000000016609c 0x303ec800000004
 .text          0x00000000001660a0      0x444 E:/nightly/rwsdk.sky/rwsdk/lib/sky2/librwcore.a(batkbin.obj)
                0x0000000000166268                _rwPluginRegistryAddPlgnStrmlwysCB
                0x0000000000166470                _rwPluginRegistryGetSize
                0x0000000000166228                _rwPluginRegistryAddPluginStream
                0x00000000001660a0                _rwPluginRegistryReadDataChunks
                0x00000000001663d0                _rwPluginRegistrySkipDataChunks
                0x00000000001662a0                _rwPluginRegistryWriteDataChunks
 *fill*         0x00000000001664e4 0x303ec800000004
 .text          0x00000000001664e8     0x2b40 E:/nightly/rwsdk.sky/rwsdk/lib/sky2/librwcore.a(badma.obj)
                0x0000000000168c00                _sweUnhook
                0x0000000000166cd0                _sweGarbageCollectChain
                0x0000000000168f10                _sweProcrastinatedAddURef
                0x0000000000167d68                _sweOpen
                0x0000000000168b60                _sweWaitQueue
                0x0000000000167bb8                _sweHook
                0x0000000000169020                _sweReadTimer
                0x0000000000168058                _sweClose
                0x0000000000168fe8                sweDmaSend
                0x0000000000168dd0                _sweWaitFlip
                0x0000000000168850                _sweAddCont
                0x00000000001664e8                sweCloseLocalPkt
                0x00000000001667b0                sweOpenLocalPkt
                0x0000000000168f88                _swePreAlloc
                0x0000000000168de8                _sweAddPkt
                0x0000000000166a98                sweFinaliseOpenLocalPkt
                0x0000000000168228                _sweFlush
                0x0000000000166660                sweFlushPURef
                0x0000000000168d20                _sweReqFlip
                0x00000000001689d8                _sweAddPrim
                0x0000000000168748                _sweAppendToChain
 .text          0x0000000000169028       0x6c E:/nightly/rwsdk.sky/rwsdk/lib/sky2/librwcore.a(baevent.obj)
                0x0000000000169028                _rwSkyInitConfigSystem
 *fill*         0x0000000000169094 0x303ec800000004
 .text          0x0000000000169098      0x828 E:/nightly/rwsdk.sky/rwsdk/lib/sky2/librwcore.a(dmaalloc.obj)
                0x0000000000169290                circularAllocOpen
                0x0000000000169878                circularLimitAlloc
                0x0000000000169790                circularAllocClose
                0x0000000000169710                circularFree
                0x00000000001693a8                circularAllocPreAlloc
                0x00000000001695a8                circularMalloc
                0x0000000000169628                circularRealloc
 .text          0x00000000001698c0      0x19c E:/usr/local/sce/ee/lib/libgraph.a(graph001.o)
                0x0000000000169a50                sceGsGetGParam
                0x00000000001698c0                sceGsResetGraph
 *fill*         0x0000000000169a5c 0x303ec800000004
 .text          0x0000000000169a60       0x68 E:/usr/local/sce/ee/lib/libgraph.a(graph002.o)
                0x0000000000169a60                sceGsResetPath
 .text          0x0000000000169ac8       0x94 E:/usr/local/sce/ee/lib/libgraph.a(graph011.o)
                0x0000000000169ac8                sceGsSyncV
 *fill*         0x0000000000169b5c 0x303ec800000004
 .text          0x0000000000169b60      0x314 E:/usr/local/sce/ee/lib/libgraph.a(graph012.o)
                0x0000000000169b60                sceGsSyncPath
 *fill*         0x0000000000169e74 0x303ec800000004
 .text          0x0000000000169e78      0x140 E:/usr/local/sce/ee/lib/libgraph.a(graph016.o)
                0x0000000000169e78                sceGsSetDefStoreImage
 .text          0x0000000000169fb8      0x68c E:/usr/local/sce/ee/lib/libgraph.a(graph018.o)
                0x0000000000169fb8                sceGsExecStoreImage
 *fill*         0x000000000016a644 0x303ec800000004
 .text          0x000000000016a648       0x88 E:/usr/local/sce/ee/lib/libgraph.a(graph021.o)
                0x000000000016a648                sceGsSetHalfOffset
 .text          0x000000000016a6d0       0x88 E:/usr/local/sce/ee/lib/libgraph.a(graph026.o)
                0x000000000016a6d0                sceGsSetHalfOffset2
 .text          0x000000000016a758      0x2e4 E:/usr/local/sce/ee/lib/libgraph.a(graph027.o)
                0x000000000016a758                sceGsSetDefDBuffDc
 *fill*         0x000000000016aa3c 0x303ec800000004
 .text          0x000000000016aa40       0x5c E:/usr/local/sce/ee/lib/libgraph.a(graph028.o)
                0x000000000016aa40                sceGsSwapDBuffDc
 *fill*         0x000000000016aa9c 0x303ec800000004
 .text          0x000000000016aaa0      0x270 E:/usr/local/sce/ee/lib/libgraph.a(graph003.o)
                0x000000000016aaa0                sceGsSetDefDispEnv
 .text          0x000000000016ad10       0xbc E:/usr/local/sce/ee/lib/libgraph.a(graph004.o)
                0x000000000016ad10                sceGsPutDispEnv
 *fill*         0x000000000016adcc 0x303ec800000004
 .text          0x000000000016add0       0xc8 E:/usr/local/sce/ee/lib/libgraph.a(graph005.o)
                0x000000000016add0                sceGszbufaddr
 .text          0x000000000016ae98      0x1e4 E:/usr/local/sce/ee/lib/libgraph.a(graph006.o)
                0x000000000016ae98                sceGsSetDefDrawEnv
 *fill*         0x000000000016b07c 0x303ec800000004
 .text          0x000000000016b080      0x104 E:/usr/local/sce/ee/lib/libgraph.a(graph007.o)
                0x000000000016b080                sceGsSetDefClear
 *fill*         0x000000000016b184 0x303ec800000004
 .text          0x000000000016b188       0xe8 E:/usr/local/sce/ee/lib/libgraph.a(graph008.o)
                0x000000000016b188                sceGsPutDrawEnv
 .text          0x000000000016b270      0x1e0 E:/usr/local/sce/ee/lib/libgraph.a(graph022.o)
                0x000000000016b270                sceGsSetDefDrawEnv2
 .text          0x000000000016b450      0xacc E:/usr/local/sce/ee/lib/libdma.a(libdma.o)
                0x000000000016bd28                sceDmaSync
                0x000000000016bc38                sceDmaRecvI
                0x000000000016bdf0                sceDmaWatch
                0x000000000016ba80                sceDmaRecv
                0x000000000016b8b0                sceDmaSendN
                0x000000000016bb48                sceDmaRecvN
                0x000000000016bf08                sceDmaRestart
                0x000000000016b4b0                sceDmaReset
                0x000000000016bec0                sceDmaPause
                0x000000000016b5a0                sceDmaPutEnv
                0x000000000016b590                sceDmaDebug
                0x000000000016b488                sceDmaGetChan
                0x000000000016b998                sceDmaSendI
                0x000000000016b7d8                sceDmaSend
                0x000000000016b7b0                sceDmaPutStallAddr
                0x000000000016b778                sceDmaGetEnv
 *fill*         0x000000000016bf1c 0x303ec800000004
 .text          0x000000000016bf20     0x13a8 E:/usr/local/sce/ee/lib/libpad.a(libpad.o)
                0x000000000016cf48                scePadInfoPressMode
                0x000000000016cb98                scePadSetMainMode
                0x000000000016c2b0                scePadPortOpen
                0x000000000016c798                scePadGetReqState
                0x000000000016cc50                scePadSetActDirect
                0x000000000016c5b0                scePadGetFrameCount
                0x000000000016c820                scePadInfoAct
                0x000000000016c680                scePadGetState
                0x000000000016ca60                scePadInfoMode
                0x000000000016c050                scePadInit
                0x000000000016cfa8                scePadEnterPressMode
                0x000000000016c230                scePadEnd
                0x000000000016c7e8                scePadReqIntToStr
                0x000000000016d190                scePadGetSlotMax
                0x000000000016c498                scePadPortClose
                0x000000000016c600                scePadRead
                0x000000000016cd08                scePadSetActAlign
                0x000000000016c6f8                scePadStateIntToStr
                0x000000000016d000                scePadExitPressMode
                0x000000000016c940                scePadInfoComb
                0x000000000016d260                scePadSetWarningLevel
 .text          0x000000000016d2c8       0xd4 E:/usr/local/sce/ee/gcc/lib/gcc-lib/ee\2.95.2\../../../../ee\lib\libm.a(sf_ceil.o)
                0x000000000016d2c8                ceilf
 *fill*         0x000000000016d39c 0x303ec800000004
 .text          0x000000000016d3a0       0xe8 E:/usr/local/sce/ee/gcc/lib/gcc-lib/ee\2.95.2\../../../../ee\lib\libm.a(sf_cos.o)
                0x000000000016d3a0                cosf
 .text          0x000000000016d488       0xf0 E:/usr/local/sce/ee/gcc/lib/gcc-lib/ee\2.95.2\../../../../ee\lib\libm.a(sf_sin.o)
                0x000000000016d488                sinf
 .text          0x000000000016d578      0x430 E:/usr/local/sce/ee/gcc/lib/gcc-lib/ee\2.95.2\../../../../ee\lib\libm.a(w_pow.o)
                0x000000000016d578                pow
 .text          0x000000000016d9a8       0xfc E:/usr/local/sce/ee/gcc/lib/gcc-lib/ee\2.95.2\../../../../ee\lib\libm.a(wf_acos.o)
                0x000000000016d9a8                acosf
 *fill*         0x000000000016daa4 0x303ec800000004
 .text          0x000000000016daa8      0x128 E:/usr/local/sce/ee/gcc/lib/gcc-lib/ee\2.95.2\../../../../ee\lib\libm.a(wf_atan2.o)
                0x000000000016daa8                atan2f
 .text          0x000000000016dbd0      0x508 E:/usr/local/sce/ee/gcc/lib/gcc-lib/ee\2.95.2\../../../../ee\lib\libm.a(wf_pow.o)
                0x000000000016dbd0                powf
 .text          0x000000000016e0d8      0xd28 E:/usr/local/sce/ee/gcc/lib/gcc-lib/ee\2.95.2\../../../../ee\lib\libm.a(e_pow.o)
                0x000000000016e0d8                __ieee754_pow
 .text          0x000000000016ee00      0x304 E:/usr/local/sce/ee/gcc/lib/gcc-lib/ee\2.95.2\../../../../ee\lib\libm.a(e_sqrt.o)
                0x000000000016ee00                __ieee754_sqrt
 *fill*         0x000000000016f104 0x303ec800000004
 .text          0x000000000016f108      0x430 E:/usr/local/sce/ee/gcc/lib/gcc-lib/ee\2.95.2\../../../../ee\lib\libm.a(ef_acos.o)
                0x000000000016f108                __ieee754_acosf
 .text          0x000000000016f538      0x2e8 E:/usr/local/sce/ee/gcc/lib/gcc-lib/ee\2.95.2\../../../../ee\lib\libm.a(ef_atan2.o)
                0x000000000016f538                __ieee754_atan2f
 .text          0x000000000016f820      0x88c E:/usr/local/sce/ee/gcc/lib/gcc-lib/ee\2.95.2\../../../../ee\lib\libm.a(ef_pow.o)
                0x000000000016f820                __ieee754_powf
 *fill*         0x00000000001700ac 0x303ec800000004
 .text          0x00000000001700b0      0x3e0 E:/usr/local/sce/ee/gcc/lib/gcc-lib/ee\2.95.2\../../../../ee\lib\libm.a(ef_rem_pio2.o)
                0x00000000001700b0                __ieee754_rem_pio2f
 .text          0x0000000000170490      0x138 E:/usr/local/sce/ee/gcc/lib/gcc-lib/ee\2.95.2\../../../../ee\lib\libm.a(ef_sqrt.o)
                0x0000000000170490                __ieee754_sqrtf
 .text          0x00000000001705c8      0x158 E:/usr/local/sce/ee/gcc/lib/gcc-lib/ee\2.95.2\../../../../ee\lib\libm.a(kf_cos.o)
                0x00000000001705c8                __kernel_cosf
 .text          0x0000000000170720      0x94c E:/usr/local/sce/ee/gcc/lib/gcc-lib/ee\2.95.2\../../../../ee\lib\libm.a(kf_rem_pio2.o)
                0x0000000000170720                __kernel_rem_pio2f
 *fill*         0x000000000017106c 0x303ec800000004
 .text          0x0000000000171070      0x104 E:/usr/local/sce/ee/gcc/lib/gcc-lib/ee\2.95.2\../../../../ee\lib\libm.a(kf_sin.o)
                0x0000000000171070                __kernel_sinf
 *fill*         0x0000000000171174 0x303ec800000004
 .text          0x0000000000171178       0x34 E:/usr/local/sce/ee/gcc/lib/gcc-lib/ee\2.95.2\../../../../ee\lib\libm.a(s_fabs.o)
                0x0000000000171178                fabs
 *fill*         0x00000000001711ac 0x303ec800000004
 .text          0x00000000001711b0       0x20 E:/usr/local/sce/ee/gcc/lib/gcc-lib/ee\2.95.2\../../../../ee\lib\libm.a(s_finite.o)
                0x00000000001711b0                finite
 .text          0x00000000001711d0       0x38 E:/usr/local/sce/ee/gcc/lib/gcc-lib/ee\2.95.2\../../../../ee\lib\libm.a(s_isnan.o)
                0x00000000001711d0                isnan
 .text          0x0000000000171208       0x24 E:/usr/local/sce/ee/gcc/lib/gcc-lib/ee\2.95.2\../../../../ee\lib\libm.a(s_matherr.o)
                0x0000000000171208                matherr
 *fill*         0x000000000017122c 0x303ec800000004
 .text          0x0000000000171230      0x1fc E:/usr/local/sce/ee/gcc/lib/gcc-lib/ee\2.95.2\../../../../ee\lib\libm.a(s_rint.o)
                0x0000000000171230                rint
 *fill*         0x000000000017142c 0x303ec800000004
 .text          0x0000000000171430      0x1b4 E:/usr/local/sce/ee/gcc/lib/gcc-lib/ee\2.95.2\../../../../ee\lib\libm.a(s_scalbn.o)
                0x0000000000171430                scalbn
 *fill*         0x00000000001715e4 0x303ec800000004
 .text          0x00000000001715e8      0x2a8 E:/usr/local/sce/ee/gcc/lib/gcc-lib/ee\2.95.2\../../../../ee\lib\libm.a(sf_atan.o)
                0x00000000001715e8                atanf
 .text          0x0000000000171890       0x1c E:/usr/local/sce/ee/gcc/lib/gcc-lib/ee\2.95.2\../../../../ee\lib\libm.a(sf_fabs.o)
                0x0000000000171890                fabsf
 *fill*         0x00000000001718ac 0x303ec800000004
 .text          0x00000000001718b0       0x24 E:/usr/local/sce/ee/gcc/lib/gcc-lib/ee\2.95.2\../../../../ee\lib\libm.a(sf_finite.o)
                0x00000000001718b0                finitef
 *fill*         0x00000000001718d4 0x303ec800000004
 .text          0x00000000001718d8       0xe4 E:/usr/local/sce/ee/gcc/lib/gcc-lib/ee\2.95.2\../../../../ee\lib\libm.a(sf_floor.o)
                0x00000000001718d8                floorf
 *fill*         0x00000000001719bc 0x303ec800000004
 .text          0x00000000001719c0       0x24 E:/usr/local/sce/ee/gcc/lib/gcc-lib/ee\2.95.2\../../../../ee\lib\libm.a(sf_isnan.o)
                0x00000000001719c0                isnanf
 *fill*         0x00000000001719e4 0x303ec800000004
 .text          0x00000000001719e8      0x160 E:/usr/local/sce/ee/gcc/lib/gcc-lib/ee\2.95.2\../../../../ee\lib\libm.a(sf_scalbn.o)
                0x00000000001719e8                scalbnf
 .text          0x0000000000171b48       0x44 E:/usr/local/sce/ee/gcc/lib/gcc-lib/ee\2.95.2\../../../../ee\lib\libm.a(s_copysign.o)
                0x0000000000171b48                copysign
 *fill*         0x0000000000171b8c 0x303ec800000004
 .text          0x0000000000171b90       0x30 E:/usr/local/sce/ee/gcc/lib/gcc-lib/ee\2.95.2\../../../../ee\lib\libm.a(sf_copysign.o)
                0x0000000000171b90                copysignf
 .text          0x0000000000171bc0      0x128 E:/usr/local/sce/ee/gcc/lib/gcc-lib/ee\2.95.2\libgcc.a(__main.o)
                0x0000000000171cc8                __main
                0x0000000000171bc0                __do_global_dtors
                0x0000000000171c18                __do_global_ctors
 .text          0x0000000000171ce8       0x5c E:/usr/local/sce/ee/gcc/lib/gcc-lib/ee\2.95.2\libgcc.a(_fixdfdi.o)
                0x0000000000171ce8                __fixdfdi
 *fill*         0x0000000000171d44 0x303ec800000004
 .text          0x0000000000171d48       0xec E:/usr/local/sce/ee/gcc/lib/gcc-lib/ee\2.95.2\libgcc.a(_fixunsdfdi.o)
                0x0000000000171d48                __fixunsdfdi
 *fill*         0x0000000000171e34 0x303ec800000004
 .text          0x0000000000171e38       0x98 E:/usr/local/sce/ee/gcc/lib/gcc-lib/ee\2.95.2\libgcc.a(_floatdidf.o)
                0x0000000000171e38                __floatdidf
 .text          0x0000000000171ed0       0xe0 E:/usr/local/sce/ee/gcc/lib/gcc-lib/ee\2.95.2\libgcc.a(_floatdisf.o)
                0x0000000000171ed0                __floatdisf
 .text          0x0000000000171fb0       0x60 E:/usr/local/sce/ee/gcc/lib/gcc-lib/ee\2.95.2\libgcc.a(_muldi3.o)
                0x0000000000171fb0                __muldi3
 .text          0x0000000000172010      0x5d0 E:/usr/local/sce/ee/gcc/lib/gcc-lib/ee\2.95.2\libgcc.a(_udivdi3.o)
                0x0000000000172010                __udivdi3
 .text          0x00000000001725e0      0x540 E:/usr/local/sce/ee/gcc/lib/gcc-lib/ee\2.95.2\libgcc.a(_umoddi3.o)
                0x00000000001725e0                __umoddi3
 .text          0x0000000000172b20      0xcf4 E:/usr/local/sce/ee/gcc/lib/gcc-lib/ee\2.95.2\libgcc.a(dp-bit.o)
                0x0000000000173790                __make_dp
                0x0000000000172f88                dpsub
                0x0000000000172ff0                dpmul
                0x00000000001737c0                dptofp
                0x0000000000173518                dpcmp
                0x0000000000172c50                __unpack_d
                0x00000000001736b8                dptoul
                0x0000000000173298                dpdiv
                0x0000000000173568                litodp
                0x0000000000173400                __fpcmp_parts_d
                0x0000000000173758                __negdf2
                0x0000000000172f30                dpadd
                0x0000000000173620                dptoli
                0x0000000000172b20                __pack_d
 *fill*         0x0000000000173814 0x303ec800000004
 .text          0x0000000000173818      0xbe0 E:/usr/local/sce/ee/gcc/lib/gcc-lib/ee\2.95.2\libgcc.a(fp-bit.o)
                0x0000000000174170                sitofp
                0x0000000000173ea8                fpdiv
                0x0000000000174388                __make_fp
                0x0000000000173928                __unpack_f
                0x00000000001742b8                fptoui
                0x0000000000173818                __pack_f
                0x00000000001743b8                fptodp
                0x0000000000174228                fptosi
                0x0000000000173bf0                fpadd
                0x0000000000174350                __negsf2
                0x0000000000173c48                fpsub
                0x0000000000174120                fpcmp
                0x0000000000173cb0                fpmul
                0x0000000000174008                __fpcmp_parts_f
 .text          0x00000000001743f8       0x2c E:/usr/local/sce/ee/gcc/lib/gcc-lib/ee\2.95.2\../../../../ee\lib\libc.a(calloc.o)
                0x00000000001743f8                calloc
 *fill*         0x0000000000174424 0x303ec800000004
 .text          0x0000000000174428       0xbc E:/usr/local/sce/ee/gcc/lib/gcc-lib/ee\2.95.2\../../../../ee\lib\libc.a(callocr.o)
                0x0000000000174428                _calloc_r
 *fill*         0x00000000001744e4 0x303ec800000004
 .text          0x00000000001744e8        0xc E:/usr/local/sce/ee/gcc/lib/gcc-lib/ee\2.95.2\../../../../ee\lib\libc.a(errno.o)
                0x00000000001744e8                __errno
 *fill*         0x00000000001744f4 0x303ec800000004
 .text          0x00000000001744f8      0x104 E:/usr/local/sce/ee/gcc/lib/gcc-lib/ee\2.95.2\../../../../ee\lib\libc.a(fclose.o)
                0x00000000001744f8                fclose
 *fill*         0x00000000001745fc 0x303ec800000004
 .text          0x0000000000174600       0x10 E:/usr/local/sce/ee/gcc/lib/gcc-lib/ee\2.95.2\../../../../ee\lib\libc.a(feof.o)
                0x0000000000174600                feof
 .text          0x0000000000174610      0x104 E:/usr/local/sce/ee/gcc/lib/gcc-lib/ee\2.95.2\../../../../ee\lib\libc.a(fflush.o)
                0x0000000000174610                fflush
 *fill*         0x0000000000174714 0x303ec800000004
 .text          0x0000000000174718      0x128 E:/usr/local/sce/ee/gcc/lib/gcc-lib/ee\2.95.2\../../../../ee\lib\libc.a(fgets.o)
                0x0000000000174718                fgets
 .text          0x0000000000174840      0x254 E:/usr/local/sce/ee/gcc/lib/gcc-lib/ee\2.95.2\../../../../ee\lib\libc.a(findfp.o)
                0x0000000000174a08                __sinit
                0x0000000000174898                __sfmoreglue
                0x00000000001749f8                _cleanup
                0x00000000001749e8                _cleanup_r
                0x0000000000174908                __sfp
 *fill*         0x0000000000174a94 0x303ec800000004
 .text          0x0000000000174a98      0x10c E:/usr/local/sce/ee/gcc/lib/gcc-lib/ee\2.95.2\../../../../ee\lib\libc.a(fopen.o)
                0x0000000000174b78                fopen
                0x0000000000174a98                _fopen_r
 *fill*         0x0000000000174ba4 0x303ec800000004
 .text          0x0000000000174ba8       0x50 E:/usr/local/sce/ee/gcc/lib/gcc-lib/ee\2.95.2\../../../../ee\lib\libc.a(fputs.o)
                0x0000000000174ba8                fputs
 .text          0x0000000000174bf8      0x11c E:/usr/local/sce/ee/gcc/lib/gcc-lib/ee\2.95.2\../../../../ee\lib\libc.a(fread.o)
                0x0000000000174bf8                fread
 *fill*         0x0000000000174d14 0x303ec800000004
 .text          0x0000000000174d18      0x48c E:/usr/local/sce/ee/gcc/lib/gcc-lib/ee\2.95.2\../../../../ee\lib\libc.a(freer.o)
                0x0000000000174d18                _free_r
                0x0000000000175038                _malloc_trim_r
 *fill*         0x00000000001751a4 0x303ec800000004
 .text          0x00000000001751a8      0x48c E:/usr/local/sce/ee/gcc/lib/gcc-lib/ee\2.95.2\../../../../ee\lib\libc.a(fseek.o)
                0x00000000001751a8                fseek
 *fill*         0x0000000000175634 0x303ec800000004
 .text          0x0000000000175638       0x5c E:/usr/local/sce/ee/gcc/lib/gcc-lib/ee\2.95.2\../../../../ee\lib\libc.a(fstatr.o)
                0x0000000000175638                _fstat_r
 *fill*         0x0000000000175694 0x303ec800000004
 .text          0x0000000000175698       0xfc E:/usr/local/sce/ee/gcc/lib/gcc-lib/ee\2.95.2\../../../../ee\lib\libc.a(ftell.o)
                0x0000000000175698                ftell
 *fill*         0x0000000000175794 0x303ec800000004
 .text          0x0000000000175798      0x3d8 E:/usr/local/sce/ee/gcc/lib/gcc-lib/ee\2.95.2\../../../../ee\lib\libc.a(fvwrite.o)
                0x0000000000175798                __sfvwrite
 .text          0x0000000000175b70       0x94 E:/usr/local/sce/ee/gcc/lib/gcc-lib/ee\2.95.2\../../../../ee\lib\libc.a(fwalk.o)
                0x0000000000175b70                _fwalk
 *fill*         0x0000000000175c04 0x303ec800000004
 .text          0x0000000000175c08       0x84 E:/usr/local/sce/ee/gcc/lib/gcc-lib/ee\2.95.2\../../../../ee\lib\libc.a(fwrite.o)
                0x0000000000175c08                fwrite
 *fill*         0x0000000000175c8c 0x303ec800000004
 .text          0x0000000000175c90      0x150 E:/usr/local/sce/ee/gcc/lib/gcc-lib/ee\2.95.2\../../../../ee\lib\libc.a(makebuf.o)
                0x0000000000175c90                __smakebuf
 .text          0x0000000000175de0       0x38 E:/usr/local/sce/ee/gcc/lib/gcc-lib/ee\2.95.2\../../../../ee\lib\libc.a(malloc.o)
                0x0000000000175de0                malloc
                0x0000000000175e08                free
 .text          0x0000000000175e18      0x9d0 E:/usr/local/sce/ee/gcc/lib/gcc-lib/ee\2.95.2\../../../../ee\lib\libc.a(mallocr.o)
                0x0000000000176070                _malloc_r
 .text          0x00000000001767e8       0xe0 E:/usr/local/sce/ee/gcc/lib/gcc-lib/ee\2.95.2\../../../../ee\lib\libc.a(memchr.o)
                0x00000000001767e8                memchr
 .text          0x00000000001768c8       0x94 E:/usr/local/sce/ee/gcc/lib/gcc-lib/ee\2.95.2\../../../../ee\lib\libc.a(memcmp.o)
                0x00000000001768c8                memcmp
 .text          0x000000000017695c       0xb0 E:/usr/local/sce/ee/gcc/lib/gcc-lib/ee\2.95.2\../../../../ee\lib\libc.a(memcpy.o)
                0x000000000017695c                memcpy
 .text          0x0000000000176a0c      0x104 E:/usr/local/sce/ee/gcc/lib/gcc-lib/ee\2.95.2\../../../../ee\lib\libc.a(memmove.o)
                0x0000000000176a0c                memmove
 .text          0x0000000000176b10       0xc0 E:/usr/local/sce/ee/gcc/lib/gcc-lib/ee\2.95.2\../../../../ee\lib\libc.a(memset.o)
                0x0000000000176b10                memset
 .text          0x0000000000176bd0       0x10 E:/usr/local/sce/ee/gcc/lib/gcc-lib/ee\2.95.2\../../../../ee\lib\libc.a(mlock.o)
                0x0000000000176bd8                __malloc_unlock
                0x0000000000176bd0                __malloc_lock
 .text          0x0000000000176be0       0x60 E:/usr/local/sce/ee/gcc/lib/gcc-lib/ee\2.95.2\../../../../ee\lib\libc.a(openr.o)
                0x0000000000176be0                _open_r
 .text          0x0000000000176c40       0x90 E:/usr/local/sce/ee/gcc/lib/gcc-lib/ee\2.95.2\../../../../ee\lib\libc.a(printf.o)
                0x0000000000176c80                printf
                0x0000000000176c40                _printf_r
 .text          0x0000000000176cd0      0xa24 E:/usr/local/sce/ee/gcc/lib/gcc-lib/ee\2.95.2\../../../../ee\lib\libc.a(qsort.o)
                0x0000000000176cd0                qsort
 *fill*         0x00000000001776f4 0x303ec800000004
 .text          0x00000000001776f8       0x2c E:/usr/local/sce/ee/gcc/lib/gcc-lib/ee\2.95.2\../../../../ee\lib\libc.a(realloc.o)
                0x00000000001776f8                realloc
 *fill*         0x0000000000177724 0x303ec800000004
 .text          0x0000000000177728      0x570 E:/usr/local/sce/ee/gcc/lib/gcc-lib/ee\2.95.2\../../../../ee\lib\libc.a(reallocr.o)
                0x0000000000177728                _realloc_r
 .text          0x0000000000177c98      0x198 E:/usr/local/sce/ee/gcc/lib/gcc-lib/ee\2.95.2\../../../../ee\lib\libc.a(refill.o)
                0x0000000000177cb8                __srefill
 .text          0x0000000000177e30       0x5c E:/usr/local/sce/ee/gcc/lib/gcc-lib/ee\2.95.2\../../../../ee\lib\libc.a(sbrkr.o)
                0x0000000000177e30                _sbrk_r
 .text          0x0000000000177e8c       0x7c E:/usr/local/sce/ee/gcc/lib/gcc-lib/ee\2.95.2\../../../../ee\lib\libc.a(setjmp.o)
                0x0000000000177ec4                longjmp
                0x0000000000177e8c                setjmp
 .text          0x0000000000177f08       0xd8 E:/usr/local/sce/ee/gcc/lib/gcc-lib/ee\2.95.2\../../../../ee\lib\libc.a(sprintf.o)
                0x0000000000177f08                _sprintf_r
                0x0000000000177f70                sprintf
 .text          0x0000000000177fe0       0x90 E:/usr/local/sce/ee/gcc/lib/gcc-lib/ee\2.95.2\../../../../ee\lib\libc.a(sscanf.o)
                0x0000000000177fe8                sscanf
 .text          0x0000000000178070      0x170 E:/usr/local/sce/ee/gcc/lib/gcc-lib/ee\2.95.2\../../../../ee\lib\libc.a(stdio.o)
                0x0000000000178158                __sseek
                0x0000000000178070                __sread
                0x00000000001781c0                __sclose
                0x00000000001780d8                __swrite
 .text          0x00000000001781e0      0x12c E:/usr/local/sce/ee/gcc/lib/gcc-lib/ee\2.95.2\../../../../ee\lib\libc.a(strcat.o)
                0x00000000001781e0                strcat
 .text          0x000000000017830c      0x190 E:/usr/local/sce/ee/gcc/lib/gcc-lib/ee\2.95.2\../../../../ee\lib\libc.a(strchr.o)
                0x000000000017830c                strchr
 .text          0x000000000017849c      0x144 E:/usr/local/sce/ee/gcc/lib/gcc-lib/ee\2.95.2\../../../../ee\lib\libc.a(strcmp.o)
                0x000000000017849c                strcmp
 .text          0x00000000001785e0      0x114 E:/usr/local/sce/ee/gcc/lib/gcc-lib/ee\2.95.2\../../../../ee\lib\libc.a(strcpy.o)
                0x00000000001785e0                strcpy
 *fill*         0x00000000001786f4 0x303ec800000004
 .text          0x00000000001786f8       0x28 E:/usr/local/sce/ee/gcc/lib/gcc-lib/ee\2.95.2\../../../../ee\lib\libc.a(strdup.o)
                0x00000000001786f8                strdup
 .text          0x0000000000178720       0x68 E:/usr/local/sce/ee/gcc/lib/gcc-lib/ee\2.95.2\../../../../ee\lib\libc.a(strdup_r.o)
                0x0000000000178720                _strdup_r
 .text          0x0000000000178788      0x138 E:/usr/local/sce/ee/gcc/lib/gcc-lib/ee\2.95.2\../../../../ee\lib\libc.a(strlen.o)
                0x0000000000178788                strlen
 .text          0x00000000001788c0      0x1ac E:/usr/local/sce/ee/gcc/lib/gcc-lib/ee\2.95.2\../../../../ee\lib\libc.a(strncat.o)
                0x00000000001788c0                strncat
 *fill*         0x0000000000178a6c 0x303ec800000004
 .text          0x0000000000178a70      0x1bc E:/usr/local/sce/ee/gcc/lib/gcc-lib/ee\2.95.2\../../../../ee\lib\libc.a(strncpy.o)
                0x0000000000178a70                strncpy
 *fill*         0x0000000000178c2c 0x303ec800000004
 .text          0x0000000000178c30       0x50 E:/usr/local/sce/ee/gcc/lib/gcc-lib/ee\2.95.2\../../../../ee\lib\libc.a(strrchr.o)
                0x0000000000178c30                strrchr
 .text          0x0000000000178c80       0x6c E:/usr/local/sce/ee/gcc/lib/gcc-lib/ee\2.95.2\../../../../ee\lib\libc.a(strstr.o)
                0x0000000000178c80                strstr
 *fill*         0x0000000000178cec 0x303ec800000004
 .text          0x0000000000178cf0      0xf54 E:/usr/local/sce/ee/gcc/lib/gcc-lib/ee\2.95.2\../../../../ee\lib\libc.a(strtod.o)
                0x0000000000178cf0                _strtod_r
                0x0000000000179c20                strtodf
                0x0000000000179bf0                strtod
 *fill*         0x0000000000179c44 0x303ec800000004
 .text          0x0000000000179c48       0x24 E:/usr/local/sce/ee/gcc/lib/gcc-lib/ee\2.95.2\../../../../ee\lib\libc.a(strtok.o)
                0x0000000000179c48                strtok
 *fill*         0x0000000000179c6c 0x303ec800000004
 .text          0x0000000000179c70       0x9c E:/usr/local/sce/ee/gcc/lib/gcc-lib/ee\2.95.2\../../../../ee\lib\libc.a(strtok_r.o)
                0x0000000000179c70                strtok_r
 *fill*         0x0000000000179d0c 0x303ec800000004
 .text          0x0000000000179d10     0x1920 E:/usr/local/sce/ee/gcc/lib/gcc-lib/ee\2.95.2\../../../../ee\lib\libc.a(vfprintf.o)
                0x0000000000179e88                _vfprintf_r
                0x0000000000179e10                vfprintf
 .text          0x000000000017b630      0xc0c E:/usr/local/sce/ee/gcc/lib/gcc-lib/ee\2.95.2\../../../../ee\lib\libc.a(vfscanf.o)
                0x000000000017b630                __svfscanf
                0x000000000017c138                __sccl
 *fill*         0x000000000017c23c 0x303ec800000004
 .text          0x000000000017c240       0x54 E:/usr/local/sce/ee/gcc/lib/gcc-lib/ee\2.95.2\../../../../ee\lib\libc.a(vsprintf.o)
                0x000000000017c240                vsprintf
 *fill*         0x000000000017c294 0x303ec800000004
 .text          0x000000000017c298       0x60 E:/usr/local/sce/ee/gcc/lib/gcc-lib/ee\2.95.2\../../../../ee\lib\libc.a(writer.o)
                0x000000000017c298                _write_r
 .text          0x000000000017c2f8      0x10c E:/usr/local/sce/ee/gcc/lib/gcc-lib/ee\2.95.2\../../../../ee\lib\libc.a(wsetup.o)
                0x000000000017c2f8                __swsetup
 *fill*         0x000000000017c404 0x303ec800000004
 .text          0x000000000017c408       0x1c E:/usr/local/sce/ee/gcc/lib/gcc-lib/ee\2.95.2\../../../../ee\lib\libc.a(atof.o)
                0x000000000017c408                atof
 *fill*         0x000000000017c424 0x303ec800000004
 .text          0x000000000017c428       0x58 E:/usr/local/sce/ee/gcc/lib/gcc-lib/ee\2.95.2\../../../../ee\lib\libc.a(closer.o)
                0x000000000017c428                _close_r
 .text          0x000000000017c480     0x13e4 E:/usr/local/sce/ee/gcc/lib/gcc-lib/ee\2.95.2\../../../../ee\lib\libc.a(dtoa.o)
                0x000000000017c698                _dtoa_r
 *fill*         0x000000000017d864 0x303ec800000004
 .text          0x000000000017d868       0xa8 E:/usr/local/sce/ee/gcc/lib/gcc-lib/ee\2.95.2\../../../../ee\lib\libc.a(flags.o)
                0x000000000017d868                __sflags
 .text          0x000000000017d910       0xec E:/usr/local/sce/ee/gcc/lib/gcc-lib/ee\2.95.2\../../../../ee\lib\libc.a(locale.o)
                0x000000000017d910                _setlocale_r
                0x000000000017d998                _localeconv_r
                0x000000000017d9a8                setlocale
                0x000000000017d9d8                localeconv
 *fill*         0x000000000017d9fc 0x303ec800000004
 .text          0x000000000017da00       0x60 E:/usr/local/sce/ee/gcc/lib/gcc-lib/ee\2.95.2\../../../../ee\lib\libc.a(lseekr.o)
                0x000000000017da00                _lseek_r
 .text          0x000000000017da60       0x3c E:/usr/local/sce/ee/gcc/lib/gcc-lib/ee\2.95.2\../../../../ee\lib\libc.a(mbtowc_r.o)
                0x000000000017da60                _mbtowc_r
 *fill*         0x000000000017da9c 0x303ec800000004
 .text          0x000000000017daa0     0x101c E:/usr/local/sce/ee/gcc/lib/gcc-lib/ee\2.95.2\../../../../ee\lib\libc.a(mprec.o)
                0x000000000017ea50                _mprec_log10
                0x000000000017ddd8                _hi0bits
                0x000000000017daa0                _Balloc
                0x000000000017e810                _d2b
                0x000000000017df58                _multiply
                0x000000000017e990                _ratio
                0x000000000017dc90                _s2b
                0x000000000017df20                _i2b
                0x000000000017de60                _lo0bits
                0x000000000017e400                __mcmp
                0x000000000017e188                _pow5mult
                0x000000000017e5f8                _ulp
                0x000000000017e690                _b2d
                0x000000000017db78                _multadd
                0x000000000017e468                __mdiff
                0x000000000017e288                _lshift
                0x000000000017db48                _Bfree
 *fill*         0x000000000017eabc 0x303ec800000004
 .text          0x000000000017eac0       0x60 E:/usr/local/sce/ee/gcc/lib/gcc-lib/ee\2.95.2\../../../../ee\lib\libc.a(readr.o)
                0x000000000017eac0                _read_r
 .text          0x000000000017eb20       0x48 E:/usr/local/sce/ee/gcc/lib/gcc-lib/ee\2.95.2\../../../../ee\lib\libc.a(s_isinf.o)
                0x000000000017eb20                isinf
 .text          0x000000000017eb68      0x26c E:/usr/local/sce/ee/gcc/lib/gcc-lib/ee\2.95.2\../../../../ee\lib\libc.a(strtol.o)
                0x000000000017eda0                strtol
                0x000000000017eb68                _strtol_r
 *fill*         0x000000000017edd4 0x303ec800000004
 .text          0x000000000017edd8      0x254 E:/usr/local/sce/ee/gcc/lib/gcc-lib/ee\2.95.2\../../../../ee\lib\libc.a(strtoul.o)
                0x000000000017eff8                strtoul
                0x000000000017edd8                _strtoul_r
 *fill*         0x000000000017f02c 0x303ec800000004
 .text          0x000000000017f030      0x278 E:/usr/local/sce/ee/gcc/lib/gcc-lib/ee\2.95.2\../../../../ee\lib\libc.a(ungetc.o)
                0x000000000017f120                ungetc
                0x000000000017f030                __submore
 *fill*         0x000000000017f2a8 0x303ec800000018
 .text          0x000000000017f2c0      0x890 E:/usr/local/sce/ee/lib\libkernl.a(klib.o)
                0x000000000017f420                _EnableIntc
                0x000000000017f3e0                RemoveIntcHandler
                0x000000000017fa10                iGsGetIMR
                0x000000000017f810                RFU083_iSetEventFlag
                0x000000000017f350                RFU009
                0x000000000017f880                RFU090_iReferEventFlagStatus
                0x000000000017f4c0                iSetAlarm
                0x000000000017f750                ReferSemaStatus
                0x000000000017f5f0                iReferThreadStatus
                0x000000000017f800                RFU082_SetEventFlag
                0x000000000017f980                iGetCop0
                0x000000000017faf0                sceSifGetReg
                0x000000000017f7b0                GetGsVParam
                0x000000000017f890                RFU091
                0x000000000017f7f0                RFU081_DeleteEventFlag
                0x000000000017f3f0                AddDmacHandler
                0x000000000017f540                iTerminateThread
                0x000000000017f8e0                EnableDmacHandler
                0x000000000017f6e0                CreateSema
                0x000000000017f760                iReferSemaStatus
                0x000000000017f3a0                SetVCommonHandler
                0x000000000017f900                DisableDmacHandler
                0x000000000017f560                EnableDispatchThread
                0x000000000017f9d0                SetCPUTimer
                0x000000000017f2c0                RFU000_FullReset
                0x000000000017f9c0                SetCPUTimerHandler
                0x000000000017f550                DisableDispatchThread
                0x000000000017f360                AddSbusIntcHandler
                0x000000000017fae0                sceSifSetReg
                0x000000000017fb10                Deci2Call
                0x000000000017f470                ReleaseAlarm
                0x000000000017f9e0                SetOsdConfigParam2
                0x000000000017f4b0                _iDisableDmac
                0x000000000017fab0                isceSifSetDma
                0x000000000017f620                _iWakeupThread
                0x000000000017f770                RFU073
                0x000000000017f790                GetOsdConfigParam
                0x000000000017f460                SetAlarm
                0x000000000017f9b0                sceSifStopDma
                0x000000000017f780                SetOsdConfigParam
                0x000000000017f940                DisableCache
                0x000000000017f7a0                GetGsHParam
                0x000000000017f7e0                RFU080_CreateEventFlag
                0x000000000017f640                iCancelWakeupThread
                0x000000000017f510                ExitThread
                0x000000000017f8b0                iEnableIntcHandler
                0x000000000017f820                RFU084_ClearEventFlag
                0x000000000017faa0                sceSifSetDma
                0x000000000017f5b0                ReleaseWaitThread
                0x000000000017f8c0                DisableIntcHandler
                0x000000000017f580                iChangeThreadPriority
                0x000000000017f7c0                SetGsHParam
                0x000000000017f920                KSeg0
                0x000000000017f430                _DisableIntc
                0x000000000017fa50                SetVSyncFlag
                0x000000000017f870                RFU089_ReferEventFlagStatus
                0x000000000017fa20                GsPutIMR
                0x000000000017fa80                sceSifDmaStat
                0x000000000017f950                GetCop0
                0x000000000017f300                Exit
                0x000000000017fac0                sceSifSetDChain
                0x000000000017fa00                GsGetIMR
                0x000000000017f5c0                iReleaseWaitThread
                0x000000000017f5d0                GetThreadId
                0x000000000017f3b0                SetVInterruptHandler
                0x000000000017f320                LoadExecPS2
                0x000000000017f440                _EnableDmac
                0x000000000017f850                RFU087_PollEvnetFlag
                0x000000000017f6d0                RFU063
                0x000000000017fb00                ExecOSD
                0x000000000017f960                FlushCache
                0x000000000017fb20                PSMode
                0x000000000017f310                RFU005
                0x000000000017f450                _DisableDmac
                0x000000000017f400                AddDmacHandler2
                0x000000000017fb30                MachineType
                0x000000000017f6b0                RFU061
                0x000000000017f670                ResumeThread
                0x000000000017f390                SetVTLBRefillHandler
                0x000000000017f7d0                SetGsVParam
                0x000000000017f710                iSignalSema
                0x000000000017f6c0                EndOfHeap
                0x000000000017f4a0                _iEnableDmac
                0x000000000017f9f0                GetOsdConfigParam2
                0x000000000017fa60                RFU116
                0x000000000017f3c0                AddIntcHandler
                0x000000000017f680                iResumeThread
                0x000000000017f740                iPollSema
                0x000000000017f8a0                EnableIntcHandler
                0x000000000017f340                RFU008
                0x000000000017f5a0                _iRotateThreadReadyQueue
                0x000000000017f5e0                ReferThreadStatus
                0x000000000017f630                CancelWakeupThread
                0x000000000017f570                ChangeThreadPriority
                0x000000000017f2e0                SetGsCrt
                0x000000000017f380                Interrupt2Iop
                0x000000000017fa30                iGsPutIMR
                0x000000000017f330                ExecPS2
                0x000000000017f410                RemoveDmacHandler
                0x000000000017f2d0                ResetEE
                0x000000000017fa90                isceSifDmaStat
                0x000000000017f700                SignalSema
                0x000000000017f830                RFU085_iClearEventFlag
                0x000000000017f9a0                iCpuConfig
                0x000000000017f480                _iEnableIntc
                0x000000000017f730                PollSema
                0x000000000017f6a0                RFU060
                0x000000000017fad0                isceSifSetDChain
                0x000000000017f8f0                iEnableDmacHandler
                0x000000000017f610                WakeupThread
                0x000000000017f530                TerminateThread
                0x000000000017f660                _iSuspendThread
                0x000000000017f930                EnableCache
                0x000000000017f4f0                DeleteThread
                0x000000000017fb40                GetMemorySize
                0x000000000017f720                WaitSema
                0x000000000017f3d0                AddIntcHandler2
                0x000000000017fa70                _print
                0x000000000017f860                RFU088_iPollEvnetFlag
                0x000000000017f590                RotateThreadReadyQueue
                0x000000000017f600                SleepThread
                0x000000000017f990                iFlushCache
                0x000000000017f2f0                RFU003
                0x000000000017f6f0                DeleteSema
                0x000000000017f4e0                CreateThread
                0x000000000017f840                RFU086_WaitEvnetFlag
                0x000000000017f490                _iDisableIntc
                0x000000000017f8d0                iDisableIntcHandler
                0x000000000017f370                RemoveSbusIntcHandler
                0x000000000017f650                SuspendThread
                0x000000000017f690                JoinThread
                0x000000000017fa40                SetPgifHandler
                0x000000000017f970                CpuConfig
                0x000000000017f520                ExitDeleteThread
                0x000000000017f4d0                iReleaseAlarm
                0x000000000017f910                iDisableDmacHandler
                0x000000000017f500                StartThread
 .text          0x000000000017fb50      0x338 E:/usr/local/sce/ee/lib\libkernl.a(glue.o)
                0x000000000017fd28                ioctl
                0x000000000017fb50                sceResetttyinit
                0x000000000017fe08                getpid
                0x000000000017fde8                isatty
                0x000000000017fd30                lseek
                0x000000000017fc00                write
                0x000000000017fdf0                fstat
                0x000000000017fe10                kill
                0x000000000017fc80                read
                0x000000000017fe60                unlink
                0x000000000017fba0                VSync2
                0x000000000017fd38                sbrk
                0x000000000017fb60                VSync
                0x000000000017fe38                stat
                0x000000000017fcf8                open
                0x000000000017fd20                close
 .text          0x000000000017fe88      0x27c E:/usr/local/sce/ee/lib\libkernl.a(cache.o)
                0x000000000017ff30                SyncDCache
                0x0000000000180070                InvalidDCache
                0x000000000017fe88                _sceSDC
                0x00000000001800f0                iInvalidDCache
                0x000000000017ffb0                iSyncDCache
                0x000000000017ffc8                _sceIDC
 *fill*         0x0000000000180104 0x303ec800000004
 .text          0x0000000000180108      0x35c E:/usr/local/sce/ee/lib\libkernl.a(intr.o)
                0x00000000001801d8                DisableDmac
                0x0000000000180108                DisableIntc
                0x00000000001802a8                iEnableIntc
                0x00000000001802c8                iDisableIntc
                0x0000000000180308                iDisableDmac
                0x0000000000180170                EnableIntc
                0x0000000000180390                InitAlarm
                0x00000000001802e8                iEnableDmac
                0x0000000000180240                EnableDmac
 *fill*         0x0000000000180464 0x303ec800000004
 .text          0x0000000000180468      0x51c E:/usr/local/sce/ee/lib\libkernl.a(tty.o)
                0x00000000001808c8                sceTtyInit
                0x00000000001806a8                sceTtyWrite
                0x00000000001807f8                sceTtyRead
 *fill*         0x0000000000180984 0x303ec800000004
 .text          0x0000000000180988      0x978 E:/usr/local/sce/ee/lib\libkernl.a(kprintf.o)
                0x00000000001812a0                scePrintf
                0x0000000000181268                kprintf
                0x0000000000180ca0                _printf
 .text          0x0000000000181300      0xf60 E:/usr/local/sce/ee/lib\libkernl.a(sifrpc.o)
                0x0000000000181d30                sceSifCheckStatRpc
                0x0000000000181ed8                sceSifRemoveRpc
                0x0000000000182000                sceSifGetNextRequest
                0x0000000000181970                sceSifBindRpc
                0x0000000000181300                sceSifInitRpc
                0x0000000000181b40                sceSifCallRpc
                0x0000000000181e08                sceSifRegisterRpc
                0x0000000000181d70                sceSifSetRpcQueue
                0x00000000001814a0                sceSifExitRpc
                0x0000000000182058                sceSifExecRequest
                0x0000000000181718                sceSifGetOtherData
                0x0000000000181f70                sceSifRemoveRpcQueue
                0x0000000000182220                sceSifRpcLoop
 .text          0x0000000000182260     0x3578 E:/usr/local/sce/ee/lib\libkernl.a(filestub.o)
                0x0000000000184458                sceDread
                0x0000000000183cb0                sceRemove
                0x0000000000182a70                sceOpen
                0x0000000000182cf8                sceClose
                0x0000000000184fa8                sceUmount
                0x0000000000182e78                sceLseek
                0x00000000001835e0                sceIoctl
                0x0000000000185200                sceDevctl
                0x0000000000184fc8                sceLseek64
                0x0000000000185430                sceSymlink
                0x0000000000182a38                sceFsReset
                0x0000000000184990                sceRename
                0x0000000000184ba0                sceSync
                0x0000000000183e80                sceRmdir
                0x0000000000185610                sceReadlink
                0x0000000000184250                sceDopen
                0x00000000001842f0                sceDclose
                0x0000000000183930                sceIoctl2
                0x0000000000182808                sceFsInit
                0x0000000000184230                sceDelDrv
                0x0000000000183320                sceWrite
                0x00000000001845b0                sceGetstat
                0x00000000001830b0                sceRead
                0x0000000000184750                sceChstat
                0x0000000000183ea0                sceFormat
                0x0000000000184b80                sceChdir
                0x0000000000184d38                sceMount
                0x0000000000183cd0                sceMkdir
                0x0000000000184110                sceAddDrv
 .text          0x00000000001857d8      0x300 E:/usr/local/sce/ee/lib\libkernl.a(iopheap.o)
                0x0000000000185950                sceSifFreeSysMemory
                0x00000000001859c8                sceSifFreeIopHeap
                0x00000000001857d8                sceSifInitIopHeap
                0x00000000001858d0                sceSifAllocSysMemory
                0x00000000001859e8                sceSifLoadIopHeap
                0x0000000000185860                sceSifAllocIopHeap
 .text          0x0000000000185ad8      0xd5c E:/usr/local/sce/ee/lib\libkernl.a(eeloadfile.o)
                0x00000000001861e0                sceSifSearchModuleByAddress
                0x00000000001860b0                sceSifUnloadModule
                0x0000000000186758                sceSifSetIopAddr
                0x0000000000185ea8                sceSifStopModule
                0x0000000000186668                sceSifGetIopAddr
                0x0000000000186140                sceSifSearchModuleByName
                0x0000000000186640                sceSifLoadElf
                0x0000000000186290                sceSifLoadStartModuleBuffer
                0x00000000001864f8                sceSifLoadStartModule
                0x00000000001864d8                sceSifLoadModule
                0x0000000000186270                sceSifLoadModuleBuffer
                0x0000000000186620                sceSifLoadElfPart
                0x0000000000185c68                sceSifLoadFileReset
 *fill*         0x0000000000186834 0x303ec800000004
 .text          0x0000000000186838       0x60 E:/usr/local/sce/ee/lib\libkernl.a(diei.o)
                0x0000000000186838                DIntr
                0x0000000000186880                EIntr
 .text          0x0000000000186898       0x6c E:/usr/local/sce/ee/lib\libkernl.a(initsys.o)
                0x00000000001868e0                _InitSys
 *fill*         0x0000000000186904 0x303ec800000004
 .text          0x0000000000186908      0x360 E:/usr/local/sce/ee/lib\libkernl.a(thread.o)
                0x0000000000186b50                iRotateThreadReadyQueue
                0x0000000000186ab8                iWakeupThread
                0x0000000000186bd0                iSuspendThread
                0x00000000001869e0                InitThread
 .text          0x0000000000186c68      0x1dc E:/usr/local/sce/ee/lib\libkernl.a(deci2.o)
                0x0000000000186d08                sceDeci2Poll
                0x0000000000186c68                sceDeci2Open
                0x0000000000186cd8                sceDeci2ReqSend
                0x0000000000186da0                sceDeci2ExReqSend
                0x0000000000186cb0                sceDeci2Close
                0x0000000000186dd0                sceDeci2ExLock
                0x0000000000186e20                kputs
                0x0000000000186d68                sceDeci2ExSend
                0x0000000000186df8                sceDeci2ExUnLock
                0x0000000000186d30                sceDeci2ExRecv
 *fill*         0x0000000000186e44 0x303ec800000004
 .text          0x0000000000186e48      0x748 E:/usr/local/sce/ee/lib\libkernl.a(sifcmd.o)
                0x00000000001871a8                sceSifAddCmdHandler
                0x0000000000187178                sceSifSetCmdBuffer
                0x0000000000187378                isceSifSendCmd
                0x0000000000186e78                sceSifGetSreg
                0x0000000000187140                sceSifExitCmd
                0x0000000000187338                sceSifSendCmd
                0x0000000000187190                sceSifSetSysCmdBuffer
                0x0000000000186eb0                sceSifGetDataTable
                0x00000000001874e0                sceSifWriteBackDCache
                0x0000000000186ec0                sceSifInitCmd
                0x00000000001871d8                sceSifRemoveCmdHandler
                0x0000000000186e90                sceSifSetSreg
 .text          0x0000000000187590      0x6ec E:/usr/local/sce/ee/gcc/lib/gcc-lib/ee\2.95.2\libgcc.a(_divdi3.o)
                0x0000000000187590                __divdi3
 *fill*         0x0000000000187c7c 0x303ec800000004
 .text          0x0000000000187c80      0x668 E:/usr/local/sce/ee/gcc/lib/gcc-lib/ee\2.95.2\libgcc.a(_moddi3.o)
                0x0000000000187c80                __moddi3
                0x00000000001882e8        0x8 QUAD 0x0

.vutext         0x00000000001882f0     0x6150
 .vutext        0x00000000001882f0     0x2ca0 E:/nightly/rwsdk.sky/rwsdk/lib/sky2/librwcore.a(GenericPRS.obj)
                0x00000000001882f0                vu1GenericPRS
 .vutext        0x000000000018af90     0x1550 E:/nightly/rwsdk.sky/rwsdk/lib/sky2/librwcore.a(SegmentsPRL.obj)
                0x000000000018af90                vu1SegmentsPRL
 .vutext        0x000000000018c4e0     0x1800 E:/nightly/rwsdk.sky/rwsdk/lib/sky2/librwcore.a(SegmentsPRS.obj)
                0x000000000018c4e0                vu1SegmentsPRS
 .vutext        0x000000000018dce0      0x200 E:/nightly/rwsdk.sky/rwsdk/lib/sky2/librwcore.a(baim2dll.obj)
                0x000000000018dce0                vu1im2dll
 .vutext        0x000000000018dee0      0x270 E:/nightly/rwsdk.sky/rwsdk/lib/sky2/librwcore.a(baim2dtl.obj)
                0x000000000018dee0                vu1im2dtl
 .vutext        0x000000000018e150      0x160 E:/nightly/rwsdk.sky/rwsdk/lib/sky2/librwcore.a(banfim2dll.obj)
                0x000000000018e150                vu1nfim2dll
 .vutext        0x000000000018e2b0      0x190 E:/nightly/rwsdk.sky/rwsdk/lib/sky2/librwcore.a(banfim2dtl.obj)
                0x000000000018e2b0                vu1nfim2dtl

.reginfo        0x000000000018e440       0x18
 *(.reginfo)
 .reginfo       0x000000000018e440       0x18 crt0.o

.data           0x000000000018e480    0x13428
 *(.data)
 .data          0x000000000018e480       0x58 obj/sky2/main.o
 .data          0x000000000018e4d8      0x458 obj/sky2/linelist.o
 .data          0x000000000018e930      0x27a obj/sky2/polyline.o
 *fill*         0x000000000018ebaa 0x3038c000000006
 .data          0x000000000018ebb0      0x3b8 obj/sky2/trilist.o
 .data          0x000000000018ef68      0x458 obj/sky2/tristrip.o
 .data          0x000000000018f3c0      0x444 obj/sky2/trifan.o
 *fill*         0x000000000018f804 0x3038c000000004
 .data          0x000000000018f808      0x410 obj/sky2/camera.o
 .data          0x000000000018fc18     0x17f0 obj/sky2/menu.o
                0x000000000018fc98                helpLines
 .data          0x0000000000191408      0x27c obj/sky2/skeleton.o
                0x0000000000191648                RsGlobal
 *fill*         0x0000000000191684 0x3038c000000004
 .data          0x0000000000191688     0x8000 E:/nightly/rwsdk.sky/rwsdk/lib/sky2/librplogo.a(rplogo.obj)
 .data          0x0000000000199688       0x14 E:/nightly/rwsdk.sky/rwsdk/lib/sky2/librtcharse.a(chrprint.obj)
                0x0000000000199688                _rtgBuffer
 *fill*         0x000000000019969c 0x3038c000000004
 .data          0x00000000001996a0       0x20 E:/nightly/rwsdk.sky/rwsdk/lib/sky2/librtpng.a(pngrtran.obj)
 .data          0x00000000001996c0       0x1f E:/nightly/rwsdk.sky/rwsdk/lib/sky2/librtpng.a(pngrutil.obj)
 *fill*         0x00000000001996df 0x3038c000000001
 .data          0x00000000001996e0      0x300 E:/nightly/rwsdk.sky/rwsdk/lib/sky2/librtpng.a(pngtrans.obj)
 .data          0x00000000001999e0       0x44 E:/nightly/rwsdk.sky/rwsdk/lib/sky2/librtpng.a(trees.obj)
 *fill*         0x0000000000199a24 0x3038c000000004
 .data          0x0000000000199a28       0x28 E:/nightly/rwsdk.sky/rwsdk/lib/sky2/librtpng.a(zutil.obj)
                0x0000000000199a28                z_errmsg
 .data          0x0000000000199a50     0x1100 E:/nightly/rwsdk.sky/rwsdk/lib/sky2/librtpng.a(inftrees.obj)
 .data          0x000000000019ab50       0x44 E:/nightly/rwsdk.sky/rwsdk/lib/sky2/librtpng.a(infutil.obj)
                0x000000000019ab50                inflate_mask
 *fill*         0x000000000019ab94 0x3038c000000004
 .data          0x000000000019ab98       0x18 E:/nightly/rwsdk.sky/rwsdk/lib/sky2/librwcore.a(bacamera.obj)
                0x000000000019ab98                cameraTKList
 .data          0x000000000019abb0     0x4118 E:/nightly/rwsdk.sky/rwsdk/lib/sky2/librwcore.a(badevice.obj)
                0x000000000019abc8                _rwMsbBit
                0x000000000019acc8                ourGlobals
 .data          0x000000000019ecc8       0x18 E:/nightly/rwsdk.sky/rwsdk/lib/sky2/librwcore.a(baframe.obj)
                0x000000000019ecc8                frameTKList
 .data          0x000000000019ece0       0x18 E:/nightly/rwsdk.sky/rwsdk/lib/sky2/librwcore.a(baimage.obj)
 .data          0x000000000019ecf8       0x18 E:/nightly/rwsdk.sky/rwsdk/lib/sky2/librwcore.a(baraster.obj)
 .data          0x000000000019ed10       0x30 E:/nightly/rwsdk.sky/rwsdk/lib/sky2/librwcore.a(batextur.obj)
                0x000000000019ed28                texDictTKList
                0x000000000019ed10                textureTKList
 .data          0x000000000019ed40      0x100 E:/nightly/rwsdk.sky/rwsdk/lib/sky2/librwcore.a(nodeClipLine.obj)
 .data          0x000000000019ee40      0x110 E:/nightly/rwsdk.sky/rwsdk/lib/sky2/librwcore.a(nodeClipTriangle.obj)
 .data          0x000000000019ef50       0xf8 E:/nightly/rwsdk.sky/rwsdk/lib/sky2/librwcore.a(nodeCullTriangle.obj)
 .data          0x000000000019f048       0xb8 E:/nightly/rwsdk.sky/rwsdk/lib/sky2/librwcore.a(nodeImmInstance.obj)
 .data          0x000000000019f100       0xc8 E:/nightly/rwsdk.sky/rwsdk/lib/sky2/librwcore.a(nodeImmMangleLineIndices.obj)
 .data          0x000000000019f1c8       0xc8 E:/nightly/rwsdk.sky/rwsdk/lib/sky2/librwcore.a(nodeImmMangleTriangleIndices.obj)
 .data          0x000000000019f290      0x138 E:/nightly/rwsdk.sky/rwsdk/lib/sky2/librwcore.a(nodeImmRenderSetup.obj)
 .data          0x000000000019f3c8       0xa8 E:/nightly/rwsdk.sky/rwsdk/lib/sky2/librwcore.a(nodeImmStash.obj)
 .data          0x000000000019f470       0xc0 E:/nightly/rwsdk.sky/rwsdk/lib/sky2/librwcore.a(nodeSubmitLine.obj)
 .data          0x000000000019f530       0xc8 E:/nightly/rwsdk.sky/rwsdk/lib/sky2/librwcore.a(nodeSubmitTriangle.obj)
 .data          0x000000000019f5f8       0xe8 E:/nightly/rwsdk.sky/rwsdk/lib/sky2/librwcore.a(nodeTransform.obj)
 .data          0x000000000019f6e0       0x18 E:/nightly/rwsdk.sky/rwsdk/lib/sky2/librwcore.a(p2altmdl.obj)
                0x000000000019f6e0                _rxExecCtxGlobal
 .data          0x000000000019f6f8       0x28 E:/nightly/rwsdk.sky/rwsdk/lib/sky2/librwcore.a(p2clpcom.obj)
                0x000000000019f6f8                _rwClipInfoGlobal
 .data          0x000000000019f720      0x1d8 E:/nightly/rwsdk.sky/rwsdk/lib/sky2/librwcore.a(p2stdcls.obj)
                0x000000000019f828                RxClIndices
                0x000000000019f7a0                RxClScrSpace2DVertices
                0x000000000019f8c8                RxClRGBAs
                0x000000000019f770                RxClCamSpace3DVertices
                0x000000000019f8e8                RxClCamNorms
                0x000000000019f7c8                RxClInterpolants
                0x000000000019f8a8                RxClVSteps
                0x000000000019f7e8                RxClMeshState
                0x000000000019f740                RxClObjSpace3DVertices
                0x000000000019f868                RxClTriPlanes
                0x000000000019f808                RxClRenderState
                0x000000000019f888                RxClUVs
                0x000000000019f848                RxClScatter
 *fill*         0x000000000019f8f8 0x3038c000000008
 .data          0x000000000019f900      0xa7c E:/nightly/rwsdk.sky/rwsdk/lib/sky2/librwcore.a(basky.obj)
                0x00000000001a0370                skyFakeCacheFrameBuffer1
                0x00000000001a0030                sweDb
                0x00000000001a0360                skyFakeCacheFrameBuffer0
 *fill*         0x00000000001a037c 0x3038c000000004
 .data          0x00000000001a0380      0x210 E:/nightly/rwsdk.sky/rwsdk/lib/sky2/librwcore.a(skyinst.obj)
                0x00000000001a0460                skyClipVect1
                0x00000000001a0420                runCmd128
                0x00000000001a0480                skyCClipVect1
                0x00000000001a03e0                gifTagPrim128
                0x00000000001a03d0                gifTag128
                0x00000000001a0390                dma10Header128
                0x00000000001a03b0                dma1Header128
                0x00000000001a0470                skyClipVect2
                0x00000000001a0400                nullLightBlock
                0x00000000001a0440                unmaskCmd128
                0x00000000001a0450                zero128
                0x00000000001a03a0                dma1End128
                0x00000000001a0430                surfLightCoeffs
                0x00000000001a0490                skyCClipVect2
                0x00000000001a0380                contCmd128
                0x00000000001a03c0                dma1Ret128
                0x00000000001a03f0                maskCmd128
 *fill*         0x00000000001a0590 0x3038c000000030
 .data          0x00000000001a05c0       0x40 E:/nightly/rwsdk.sky/rwsdk/lib/sky2/librwcore.a(texcache.obj)
 .data          0x00000000001a0600       0x80 E:/nightly/rwsdk.sky/rwsdk/lib/sky2/librwcore.a(imrascnv.obj)
 .data          0x00000000001a0680      0x100 E:/nightly/rwsdk.sky/rwsdk/lib/sky2/librwcore.a(badma.obj)
                0x00000000001a06c0                tcaaDisp
                0x00000000001a0680                _RwSavedGP
 .data          0x00000000001a0780       0x20 E:/usr/local/sce/ee/lib/libgraph.a(graph001.o)
 .data          0x00000000001a07a0       0x20 E:/usr/local/sce/ee/lib/libgraph.a(graph002.o)
 .data          0x00000000001a07c0       0x10 E:/usr/local/sce/ee/lib/libgraph.a(graph018.o)
 .data          0x00000000001a07d0       0xac E:/usr/local/sce/ee/lib/libdma.a(libdma.o)
                0x00000000001a0868                sceDmaCurrentEnv
                0x00000000001a07d0                dch
                0x00000000001a07f8                sceDmaDebugMode
 *fill*         0x00000000001a087c 0x3038c000000004
 .data          0x00000000001a0880       0x44 E:/usr/local/sce/ee/lib/libpad.a(libpad.o)
 .data          0x00000000001a08c4        0x4 E:/usr/local/sce/ee/gcc/lib/gcc-lib/ee\2.95.2\libgcc.a(__main.o)
 .data          0x00000000001a08c8      0x2f0 E:/usr/local/sce/ee/gcc/lib/gcc-lib/ee\2.95.2\../../../../ee\lib\libc.a(impure.o)
                0x00000000001a0bb4                _impure_ptr
 .data          0x00000000001a0bb8      0x458 E:/usr/local/sce/ee/gcc/lib/gcc-lib/ee\2.95.2\../../../../ee\lib\libc.a(mallocr.o)
                0x00000000001a0fc8                __malloc_top_pad
                0x00000000001a0fd8                __malloc_max_sbrked_mem
                0x00000000001a0fd0                __malloc_sbrk_base
                0x00000000001a0fe8                __malloc_current_mallinfo
                0x00000000001a0bb8                __malloc_av_
                0x00000000001a0fe0                __malloc_max_total_mem
                0x00000000001a0fc0                __malloc_trim_threshold
 .data          0x00000000001a1010       0x18 E:/usr/local/sce/ee/gcc/lib/gcc-lib/ee\2.95.2\../../../../ee\lib\libc.a(locale.o)
                0x00000000001a1010                __mb_cur_max
 .data          0x00000000001a1028       0x10 E:/usr/local/sce/ee/lib\libkernl.a(klib.o)
                0x00000000001a1028                __ps2_klibinfo__
 .data          0x00000000001a1038        0x8 E:/usr/local/sce/ee/lib\libkernl.a(glue.o)
 .data          0x00000000001a1040      0x7a8 E:/usr/local/sce/ee/lib\libkernl.a(intr.o)
 .data          0x00000000001a17e8        0x8 E:/usr/local/sce/ee/lib\libkernl.a(kprintf.o)
 .data          0x00000000001a17f0        0x4 E:/usr/local/sce/ee/lib\libkernl.a(sifrpc.o)
 *fill*         0x00000000001a17f4 0x3038c000000004
 .data          0x00000000001a17f8       0x94 E:/usr/local/sce/ee/lib\libkernl.a(filestub.o)
                0x00000000001a17f8                _sceFs_q
 .data          0x00000000001a188c        0x4 E:/usr/local/sce/ee/lib\libkernl.a(iopheap.o)
 .data          0x00000000001a1890        0x8 E:/usr/local/sce/ee/lib\libkernl.a(eeloadfile.o)
 .data          0x00000000001a1898        0x8 E:/usr/local/sce/ee/lib\libkernl.a(initsys.o)
                0x00000000001a1898                __sce_sema_id
                0x00000000001a189c                __sce_eh_sema_id
 .data          0x00000000001a18a0        0x4 E:/usr/local/sce/ee/lib\libkernl.a(thread.o)
 .data          0x00000000001a18a4        0x4 E:/usr/local/sce/ee/lib\libkernl.a(sifcmd.o)

.vudata         0x00000000001a18b0       0xc0
 .vudata        0x00000000001a18b0       0xc0 E:/nightly/rwsdk.sky/rwsdk/lib/sky2/librwcore.a(baasm.obj)
                0x00000000001a18b0                gs_set_up
                0x00000000001a1930                screen_refresh

.rodata         0x00000000001a1980     0x8a48
 *(.rodata)
 .rodata        0x00000000001a1980      0x27c obj/sky2/main.o
 *fill*         0x00000000001a1bfc 0x30395800000004
 .rodata        0x00000000001a1c00       0x41 obj/sky2/im3d.o
 *fill*         0x00000000001a1c41 0x3039580000000f
 .rodata        0x00000000001a1c50       0x64 obj/sky2/menu.o
 *fill*         0x00000000001a1cb4 0x3039580000000c
 .rodata        0x00000000001a1cc0      0x15d obj/sky2/skeleton.o
 *fill*         0x00000000001a1e1d 0x30395800000003
 .rodata        0x00000000001a1e20      0x1ec obj/sky2/sky.o
 *fill*         0x00000000001a200c 0x30395800000004
 .rodata        0x00000000001a2010       0x60 E:/nightly/rwsdk.sky/rwsdk/lib/sky2/librplogo.a(rplogo.obj)
 .rodata        0x00000000001a2070       0x3d E:/nightly/rwsdk.sky/rwsdk/lib/sky2/librtcharse.a(chrprint.obj)
 *fill*         0x00000000001a20ad 0x30395800000003
 .rodata        0x00000000001a20b0      0x53a E:/nightly/rwsdk.sky/rwsdk/lib/sky2/librtcharse.a(rtcharse.obj)
 *fill*         0x00000000001a25ea 0x30395800000006
 .rodata        0x00000000001a25f0       0x5c E:/nightly/rwsdk.sky/rwsdk/lib/sky2/librtpng.a(rtpng.obj)
 *fill*         0x00000000001a264c 0x30395800000004
 .rodata        0x00000000001a2650      0x228 E:/nightly/rwsdk.sky/rwsdk/lib/sky2/librtpng.a(png.obj)
                0x00000000001a26a8                png_pass_ystart
                0x00000000001a2668                png_pass_start
                0x00000000001a2708                png_pass_dsp_mask
                0x00000000001a26e8                png_pass_mask
                0x00000000001a2688                png_pass_inc
                0x00000000001a26c8                png_pass_yinc
                0x00000000001a2650                png_libpng_ver
 .rodata        0x00000000001a2878       0x10 E:/nightly/rwsdk.sky/rwsdk/lib/sky2/librtpng.a(pngerror.obj)
 .rodata        0x00000000001a2888       0x32 E:/nightly/rwsdk.sky/rwsdk/lib/sky2/librtpng.a(pngget.obj)
 *fill*         0x00000000001a28ba 0x30395800000006
 .rodata        0x00000000001a28c0       0x5e E:/nightly/rwsdk.sky/rwsdk/lib/sky2/librtpng.a(pngmem.obj)
 *fill*         0x00000000001a291e 0x30395800000002
 .rodata        0x00000000001a2920      0x346 E:/nightly/rwsdk.sky/rwsdk/lib/sky2/librtpng.a(pngread.obj)
 *fill*         0x00000000001a2c66 0x30395800000002
 .rodata        0x00000000001a2c68       0x9a E:/nightly/rwsdk.sky/rwsdk/lib/sky2/librtpng.a(pngrio.obj)
 *fill*         0x00000000001a2d02 0x3039580000000e
 .rodata        0x00000000001a2d10      0x278 E:/nightly/rwsdk.sky/rwsdk/lib/sky2/librtpng.a(pngrtran.obj)
 *fill*         0x00000000001a2f88 0x30395800000008
 .rodata        0x00000000001a2f90      0xcf0 E:/nightly/rwsdk.sky/rwsdk/lib/sky2/librtpng.a(pngrutil.obj)
 .rodata        0x00000000001a3c80      0x240 E:/nightly/rwsdk.sky/rwsdk/lib/sky2/librtpng.a(pngset.obj)
 .rodata        0x00000000001a3ec0       0x8d E:/nightly/rwsdk.sky/rwsdk/lib/sky2/librtpng.a(pngwio.obj)
 *fill*         0x00000000001a3f4d 0x30395800000003
 .rodata        0x00000000001a3f50      0x3ee E:/nightly/rwsdk.sky/rwsdk/lib/sky2/librtpng.a(pngwrite.obj)
 *fill*         0x00000000001a433e 0x30395800000002
 .rodata        0x00000000001a4340      0x6d8 E:/nightly/rwsdk.sky/rwsdk/lib/sky2/librtpng.a(pngwutil.obj)
 .rodata        0x00000000001a4a18       0xb0 E:/nightly/rwsdk.sky/rwsdk/lib/sky2/librtpng.a(deflate.obj)
                0x00000000001a4a18                deflate_copyright
 .rodata        0x00000000001a4ac8      0xa40 E:/nightly/rwsdk.sky/rwsdk/lib/sky2/librtpng.a(trees.obj)
                0x00000000001a5318                _length_code
                0x00000000001a5118                _dist_code
 .rodata        0x00000000001a5508       0x90 E:/nightly/rwsdk.sky/rwsdk/lib/sky2/librtpng.a(zutil.obj)
 *fill*         0x00000000001a5598 0x30395800000008
 .rodata        0x00000000001a55a0       0xb8 E:/nightly/rwsdk.sky/rwsdk/lib/sky2/librtpng.a(inflate.obj)
 *fill*         0x00000000001a5658 0x30395800000008
 .rodata        0x00000000001a5660       0xf8 E:/nightly/rwsdk.sky/rwsdk/lib/sky2/librtpng.a(infblock.obj)
 .rodata        0x00000000001a5758      0x319 E:/nightly/rwsdk.sky/rwsdk/lib/sky2/librtpng.a(inftrees.obj)
                0x00000000001a5758                inflate_copyright
 *fill*         0x00000000001a5a71 0x3039580000000f
 .rodata        0x00000000001a5a80       0x68 E:/nightly/rwsdk.sky/rwsdk/lib/sky2/librtpng.a(infcodes.obj)
 .rodata        0x00000000001a5ae8       0x34 E:/nightly/rwsdk.sky/rwsdk/lib/sky2/librtpng.a(inffast.obj)
 *fill*         0x00000000001a5b1c 0x30395800000004
 .rodata        0x00000000001a5b20      0x800 E:/nightly/rwsdk.sky/rwsdk/lib/sky2/librtpng.a(crc32.obj)
 .rodata        0x00000000001a6320       0xc0 E:/nightly/rwsdk.sky/rwsdk/lib/sky2/librtbmp.a(rtbmp.obj)
 .rodata        0x00000000001a63e0       0xa8 E:/nightly/rwsdk.sky/rwsdk/lib/sky2/librwcore.a(babinary.obj)
 .rodata        0x00000000001a6488       0x62 E:/nightly/rwsdk.sky/rwsdk/lib/sky2/librwcore.a(bacamera.obj)
 *fill*         0x00000000001a64ea 0x30395800000006
 .rodata        0x00000000001a64f0       0xa8 E:/nightly/rwsdk.sky/rwsdk/lib/sky2/librwcore.a(badevice.obj)
 .rodata        0x00000000001a6598       0x3e E:/nightly/rwsdk.sky/rwsdk/lib/sky2/librwcore.a(baerr.obj)
 *fill*         0x00000000001a65d6 0x30395800000002
 .rodata        0x00000000001a65d8       0x3c E:/nightly/rwsdk.sky/rwsdk/lib/sky2/librwcore.a(baframe.obj)
 *fill*         0x00000000001a6614 0x30395800000004
 .rodata        0x00000000001a6618       0x3a E:/nightly/rwsdk.sky/rwsdk/lib/sky2/librwcore.a(bafsys.obj)
 *fill*         0x00000000001a6652 0x30395800000006
 .rodata        0x00000000001a6658       0x43 E:/nightly/rwsdk.sky/rwsdk/lib/sky2/librwcore.a(baimage.obj)
 *fill*         0x00000000001a669b 0x30395800000005
 .rodata        0x00000000001a66a0       0x3f E:/nightly/rwsdk.sky/rwsdk/lib/sky2/librwcore.a(baimmedi.obj)
 *fill*         0x00000000001a66df 0x30395800000001
 .rodata        0x00000000001a66e0       0x3b E:/nightly/rwsdk.sky/rwsdk/lib/sky2/librwcore.a(baimras.obj)
 *fill*         0x00000000001a671b 0x30395800000005
 .rodata        0x00000000001a6720       0x59 E:/nightly/rwsdk.sky/rwsdk/lib/sky2/librwcore.a(bamatrix.obj)
 *fill*         0x00000000001a6779 0x30395800000007
 .rodata        0x00000000001a6780       0x3d E:/nightly/rwsdk.sky/rwsdk/lib/sky2/librwcore.a(bamemory.obj)
 *fill*         0x00000000001a67bd 0x30395800000003
 .rodata        0x00000000001a67c0       0x3f E:/nightly/rwsdk.sky/rwsdk/lib/sky2/librwcore.a(baraster.obj)
 *fill*         0x00000000001a67ff 0x30395800000001
 .rodata        0x00000000001a6800       0x3c E:/nightly/rwsdk.sky/rwsdk/lib/sky2/librwcore.a(baresamp.obj)
 *fill*         0x00000000001a683c 0x30395800000004
 .rodata        0x00000000001a6840       0x41 E:/nightly/rwsdk.sky/rwsdk/lib/sky2/librwcore.a(baresour.obj)
 *fill*         0x00000000001a6881 0x30395800000007
 .rodata        0x00000000001a6888       0x3c E:/nightly/rwsdk.sky/rwsdk/lib/sky2/librwcore.a(bastream.obj)
 *fill*         0x00000000001a68c4 0x30395800000004
 .rodata        0x00000000001a68c8       0x38 E:/nightly/rwsdk.sky/rwsdk/lib/sky2/librwcore.a(basync.obj)
 .rodata        0x00000000001a6900       0x51 E:/nightly/rwsdk.sky/rwsdk/lib/sky2/librwcore.a(batextur.obj)
 *fill*         0x00000000001a6951 0x30395800000007
 .rodata        0x00000000001a6958       0x3b E:/nightly/rwsdk.sky/rwsdk/lib/sky2/librwcore.a(batkreg.obj)
 *fill*         0x00000000001a6993 0x30395800000005
 .rodata        0x00000000001a6998       0x41 E:/nightly/rwsdk.sky/rwsdk/lib/sky2/librwcore.a(batypehf.obj)
 *fill*         0x00000000001a69d9 0x30395800000007
 .rodata        0x00000000001a69e0       0x42 E:/nightly/rwsdk.sky/rwsdk/lib/sky2/librwcore.a(bavector.obj)
 *fill*         0x00000000001a6a22 0x30395800000006
 .rodata        0x00000000001a6a28       0x3b E:/nightly/rwsdk.sky/rwsdk/lib/sky2/librwcore.a(resmem.obj)
 *fill*         0x00000000001a6a63 0x30395800000005
 .rodata        0x00000000001a6a68       0x3c E:/nightly/rwsdk.sky/rwsdk/lib/sky2/librwcore.a(rwstring.obj)
 *fill*         0x00000000001a6aa4 0x3039580000000c
 .rodata        0x00000000001a6ab0      0x1b8 E:/nightly/rwsdk.sky/rwsdk/lib/sky2/librwcore.a(baim3d.obj)
 .rodata        0x00000000001a6c68       0x3c E:/nightly/rwsdk.sky/rwsdk/lib/sky2/librwcore.a(bapipe.obj)
 *fill*         0x00000000001a6ca4 0x30395800000004
 .rodata        0x00000000001a6ca8       0x78 E:/nightly/rwsdk.sky/rwsdk/lib/sky2/librwcore.a(nodeClipLine.obj)
 .rodata        0x00000000001a6d20       0x78 E:/nightly/rwsdk.sky/rwsdk/lib/sky2/librwcore.a(nodeClipTriangle.obj)
 .rodata        0x00000000001a6d98       0x43 E:/nightly/rwsdk.sky/rwsdk/lib/sky2/librwcore.a(nodeCullTriangle.obj)
 *fill*         0x00000000001a6ddb 0x30395800000005
 .rodata        0x00000000001a6de0       0x42 E:/nightly/rwsdk.sky/rwsdk/lib/sky2/librwcore.a(nodeImmInstance.obj)
 *fill*         0x00000000001a6e22 0x30395800000006
 .rodata        0x00000000001a6e28       0x4b E:/nightly/rwsdk.sky/rwsdk/lib/sky2/librwcore.a(nodeImmMangleLineIndices.obj)
 *fill*         0x00000000001a6e73 0x30395800000005
 .rodata        0x00000000001a6e78       0x50 E:/nightly/rwsdk.sky/rwsdk/lib/sky2/librwcore.a(nodeImmMangleTriangleIndices.obj)
 *fill*         0x00000000001a6ec8 0x30395800000008
 .rodata        0x00000000001a6ed0       0x68 E:/nightly/rwsdk.sky/rwsdk/lib/sky2/librwcore.a(nodeImmRenderSetup.obj)
 .rodata        0x00000000001a6f38       0x42 E:/nightly/rwsdk.sky/rwsdk/lib/sky2/librwcore.a(nodeImmStash.obj)
 *fill*         0x00000000001a6f7a 0x30395800000006
 .rodata        0x00000000001a6f80       0x41 E:/nightly/rwsdk.sky/rwsdk/lib/sky2/librwcore.a(nodeSubmitLine.obj)
 *fill*         0x00000000001a6fc1 0x30395800000007
 .rodata        0x00000000001a6fc8       0x49 E:/nightly/rwsdk.sky/rwsdk/lib/sky2/librwcore.a(nodeSubmitTriangle.obj)
 *fill*         0x00000000001a7011 0x30395800000007
 .rodata        0x00000000001a7018       0x43 E:/nightly/rwsdk.sky/rwsdk/lib/sky2/librwcore.a(nodeTransform.obj)
 *fill*         0x00000000001a705b 0x30395800000005
 .rodata        0x00000000001a7060       0x3e E:/nightly/rwsdk.sky/rwsdk/lib/sky2/librwcore.a(p2clpcom.obj)
 *fill*         0x00000000001a709e 0x30395800000002
 .rodata        0x00000000001a70a0       0x3d E:/nightly/rwsdk.sky/rwsdk/lib/sky2/librwcore.a(p2core.obj)
 *fill*         0x00000000001a70dd 0x30395800000003
 .rodata        0x00000000001a70e0       0x39 E:/nightly/rwsdk.sky/rwsdk/lib/sky2/librwcore.a(p2dep.obj)
 *fill*         0x00000000001a7119 0x30395800000007
 .rodata        0x00000000001a7120       0x61 E:/nightly/rwsdk.sky/rwsdk/lib/sky2/librwcore.a(p2heap.obj)
 *fill*         0x00000000001a7181 0x30395800000007
 .rodata        0x00000000001a7188       0x41 E:/nightly/rwsdk.sky/rwsdk/lib/sky2/librwcore.a(p2renderstate.obj)
 *fill*         0x00000000001a71c9 0x30395800000007
 .rodata        0x00000000001a71d0       0x3c E:/nightly/rwsdk.sky/rwsdk/lib/sky2/librwcore.a(p2resort.obj)
 *fill*         0x00000000001a720c 0x30395800000004
 .rodata        0x00000000001a7210       0x3c E:/nightly/rwsdk.sky/rwsdk/lib/sky2/librwcore.a(p2stdcls.obj)
 *fill*         0x00000000001a724c 0x30395800000004
 .rodata        0x00000000001a7250       0x3e E:/nightly/rwsdk.sky/rwsdk/lib/sky2/librwcore.a(im3dpipe.obj)
 *fill*         0x00000000001a728e 0x30395800000002
 .rodata        0x00000000001a7290      0x974 E:/nightly/rwsdk.sky/rwsdk/lib/sky2/librwcore.a(basky.obj)
 *fill*         0x00000000001a7c04 0x30395800000004
 .rodata        0x00000000001a7c08       0x3c E:/nightly/rwsdk.sky/rwsdk/lib/sky2/librwcore.a(baskytran.obj)
 *fill*         0x00000000001a7c44 0x3039580000000c
 .rodata        0x00000000001a7c50      0x154 E:/nightly/rwsdk.sky/rwsdk/lib/sky2/librwcore.a(skyblit.obj)
 *fill*         0x00000000001a7da4 0x3039580000000c
 .rodata        0x00000000001a7db0      0x228 E:/nightly/rwsdk.sky/rwsdk/lib/sky2/librwcore.a(skyconv.obj)
 .rodata        0x00000000001a7fd8       0x7c E:/nightly/rwsdk.sky/rwsdk/lib/sky2/librwcore.a(skyinst.obj)
 *fill*         0x00000000001a8054 0x3039580000000c
 .rodata        0x00000000001a8060       0xac E:/nightly/rwsdk.sky/rwsdk/lib/sky2/librwcore.a(texcache.obj)
 *fill*         0x00000000001a810c 0x30395800000004
 .rodata        0x00000000001a8110       0x3c E:/nightly/rwsdk.sky/rwsdk/lib/sky2/librwcore.a(imrascnv.obj)
 *fill*         0x00000000001a814c 0x30395800000004
 .rodata        0x00000000001a8150       0x3c E:/nightly/rwsdk.sky/rwsdk/lib/sky2/librwcore.a(palquant.obj)
 *fill*         0x00000000001a818c 0x30395800000004
 .rodata        0x00000000001a8190       0x39 E:/nightly/rwsdk.sky/rwsdk/lib/sky2/librwcore.a(osintf.obj)
 *fill*         0x00000000001a81c9 0x30395800000007
 .rodata        0x00000000001a81d0       0x3f E:/nightly/rwsdk.sky/rwsdk/lib/sky2/librwcore.a(babbox.obj)
 *fill*         0x00000000001a820f 0x30395800000001
 .rodata        0x00000000001a8210       0x3d E:/nightly/rwsdk.sky/rwsdk/lib/sky2/librwcore.a(babintex.obj)
 *fill*         0x00000000001a824d 0x30395800000003
 .rodata        0x00000000001a8250       0x40 E:/nightly/rwsdk.sky/rwsdk/lib/sky2/librwcore.a(bacolor.obj)
 .rodata        0x00000000001a8290       0x3b E:/nightly/rwsdk.sky/rwsdk/lib/sky2/librwcore.a(batkbin.obj)
 *fill*         0x00000000001a82cb 0x30395800000005
 .rodata        0x00000000001a82d0      0x1ab E:/nightly/rwsdk.sky/rwsdk/lib/sky2/librwcore.a(badma.obj)
 *fill*         0x00000000001a847b 0x30395800000005
 .rodata        0x00000000001a8480       0x3d E:/nightly/rwsdk.sky/rwsdk/lib/sky2/librwcore.a(baevent.obj)
 *fill*         0x00000000001a84bd 0x30395800000003
 .rodata        0x00000000001a84c0       0xf5 E:/nightly/rwsdk.sky/rwsdk/lib/sky2/librwcore.a(dmaalloc.obj)
 *fill*         0x00000000001a85b5 0x30395800000003
 .rodata        0x00000000001a85b8      0x190 E:/usr/local/sce/ee/lib/libgraph.a(graph012.o)
 *fill*         0x00000000001a8748 0x30395800000008
 .rodata        0x00000000001a8750      0x1cc E:/usr/local/sce/ee/lib/libgraph.a(graph018.o)
 *fill*         0x00000000001a891c 0x30395800000004
 .rodata        0x00000000001a8920       0x32 E:/usr/local/sce/ee/lib/libgraph.a(graph003.o)
 *fill*         0x00000000001a8952 0x30395800000006
 .rodata        0x00000000001a8958       0x2f E:/usr/local/sce/ee/lib/libgraph.a(graph008.o)
 *fill*         0x00000000001a8987 0x30395800000001
 .rodata        0x00000000001a8988       0x16 E:/usr/local/sce/ee/lib/libdma.a(libdma.o)
 *fill*         0x00000000001a899e 0x30395800000002
 .rodata        0x00000000001a89a0      0x151 E:/usr/local/sce/ee/lib/libpad.a(libpad.o)
 *fill*         0x00000000001a8af1 0x30395800000003
 .rodata        0x00000000001a8af4        0x4 E:/usr/local/sce/ee/gcc/lib/gcc-lib/ee\2.95.2\../../../../ee\lib\libm.a(sf_ceil.o)
 .rodata        0x00000000001a8af8        0x4 E:/usr/local/sce/ee/gcc/lib/gcc-lib/ee\2.95.2\../../../../ee\lib\libm.a(sf_cos.o)
 *fill*         0x00000000001a8afc 0x30395800000004
 .rodata        0x00000000001a8b00       0x20 E:/usr/local/sce/ee/gcc/lib/gcc-lib/ee\2.95.2\../../../../ee\lib\libm.a(w_pow.o)
 .rodata        0x00000000001a8b20        0x6 E:/usr/local/sce/ee/gcc/lib/gcc-lib/ee\2.95.2\../../../../ee\lib\libm.a(wf_acos.o)
 *fill*         0x00000000001a8b26 0x30395800000002
 .rodata        0x00000000001a8b28        0x7 E:/usr/local/sce/ee/gcc/lib/gcc-lib/ee\2.95.2\../../../../ee\lib\libm.a(wf_atan2.o)
 *fill*         0x00000000001a8b2f 0x30395800000001
 .rodata        0x00000000001a8b30       0x20 E:/usr/local/sce/ee/gcc/lib/gcc-lib/ee\2.95.2\../../../../ee\lib\libm.a(wf_pow.o)
 .rodata        0x00000000001a8b50      0x1d0 E:/usr/local/sce/ee/gcc/lib/gcc-lib/ee\2.95.2\../../../../ee\lib\libm.a(e_pow.o)
 .rodata        0x00000000001a8d20       0x10 E:/usr/local/sce/ee/gcc/lib/gcc-lib/ee\2.95.2\../../../../ee\lib\libm.a(e_sqrt.o)
 .rodata        0x00000000001a8d30       0x38 E:/usr/local/sce/ee/gcc/lib/gcc-lib/ee\2.95.2\../../../../ee\lib\libm.a(ef_acos.o)
 .rodata        0x00000000001a8d68       0x1c E:/usr/local/sce/ee/gcc/lib/gcc-lib/ee\2.95.2\../../../../ee\lib\libm.a(ef_atan2.o)
 *fill*         0x00000000001a8d84 0x30395800000004
 .rodata        0x00000000001a8d88       0x88 E:/usr/local/sce/ee/gcc/lib/gcc-lib/ee\2.95.2\../../../../ee\lib\libm.a(ef_pow.o)
 .rodata        0x00000000001a8e10      0x3c0 E:/usr/local/sce/ee/gcc/lib/gcc-lib/ee\2.95.2\../../../../ee\lib\libm.a(ef_rem_pio2.o)
 .rodata        0x00000000001a91d0        0x8 E:/usr/local/sce/ee/gcc/lib/gcc-lib/ee\2.95.2\../../../../ee\lib\libm.a(ef_sqrt.o)
 .rodata        0x00000000001a91d8       0x1c E:/usr/local/sce/ee/gcc/lib/gcc-lib/ee\2.95.2\../../../../ee\lib\libm.a(kf_cos.o)
 *fill*         0x00000000001a91f4 0x30395800000004
 .rodata        0x00000000001a91f8       0x4c E:/usr/local/sce/ee/gcc/lib/gcc-lib/ee\2.95.2\../../../../ee\lib\libm.a(kf_rem_pio2.o)
 .rodata        0x00000000001a9244       0x1c E:/usr/local/sce/ee/gcc/lib/gcc-lib/ee\2.95.2\../../../../ee\lib\libm.a(kf_sin.o)
 .rodata        0x00000000001a9260        0x8 E:/usr/local/sce/ee/gcc/lib/gcc-lib/ee\2.95.2\../../../../ee\lib\libm.a(s_infconst.o)
                0x00000000001a9260                __infinity
 .rodata        0x00000000001a9268        0x4 E:/usr/local/sce/ee/gcc/lib/gcc-lib/ee\2.95.2\../../../../ee\lib\libm.a(s_lib_ver.o)
                0x00000000001a9268                __fdlib_version
 *fill*         0x00000000001a926c 0x30395800000004
 .rodata        0x00000000001a9270       0x10 E:/usr/local/sce/ee/gcc/lib/gcc-lib/ee\2.95.2\../../../../ee\lib\libm.a(s_rint.o)
 .rodata        0x00000000001a9280       0x30 E:/usr/local/sce/ee/gcc/lib/gcc-lib/ee\2.95.2\../../../../ee\lib\libm.a(s_scalbn.o)
 .rodata        0x00000000001a92b0       0x54 E:/usr/local/sce/ee/gcc/lib/gcc-lib/ee\2.95.2\../../../../ee\lib\libm.a(sf_atan.o)
 .rodata        0x00000000001a9304        0x4 E:/usr/local/sce/ee/gcc/lib/gcc-lib/ee\2.95.2\../../../../ee\lib\libm.a(sf_floor.o)
 .rodata        0x00000000001a9308       0x10 E:/usr/local/sce/ee/gcc/lib/gcc-lib/ee\2.95.2\../../../../ee\lib\libm.a(sf_scalbn.o)
 .rodata        0x00000000001a9318      0x100 E:/usr/local/sce/ee/gcc/lib/gcc-lib/ee\2.95.2\libgcc.a(_udivdi3.o)
 .rodata        0x00000000001a9418      0x100 E:/usr/local/sce/ee/gcc/lib/gcc-lib/ee\2.95.2\libgcc.a(_umoddi3.o)
 .rodata        0x00000000001a9518      0x101 E:/usr/local/sce/ee/gcc/lib/gcc-lib/ee\2.95.2\../../../../ee\lib\libc.a(ctype_.o)
                0x00000000001a9518                _ctype_
 *fill*         0x00000000001a9619 0x30395800000007
 .rodata        0x00000000001a9620        0x2 E:/usr/local/sce/ee/gcc/lib/gcc-lib/ee\2.95.2\../../../../ee\lib\libc.a(impure.o)
 *fill*         0x00000000001a9622 0x3039580000000e
 .rodata        0x00000000001a9630       0xd0 E:/usr/local/sce/ee/gcc/lib/gcc-lib/ee\2.95.2\../../../../ee\lib\libc.a(strtod.o)
 .rodata        0x00000000001a9700      0x204 E:/usr/local/sce/ee/gcc/lib/gcc-lib/ee\2.95.2\../../../../ee\lib\libc.a(vfprintf.o)
 *fill*         0x00000000001a9904 0x3039580000000c
 .rodata        0x00000000001a9910      0x46c E:/usr/local/sce/ee/gcc/lib/gcc-lib/ee\2.95.2\../../../../ee\lib\libc.a(vfscanf.o)
 *fill*         0x00000000001a9d7c 0x30395800000004
 .rodata        0x00000000001a9d80       0x58 E:/usr/local/sce/ee/gcc/lib/gcc-lib/ee\2.95.2\../../../../ee\lib\libc.a(dtoa.o)
 .rodata        0x00000000001a9dd8       0x42 E:/usr/local/sce/ee/gcc/lib/gcc-lib/ee\2.95.2\../../../../ee\lib\libc.a(locale.o)
 *fill*         0x00000000001a9e1a 0x30395800000006
 .rodata        0x00000000001a9e20      0x128 E:/usr/local/sce/ee/gcc/lib/gcc-lib/ee\2.95.2\../../../../ee\lib\libc.a(mprec.o)
                0x00000000001a9f20                __mprec_tinytens
                0x00000000001a9e30                __mprec_tens
                0x00000000001a9ef8                __mprec_bigtens
 .rodata        0x00000000001a9f48       0x70 E:/usr/local/sce/ee/lib\libkernl.a(tty.o)
 *fill*         0x00000000001a9fb8 0x30395800000008
 .rodata        0x00000000001a9fc0      0x154 E:/usr/local/sce/ee/lib\libkernl.a(kprintf.o)
 *fill*         0x00000000001aa114 0x3039580000000c
 .rodata        0x00000000001aa120       0x6d E:/usr/local/sce/ee/lib\libkernl.a(filestub.o)
 *fill*         0x00000000001aa18d 0x30395800000003
 .rodata        0x00000000001aa190        0xc E:/usr/local/sce/ee/lib\libkernl.a(eeloadfile.o)
 *fill*         0x00000000001aa19c 0x30395800000004
 .rodata        0x00000000001aa1a0       0x22 E:/usr/local/sce/ee/lib\libkernl.a(thread.o)
 *fill*         0x00000000001aa1c2 0x30395800000006
 .rodata        0x00000000001aa1c8      0x100 E:/usr/local/sce/ee/gcc/lib/gcc-lib/ee\2.95.2\libgcc.a(_divdi3.o)
 .rodata        0x00000000001aa2c8      0x100 E:/usr/local/sce/ee/gcc/lib/gcc-lib/ee\2.95.2\libgcc.a(_moddi3.o)

.rel.dyn        0x00000000001aa3d0        0x0

.rdata
 *(.rdata)

.gcc_except_table
 *(.gcc_except_table)
                0x00000000001b23f0                _gp=(ALIGN(0x80)+0x7ff0)

.lit8
 *(.lit8)

.lit4           0x00000000001aa400       0xd4
 *(.lit4)
 .lit4          0x00000000001aa400        0x8 obj/sky2/main.o
 .lit4          0x00000000001aa408       0x20 obj/sky2/menu.o
 .lit4          0x00000000001aa428        0x8 obj/sky2/skeleton.o
 .lit4          0x00000000001aa430        0x4 obj/sky2/sky.o
 .lit4          0x00000000001aa434        0x8 E:/nightly/rwsdk.sky/rwsdk/lib/sky2/librplogo.a(rplogo.obj)
 .lit4          0x00000000001aa43c        0x8 E:/nightly/rwsdk.sky/rwsdk/lib/sky2/librtpng.a(pngrutil.obj)
 .lit4          0x00000000001aa444       0x24 E:/nightly/rwsdk.sky/rwsdk/lib/sky2/librtpng.a(pngset.obj)
 .lit4          0x00000000001aa468       0x18 E:/nightly/rwsdk.sky/rwsdk/lib/sky2/librwcore.a(bacamera.obj)
 .lit4          0x00000000001aa480        0x4 E:/nightly/rwsdk.sky/rwsdk/lib/sky2/librwcore.a(baimage.obj)
 .lit4          0x00000000001aa484        0xc E:/nightly/rwsdk.sky/rwsdk/lib/sky2/librwcore.a(bamatrix.obj)
 .lit4          0x00000000001aa490        0xc E:/nightly/rwsdk.sky/rwsdk/lib/sky2/librwcore.a(baresamp.obj)
 .lit4          0x00000000001aa49c       0x1c E:/nightly/rwsdk.sky/rwsdk/lib/sky2/librwcore.a(basky.obj)
 .lit4          0x00000000001aa4b8       0x10 E:/nightly/rwsdk.sky/rwsdk/lib/sky2/librwcore.a(skyinst.obj)
 .lit4          0x00000000001aa4c8        0xc E:/nightly/rwsdk.sky/rwsdk/lib/sky2/librwcore.a(palquant.obj)

.sdata          0x00000000001aa500      0x5fc
 *(.sdata)
 .sdata         0x00000000001aa500       0x3c obj/sky2/main.o
                0x00000000001aa520                Camera
 *fill*         0x00000000001aa53c 0x3034e000000004
 .sdata         0x00000000001aa540       0x5c obj/sky2/im3d.o
                0x00000000001aa578                SolidPurple
                0x00000000001aa580                SolidCyan
                0x00000000001aa550                SolidBlack
                0x00000000001aa584                Im3DPrimType
                0x00000000001aa558                SolidRed
                0x00000000001aa588                Im3DTextured
                0x00000000001aa560                SolidGreen
                0x00000000001aa548                SolidWhite
                0x00000000001aa570                SolidYellow
                0x00000000001aa568                SolidBlue
                0x00000000001aa58c                Im3DColored
 .sdata         0x00000000001aa59c        0x4 obj/sky2/linelist.o
 .sdata         0x00000000001aa5a0        0x4 obj/sky2/polyline.o
 .sdata         0x00000000001aa5a4        0x4 obj/sky2/trilist.o
 .sdata         0x00000000001aa5a8        0x4 obj/sky2/tristrip.o
 .sdata         0x00000000001aa5ac        0x4 obj/sky2/trifan.o
 .sdata         0x00000000001aa5b0        0x4 obj/sky2/events.o
 .sdata         0x00000000001aa5b4        0x4 obj/sky2/camera.o
 .sdata         0x00000000001aa5b8       0x9d obj/sky2/menu.o
 *fill*         0x00000000001aa655 0x3034e000000003
 .sdata         0x00000000001aa658       0x4a obj/sky2/skeleton.o
 *fill*         0x00000000001aa6a2 0x3034e000000006
 .sdata         0x00000000001aa6a8       0x40 obj/sky2/sky.o
 .sdata         0x00000000001aa6e8       0x12 obj/sky2/skyfs.o
 *fill*         0x00000000001aa6fa 0x3034e000000002
 .sdata         0x00000000001aa6fc       0x18 E:/nightly/rwsdk.sky/rwsdk/lib/sky2/librplogo.a(rplogo.obj)
 *fill*         0x00000000001aa714 0x3034e000000004
 .sdata         0x00000000001aa718        0xa E:/nightly/rwsdk.sky/rwsdk/lib/sky2/librtcharse.a(chrprint.obj)
 *fill*         0x00000000001aa722 0x3034e000000002
 .sdata         0x00000000001aa724        0x4 E:/nightly/rwsdk.sky/rwsdk/lib/sky2/librtcharse.a(rtcharse.obj)
 .sdata         0x00000000001aa728        0xf E:/nightly/rwsdk.sky/rwsdk/lib/sky2/librtpng.a(rtpng.obj)
 *fill*         0x00000000001aa737 0x3034e000000001
 .sdata         0x00000000001aa738       0xc7 E:/nightly/rwsdk.sky/rwsdk/lib/sky2/librtpng.a(png.obj)
                0x00000000001aa7d8                png_tRNS
                0x00000000001aa788                png_iTXt
                0x00000000001aa750                png_IEND
                0x00000000001aa778                png_hIST
                0x00000000001aa770                png_gAMA
                0x00000000001aa760                png_bKGD
                0x00000000001aa7b8                png_sPLT
                0x00000000001aa7b0                png_sBIT
                0x00000000001aa7a0                png_sCAL
                0x00000000001aa758                png_PLTE
                0x00000000001aa738                png_sig
                0x00000000001aa780                png_iCCP
                0x00000000001aa7e0                png_zTXt
                0x00000000001aa740                png_IHDR
                0x00000000001aa7d0                png_tIME
                0x00000000001aa768                png_cHRM
                0x00000000001aa798                png_pCAL
                0x00000000001aa7c0                png_sRGB
                0x00000000001aa7c8                png_tEXt
                0x00000000001aa7a8                png_pHYs
                0x00000000001aa748                png_IDAT
                0x00000000001aa790                png_oFFs
 *fill*         0x00000000001aa7ff 0x3034e000000001
 .sdata         0x00000000001aa800        0x6 E:/nightly/rwsdk.sky/rwsdk/lib/sky2/librtpng.a(pngread.obj)
 *fill*         0x00000000001aa806 0x3034e000000002
 .sdata         0x00000000001aa808        0xe E:/nightly/rwsdk.sky/rwsdk/lib/sky2/librtpng.a(pngwutil.obj)
 *fill*         0x00000000001aa816 0x3034e000000002
 .sdata         0x00000000001aa818        0xc E:/nightly/rwsdk.sky/rwsdk/lib/sky2/librtpng.a(deflate.obj)
 *fill*         0x00000000001aa824 0x3034e000000004
 .sdata         0x00000000001aa828        0xe E:/nightly/rwsdk.sky/rwsdk/lib/sky2/librtpng.a(zutil.obj)
 *fill*         0x00000000001aa836 0x3034e000000002
 .sdata         0x00000000001aa838        0x4 E:/nightly/rwsdk.sky/rwsdk/lib/sky2/librtpng.a(inflate.obj)
 .sdata         0x00000000001aa83c        0x8 E:/nightly/rwsdk.sky/rwsdk/lib/sky2/librtpng.a(inftrees.obj)
 .sdata         0x00000000001aa844        0x4 E:/nightly/rwsdk.sky/rwsdk/lib/sky2/librtbmp.a(rtbmp.obj)
 .sdata         0x00000000001aa848        0x4 E:/nightly/rwsdk.sky/rwsdk/lib/sky2/librwcore.a(babinary.obj)
 .sdata         0x00000000001aa84c        0x4 E:/nightly/rwsdk.sky/rwsdk/lib/sky2/librwcore.a(badevice.obj)
 .sdata         0x00000000001aa850        0x3 E:/nightly/rwsdk.sky/rwsdk/lib/sky2/librwcore.a(bafsys.obj)
 *fill*         0x00000000001aa853 0x3034e000000001
 .sdata         0x00000000001aa854        0x4 E:/nightly/rwsdk.sky/rwsdk/lib/sky2/librwcore.a(baresour.obj)
 .sdata         0x00000000001aa858       0x13 E:/nightly/rwsdk.sky/rwsdk/lib/sky2/librwcore.a(bastream.obj)
 *fill*         0x00000000001aa86b 0x3034e000000005
 .sdata         0x00000000001aa870       0x17 E:/nightly/rwsdk.sky/rwsdk/lib/sky2/librwcore.a(batextur.obj)
 *fill*         0x00000000001aa887 0x3034e000000001
 .sdata         0x00000000001aa888       0x10 E:/nightly/rwsdk.sky/rwsdk/lib/sky2/librwcore.a(baim3d.obj)
                0x00000000001aa890                _rwIm3DModule
                0x00000000001aa888                _rwIm3DGlobals
 .sdata         0x00000000001aa898        0x4 E:/nightly/rwsdk.sky/rwsdk/lib/sky2/librwcore.a(bapipe.obj)
                0x00000000001aa898                _rxPipelineGlobalsOffset
 *fill*         0x00000000001aa89c 0x3034e000000004
 .sdata         0x00000000001aa8a0       0x10 E:/nightly/rwsdk.sky/rwsdk/lib/sky2/librwcore.a(nodeClipLine.obj)
 .sdata         0x00000000001aa8b0       0x10 E:/nightly/rwsdk.sky/rwsdk/lib/sky2/librwcore.a(nodeClipTriangle.obj)
 .sdata         0x00000000001aa8c0        0x8 E:/nightly/rwsdk.sky/rwsdk/lib/sky2/librwcore.a(nodeCullTriangle.obj)
 .sdata         0x00000000001aa8c8        0x4 E:/nightly/rwsdk.sky/rwsdk/lib/sky2/librwcore.a(nodeImmInstance.obj)
 *fill*         0x00000000001aa8cc 0x3034e000000004
 .sdata         0x00000000001aa8d0       0x18 E:/nightly/rwsdk.sky/rwsdk/lib/sky2/librwcore.a(nodeImmMangleLineIndices.obj)
 .sdata         0x00000000001aa8e8       0x18 E:/nightly/rwsdk.sky/rwsdk/lib/sky2/librwcore.a(nodeImmMangleTriangleIndices.obj)
 .sdata         0x00000000001aa900        0xc E:/nightly/rwsdk.sky/rwsdk/lib/sky2/librwcore.a(p2core.obj)
                0x00000000001aa904                RxPipelineInstanced
                0x00000000001aa908                _rxHeapGlobal
                0x00000000001aa900                _rwRxHeapInitialSize
 *fill*         0x00000000001aa90c 0x3034e000000004
 .sdata         0x00000000001aa910        0x4 E:/nightly/rwsdk.sky/rwsdk/lib/sky2/librwcore.a(p2renderstate.obj)
 *fill*         0x00000000001aa914 0x3034e000000004
 .sdata         0x00000000001aa918       0xe4 E:/nightly/rwsdk.sky/rwsdk/lib/sky2/librwcore.a(basky.obj)
                0x00000000001aa980                skyDisplayRaster
                0x00000000001aa9c8                skyFSAA0RenderHeight
                0x00000000001aa9e4                skyCameraExt
                0x00000000001aa984                skyDrawRaster
                0x00000000001aa9a8                skyXOff
                0x00000000001aa9c0                skyFSAA0VisibleWidth
                0x00000000001aa948                skyFrame_1
                0x00000000001aa9b0                skyYOff
                0x00000000001aa9f4                gSkyCullState
                0x00000000001aa9d8                dgGGlobals
                0x00000000001aa970                skyTex1_1
                0x00000000001aa91c                skyVideoMode
                0x00000000001aa9e8                skyTextureRaster
                0x00000000001aa924                needCache
                0x00000000001aa9c4                skyFSAA0RenderWidth
                0x00000000001aa93c                skySuspended
                0x00000000001aa9f8                fogTable
                0x00000000001aa958                skyXyoffset_1
                0x00000000001aa940                skyZbuf_1
                0x00000000001aa9e0                skyRasterExt
                0x00000000001aa9ec                skyAlphaTex
                0x00000000001aa998                skyMaxMipLevels
                0x00000000001aa988                skyPrim_State
                0x00000000001aa978                skyAlpha_1
                0x00000000001aa968                skyClamp_1
                0x00000000001aa9cc                skyFSAA0FrameCount
                0x00000000001aa99c                skyFrameBit
                0x00000000001aa950                skyTest_1
                0x00000000001aa920                cacheOpened
                0x00000000001aa960                skyFogcol
                0x00000000001aa9f0                skyVertexAlpha
 .sdata         0x00000000001aa9fc        0x4 E:/nightly/rwsdk.sky/rwsdk/lib/sky2/librwcore.a(skyblit.obj)
 .sdata         0x00000000001aaa00       0x34 E:/nightly/rwsdk.sky/rwsdk/lib/sky2/librwcore.a(skyinst.obj)
                0x00000000001aaa04                overloadWorldPipes
                0x00000000001aaa10                skyUploadedCode
                0x00000000001aaa18                skyUserSwitch2
                0x00000000001aaa0c                skyTransType
                0x00000000001aaa20                skyTLClipperMode
                0x00000000001aaa30                farFogPlane
                0x00000000001aaa1c                skyTSClipperMode
                0x00000000001aaa14                skyUserSwitch1
                0x00000000001aaa08                unOverloadWorldPipes
                0x00000000001aaa2c                useFarClip
 .sdata         0x00000000001aaa34        0xc E:/nightly/rwsdk.sky/rwsdk/lib/sky2/librwcore.a(texcache.obj)
                0x00000000001aaa38                skyGNumTexMemBlocks
 .sdata         0x00000000001aaa40        0x9 E:/nightly/rwsdk.sky/rwsdk/lib/sky2/librwcore.a(babintex.obj)
 *fill*         0x00000000001aaa49 0x3034e000000007
 .sdata         0x00000000001aaa50       0xa4 E:/nightly/rwsdk.sky/rwsdk/lib/sky2/librwcore.a(badma.obj)
                0x00000000001aaaa0                sweDebugMark
                0x00000000001aaae8                sweLocalPacketSize
                0x00000000001aaac0                sweLocalPacket
                0x00000000001aaab4                sweRealLocalPacketBase
                0x00000000001aaacc                sweCurrentBase
                0x00000000001aaa6c                sweFlipPending
                0x00000000001aaad0                sweChainEnd
                0x00000000001aaa78                sweFrameRenderCount
                0x00000000001aaa74                sweNumFlipsInQueue
                0x00000000001aaadc                sweCurrentBlockBase
                0x00000000001aaaa8                swePreAllocCount
                0x00000000001aaa5c                sweDontFlushRefs
                0x00000000001aaa50                sweMaxFlips
                0x00000000001aaac4                __localLocalPacketPointer
                0x00000000001aaa98                sweCurrentHalfOffset
                0x00000000001aaa80                sweFrameRenderCount2
                0x00000000001aaae0                sweNumDispatched
                0x00000000001aaab8                sweLocalPacketBase
                0x00000000001aaac8                circAllocator
                0x00000000001aaaec                swePacketToAddFirst
                0x00000000001aaaa4                swePreAllocSize
                0x00000000001aaad4                sweNumAsyncDispatched
                0x00000000001aaad8                sweChainBase
                0x00000000001aaa70                sweAutoFlip
                0x00000000001aaaac                swePreAllocLimit
                0x00000000001aaae4                sweNumHandler
                0x00000000001aaab0                sweLocalPacketState
                0x00000000001aaabc                sweLocalPacketHigh
                0x00000000001aaa94                sweUseHalfOffset
                0x00000000001aaaf0                swePacketToAddFirstChannel
 .sdata         0x00000000001aaaf4        0x8 E:/nightly/rwsdk.sky/rwsdk/lib/sky2/librwcore.a(dmaalloc.obj)
                0x00000000001aaaf8                sweCircAllocBlockSize

.sbss           0x00000000001aab00      0x11c
                0x00000000001aab00                _fbss=.
 *(.sbss)
 .sbss          0x00000000001aab00        0x4 obj/sky2/main.o
 *fill*         0x00000000001aab04 0x30357800000004
 .sbss          0x00000000001aab08        0x9 obj/sky2/menu.o
 *fill*         0x00000000001aab11 0x30357800000003
 .sbss          0x00000000001aab14       0x1c obj/sky2/sky.o
 .sbss          0x00000000001aab30        0x8 E:/nightly/rwsdk.sky/rwsdk/lib/sky2/librwcore.a(bacamera.obj)
 .sbss          0x00000000001aab38        0x8 E:/nightly/rwsdk.sky/rwsdk/lib/sky2/librwcore.a(baerr.obj)
 .sbss          0x00000000001aab40        0x8 E:/nightly/rwsdk.sky/rwsdk/lib/sky2/librwcore.a(baframe.obj)
 .sbss          0x00000000001aab48        0x8 E:/nightly/rwsdk.sky/rwsdk/lib/sky2/librwcore.a(baimage.obj)
 .sbss          0x00000000001aab50        0x8 E:/nightly/rwsdk.sky/rwsdk/lib/sky2/librwcore.a(bamatrix.obj)
 .sbss          0x00000000001aab58        0x8 E:/nightly/rwsdk.sky/rwsdk/lib/sky2/librwcore.a(bamemory.obj)
 .sbss          0x00000000001aab60        0x8 E:/nightly/rwsdk.sky/rwsdk/lib/sky2/librwcore.a(baraster.obj)
 .sbss          0x00000000001aab68        0x8 E:/nightly/rwsdk.sky/rwsdk/lib/sky2/librwcore.a(baresour.obj)
 .sbss          0x00000000001aab70        0x8 E:/nightly/rwsdk.sky/rwsdk/lib/sky2/librwcore.a(bastream.obj)
 .sbss          0x00000000001aab78        0x8 E:/nightly/rwsdk.sky/rwsdk/lib/sky2/librwcore.a(batextur.obj)
 .sbss          0x00000000001aab80        0x4 E:/nightly/rwsdk.sky/rwsdk/lib/sky2/librwcore.a(batkreg.obj)
 *fill*         0x00000000001aab84 0x30357800000004
 .sbss          0x00000000001aab88        0x8 E:/nightly/rwsdk.sky/rwsdk/lib/sky2/librwcore.a(bavector.obj)
 .sbss          0x00000000001aab90       0x18 E:/nightly/rwsdk.sky/rwsdk/lib/sky2/librwcore.a(basky.obj)
 .sbss          0x00000000001aaba8       0x20 E:/nightly/rwsdk.sky/rwsdk/lib/sky2/librwcore.a(skyblit.obj)
 .sbss          0x00000000001aabc8        0x8 E:/nightly/rwsdk.sky/rwsdk/lib/sky2/librwcore.a(bacolor.obj)
 .sbss          0x00000000001aabd0       0x38 E:/nightly/rwsdk.sky/rwsdk/lib/sky2/librwcore.a(badma.obj)
 *(.scommon)
 .scommon       0x00000000001aac08       0x10 E:/usr/local/sce/ee/gcc/lib/gcc-lib/ee\2.95.2\libgcc.a(_ctors.o)
                                          0x0 (size before relaxing)
                0x00000000001aac08                __CTOR_LIST__
                0x00000000001aac10                __DTOR_LIST__
 .scommon       0x00000000001aac18        0x4 E:/usr/local/sce/ee/gcc/lib/gcc-lib/ee\2.95.2\../../../../ee\lib\libc.a(sbrkr.o)
                                          0x0 (size before relaxing)
                0x00000000001aac18                errno

.bss            0x00000000001aac80     0x7e80
 *(.bss)
 .bss           0x00000000001aac80      0x144 crt0.o
 *fill*         0x00000000001aadc4 0x30366800000004
 .bss           0x00000000001aadc8      0x678 obj/sky2/linelist.o
 .bss           0x00000000001ab440      0x418 obj/sky2/polyline.o
 .bss           0x00000000001ab858      0x630 obj/sky2/trilist.o
 .bss           0x00000000001abe88      0x750 obj/sky2/tristrip.o
 .bss           0x00000000001ac5d8      0x72c obj/sky2/trifan.o
 *fill*         0x00000000001acd04 0x30366800000004
 .bss           0x00000000001acd08       0x10 obj/sky2/camera.o
 .bss           0x00000000001acd18      0x400 obj/sky2/menu.o
 *fill*         0x00000000001ad118 0x30366800000028
 .bss           0x00000000001ad140      0x280 obj/sky2/sky.o
 .bss           0x00000000001ad3c0      0x10c obj/sky2/skyfs.o
 *fill*         0x00000000001ad4cc 0x30366800000034
 .bss           0x00000000001ad500      0x5f0 E:/nightly/rwsdk.sky/rwsdk/lib/sky2/librwcore.a(basky.obj)
 .bss           0x00000000001adaf0       0x10 E:/nightly/rwsdk.sky/rwsdk/lib/sky2/librwcore.a(skyblit.obj)
 .bss           0x00000000001adb00       0x40 E:/nightly/rwsdk.sky/rwsdk/lib/sky2/librwcore.a(texcache.obj)
 .bss           0x00000000001adb40      0x800 E:/nightly/rwsdk.sky/rwsdk/lib/sky2/librwcore.a(palquant.obj)
 .bss           0x00000000001ae340      0x500 E:/nightly/rwsdk.sky/rwsdk/lib/sky2/librwcore.a(badma.obj)
 .bss           0x00000000001ae840      0x3c0 E:/usr/local/sce/ee/lib/libpad.a(libpad.o)
 .bss           0x00000000001aec00        0x4 E:/usr/local/sce/ee/gcc/lib/gcc-lib/ee\2.95.2\libgcc.a(__main.o)
 *fill*         0x00000000001aec04 0x30366800000004
 .bss           0x00000000001aec08       0x18 E:/usr/local/sce/ee/gcc/lib/gcc-lib/ee\2.95.2\libgcc.a(dp-bit.o)
 .bss           0x00000000001aec20       0x10 E:/usr/local/sce/ee/gcc/lib/gcc-lib/ee\2.95.2\libgcc.a(fp-bit.o)
 *fill*         0x00000000001aec30 0x30366800000010
 .bss           0x00000000001aec40      0x3c0 E:/usr/local/sce/ee/lib\libkernl.a(tty.o)
 .bss           0x00000000001af000       0x80 E:/usr/local/sce/ee/lib\libkernl.a(kprintf.o)
 .bss           0x00000000001af080     0x182c E:/usr/local/sce/ee/lib\libkernl.a(sifrpc.o)
 *fill*         0x00000000001b08ac 0x30366800000014
 .bss           0x00000000001b08c0     0x1380 E:/usr/local/sce/ee/lib\libkernl.a(filestub.o)
 .bss           0x00000000001b1c40      0x1c0 E:/usr/local/sce/ee/lib\libkernl.a(iopheap.o)
 .bss           0x00000000001b1e00      0x22c E:/usr/local/sce/ee/lib\libkernl.a(eeloadfile.o)
 *fill*         0x00000000001b202c 0x30366800000004
 .bss           0x00000000001b2030      0x810 E:/usr/local/sce/ee/lib\libkernl.a(thread.o)
 .bss           0x00000000001b2840       0x24 E:/usr/local/sce/ee/lib\libkernl.a(deci2.o)
 *fill*         0x00000000001b2864 0x3036680000001c
 .bss           0x00000000001b2880      0x280 E:/usr/local/sce/ee/lib\libkernl.a(sifcmd.o)

.vubss          0x00000000001b2b00        0x0
                0x00000000001b2b00                end=.
                0x00000000001b2b00                _end=.

.spad
 crt0.o(.spad)
 *(.spad)
OUTPUT(im3d_sky2.elf elf32-littlemips)

.mdebug         0x00000000001b2b00    0x797d0
 .mdebug        0x00000000001b2b00      0x404 crt0.o
 .mdebug        0x00000000001b2f04      0xc7c obj/sky2/main.o
 .mdebug        0x00000000001b3b80      0xb6c obj/sky2/im3d.o
 .mdebug        0x00000000001b46ec      0x710 obj/sky2/linelist.o
 .mdebug        0x00000000001b4dfc      0x77c obj/sky2/polyline.o
 .mdebug        0x00000000001b5578      0x764 obj/sky2/trilist.o
 .mdebug        0x00000000001b5cdc      0x72c obj/sky2/tristrip.o
 .mdebug        0x00000000001b6408      0x734 obj/sky2/trifan.o
 .mdebug        0x00000000001b6b3c      0x330 obj/sky2/events.o
 .mdebug        0x00000000001b6e6c      0x960 obj/sky2/camera.o
 .mdebug        0x00000000001b77cc     0x1674 obj/sky2/menu.o
 .mdebug        0x00000000001b8e40     0x1c1c obj/sky2/skeleton.o
 .mdebug        0x00000000001baa5c     0x1d34 obj/sky2/sky.o
 .mdebug        0x00000000001bc790      0xad0 obj/sky2/skyfs.o
 .mdebug        0x00000000001bd260      0xce0 E:/nightly/rwsdk.sky/rwsdk/lib/sky2/librplogo.a(rplogo.obj)
 .mdebug        0x00000000001bdf40      0x644 E:/nightly/rwsdk.sky/rwsdk/lib/sky2/librtcharse.a(chrprint.obj)
 .mdebug        0x00000000001be584      0x7e8 E:/nightly/rwsdk.sky/rwsdk/lib/sky2/librtcharse.a(rtcharse.obj)
 .mdebug        0x00000000001bed6c      0xb78 E:/nightly/rwsdk.sky/rwsdk/lib/sky2/librtpng.a(rtpng.obj)
 .mdebug        0x00000000001bf8e4     0x11d4 E:/nightly/rwsdk.sky/rwsdk/lib/sky2/librtpng.a(png.obj)
 .mdebug        0x00000000001c0ab8      0x5d8 E:/nightly/rwsdk.sky/rwsdk/lib/sky2/librtpng.a(pngerror.obj)
 .mdebug        0x00000000001c1090     0x18d4 E:/nightly/rwsdk.sky/rwsdk/lib/sky2/librtpng.a(pngget.obj)
 .mdebug        0x00000000001c2964      0x820 E:/nightly/rwsdk.sky/rwsdk/lib/sky2/librtpng.a(pngmem.obj)
 .mdebug        0x00000000001c3184     0x1504 E:/nightly/rwsdk.sky/rwsdk/lib/sky2/librtpng.a(pngread.obj)
 .mdebug        0x00000000001c4688      0x2a8 E:/nightly/rwsdk.sky/rwsdk/lib/sky2/librtpng.a(pngrio.obj)
 .mdebug        0x00000000001c4930     0x15cc E:/nightly/rwsdk.sky/rwsdk/lib/sky2/librtpng.a(pngrtran.obj)
 .mdebug        0x00000000001c5efc     0x1884 E:/nightly/rwsdk.sky/rwsdk/lib/sky2/librtpng.a(pngrutil.obj)
 .mdebug        0x00000000001c7780     0x11f4 E:/nightly/rwsdk.sky/rwsdk/lib/sky2/librtpng.a(pngset.obj)
 .mdebug        0x00000000001c8974      0xb3c E:/nightly/rwsdk.sky/rwsdk/lib/sky2/librtpng.a(pngtrans.obj)
 .mdebug        0x00000000001c94b0      0x324 E:/nightly/rwsdk.sky/rwsdk/lib/sky2/librtpng.a(pngwio.obj)
 .mdebug        0x00000000001c97d4     0x16ec E:/nightly/rwsdk.sky/rwsdk/lib/sky2/librtpng.a(pngwrite.obj)
 .mdebug        0x00000000001caec0      0x500 E:/nightly/rwsdk.sky/rwsdk/lib/sky2/librtpng.a(pngwtran.obj)
 .mdebug        0x00000000001cb3c0     0x1908 E:/nightly/rwsdk.sky/rwsdk/lib/sky2/librtpng.a(pngwutil.obj)
 .mdebug        0x00000000001cccc8      0xa28 E:/nightly/rwsdk.sky/rwsdk/lib/sky2/librtpng.a(deflate.obj)
 .mdebug        0x00000000001cd6f0      0xcb4 E:/nightly/rwsdk.sky/rwsdk/lib/sky2/librtpng.a(trees.obj)
 .mdebug        0x00000000001ce3a4      0x384 E:/nightly/rwsdk.sky/rwsdk/lib/sky2/librtpng.a(zutil.obj)
 .mdebug        0x00000000001ce728      0x6b4 E:/nightly/rwsdk.sky/rwsdk/lib/sky2/librtpng.a(inflate.obj)
 .mdebug        0x00000000001ceddc      0x60c E:/nightly/rwsdk.sky/rwsdk/lib/sky2/librtpng.a(infblock.obj)
 .mdebug        0x00000000001cf3e8      0x510 E:/nightly/rwsdk.sky/rwsdk/lib/sky2/librtpng.a(inftrees.obj)
 .mdebug        0x00000000001cf8f8      0x358 E:/nightly/rwsdk.sky/rwsdk/lib/sky2/librtpng.a(infcodes.obj)
 .mdebug        0x00000000001cfc50      0x224 E:/nightly/rwsdk.sky/rwsdk/lib/sky2/librtpng.a(infutil.obj)
 .mdebug        0x00000000001cfe74      0x208 E:/nightly/rwsdk.sky/rwsdk/lib/sky2/librtpng.a(inffast.obj)
 .mdebug        0x00000000001d007c      0x28c E:/nightly/rwsdk.sky/rwsdk/lib/sky2/librtpng.a(crc32.obj)
 .mdebug        0x00000000001d0308      0x1fc E:/nightly/rwsdk.sky/rwsdk/lib/sky2/librtpng.a(adler32.obj)
 .mdebug        0x00000000001d0504      0x70c E:/nightly/rwsdk.sky/rwsdk/lib/sky2/librtbmp.a(rtbmp.obj)
 .mdebug        0x00000000001d0c10      0xbc0 E:/nightly/rwsdk.sky/rwsdk/lib/sky2/librwcore.a(babinary.obj)
 .mdebug        0x00000000001d17d0     0x1a70 E:/nightly/rwsdk.sky/rwsdk/lib/sky2/librwcore.a(bacamera.obj)
 .mdebug        0x00000000001d3240     0x1690 E:/nightly/rwsdk.sky/rwsdk/lib/sky2/librwcore.a(badevice.obj)
 .mdebug        0x00000000001d48d0      0x43c E:/nightly/rwsdk.sky/rwsdk/lib/sky2/librwcore.a(baerr.obj)
 .mdebug        0x00000000001d4d0c     0x1634 E:/nightly/rwsdk.sky/rwsdk/lib/sky2/librwcore.a(baframe.obj)
 .mdebug        0x00000000001d6340      0x494 E:/nightly/rwsdk.sky/rwsdk/lib/sky2/librwcore.a(bafsys.obj)
 .mdebug        0x00000000001d67d4     0x1b74 E:/nightly/rwsdk.sky/rwsdk/lib/sky2/librwcore.a(baimage.obj)
 .mdebug        0x00000000001d8348      0x640 E:/nightly/rwsdk.sky/rwsdk/lib/sky2/librwcore.a(baimmedi.obj)
 .mdebug        0x00000000001d8988      0x658 E:/nightly/rwsdk.sky/rwsdk/lib/sky2/librwcore.a(baimras.obj)
 .mdebug        0x00000000001d8fe0     0x10d0 E:/nightly/rwsdk.sky/rwsdk/lib/sky2/librwcore.a(bamatrix.obj)
 .mdebug        0x00000000001da0b0      0x9f4 E:/nightly/rwsdk.sky/rwsdk/lib/sky2/librwcore.a(bamemory.obj)
 .mdebug        0x00000000001daaa4      0xfcc E:/nightly/rwsdk.sky/rwsdk/lib/sky2/librwcore.a(baraster.obj)
 .mdebug        0x00000000001dba70      0x4c0 E:/nightly/rwsdk.sky/rwsdk/lib/sky2/librwcore.a(baresamp.obj)
 .mdebug        0x00000000001dbf30      0x89c E:/nightly/rwsdk.sky/rwsdk/lib/sky2/librwcore.a(baresour.obj)
 .mdebug        0x00000000001dc7cc      0x684 E:/nightly/rwsdk.sky/rwsdk/lib/sky2/librwcore.a(bastream.obj)
 .mdebug        0x00000000001dce50      0x5e0 E:/nightly/rwsdk.sky/rwsdk/lib/sky2/librwcore.a(basync.obj)
 .mdebug        0x00000000001dd430     0x25f0 E:/nightly/rwsdk.sky/rwsdk/lib/sky2/librwcore.a(batextur.obj)
 .mdebug        0x00000000001dfa20      0x9c4 E:/nightly/rwsdk.sky/rwsdk/lib/sky2/librwcore.a(batkreg.obj)
 .mdebug        0x00000000001e03e4      0x2e4 E:/nightly/rwsdk.sky/rwsdk/lib/sky2/librwcore.a(batypehf.obj)
 .mdebug        0x00000000001e06c8      0xa3c E:/nightly/rwsdk.sky/rwsdk/lib/sky2/librwcore.a(bavector.obj)
 .mdebug        0x00000000001e1104      0x544 E:/nightly/rwsdk.sky/rwsdk/lib/sky2/librwcore.a(resmem.obj)
 .mdebug        0x00000000001e1648      0x5e8 E:/nightly/rwsdk.sky/rwsdk/lib/sky2/librwcore.a(rwstring.obj)
 .mdebug        0x00000000001e1c30     0x1150 E:/nightly/rwsdk.sky/rwsdk/lib/sky2/librwcore.a(baim3d.obj)
 .mdebug        0x00000000001e2d80      0x428 E:/nightly/rwsdk.sky/rwsdk/lib/sky2/librwcore.a(bapipe.obj)
 .mdebug        0x00000000001e31a8      0xb4c E:/nightly/rwsdk.sky/rwsdk/lib/sky2/librwcore.a(nodeClipLine.obj)
 .mdebug        0x00000000001e3cf4      0xbbc E:/nightly/rwsdk.sky/rwsdk/lib/sky2/librwcore.a(nodeClipTriangle.obj)
 .mdebug        0x00000000001e48b0      0x79c E:/nightly/rwsdk.sky/rwsdk/lib/sky2/librwcore.a(nodeCullTriangle.obj)
 .mdebug        0x00000000001e504c      0x634 E:/nightly/rwsdk.sky/rwsdk/lib/sky2/librwcore.a(nodeImmInstance.obj)
 .mdebug        0x00000000001e5680      0x688 E:/nightly/rwsdk.sky/rwsdk/lib/sky2/librwcore.a(nodeImmMangleLineIndices.obj)
 .mdebug        0x00000000001e5d08      0x660 E:/nightly/rwsdk.sky/rwsdk/lib/sky2/librwcore.a(nodeImmMangleTriangleIndices.obj)
 .mdebug        0x00000000001e6368      0x740 E:/nightly/rwsdk.sky/rwsdk/lib/sky2/librwcore.a(nodeImmRenderSetup.obj)
 .mdebug        0x00000000001e6aa8      0x4b0 E:/nightly/rwsdk.sky/rwsdk/lib/sky2/librwcore.a(nodeImmStash.obj)
 .mdebug        0x00000000001e6f58      0x5fc E:/nightly/rwsdk.sky/rwsdk/lib/sky2/librwcore.a(nodeSubmitLine.obj)
 .mdebug        0x00000000001e7554      0x620 E:/nightly/rwsdk.sky/rwsdk/lib/sky2/librwcore.a(nodeSubmitTriangle.obj)
 .mdebug        0x00000000001e7b74      0x7a0 E:/nightly/rwsdk.sky/rwsdk/lib/sky2/librwcore.a(nodeTransform.obj)
 .mdebug        0x00000000001e8314      0x390 E:/nightly/rwsdk.sky/rwsdk/lib/sky2/librwcore.a(p2altmdl.obj)
 .mdebug        0x00000000001e86a4      0xbf0 E:/nightly/rwsdk.sky/rwsdk/lib/sky2/librwcore.a(p2clpcom.obj)
 .mdebug        0x00000000001e9294     0x1114 E:/nightly/rwsdk.sky/rwsdk/lib/sky2/librwcore.a(p2core.obj)
 .mdebug        0x00000000001ea3a8     0x1164 E:/nightly/rwsdk.sky/rwsdk/lib/sky2/librwcore.a(p2define.obj)
 .mdebug        0x00000000001eb50c      0x69c E:/nightly/rwsdk.sky/rwsdk/lib/sky2/librwcore.a(p2dep.obj)
 .mdebug        0x00000000001ebba8      0x5e0 E:/nightly/rwsdk.sky/rwsdk/lib/sky2/librwcore.a(p2heap.obj)
 .mdebug        0x00000000001ec188      0x590 E:/nightly/rwsdk.sky/rwsdk/lib/sky2/librwcore.a(p2renderstate.obj)
 .mdebug        0x00000000001ec718      0x2a8 E:/nightly/rwsdk.sky/rwsdk/lib/sky2/librwcore.a(p2resort.obj)
 .mdebug        0x00000000001ec9c0      0x650 E:/nightly/rwsdk.sky/rwsdk/lib/sky2/librwcore.a(p2stdcls.obj)
 .mdebug        0x00000000001ed010      0x458 E:/nightly/rwsdk.sky/rwsdk/lib/sky2/librwcore.a(im3dpipe.obj)
 .mdebug        0x00000000001ed468     0x3d98 E:/nightly/rwsdk.sky/rwsdk/lib/sky2/librwcore.a(basky.obj)
 .mdebug        0x00000000001f1200     0x1128 E:/nightly/rwsdk.sky/rwsdk/lib/sky2/librwcore.a(baskytran.obj)
 .mdebug        0x00000000001f2328      0xde0 E:/nightly/rwsdk.sky/rwsdk/lib/sky2/librwcore.a(skyblit.obj)
 .mdebug        0x00000000001f3108      0x874 E:/nightly/rwsdk.sky/rwsdk/lib/sky2/librwcore.a(skyconv.obj)
 .mdebug        0x00000000001f397c     0x19a4 E:/nightly/rwsdk.sky/rwsdk/lib/sky2/librwcore.a(skyinst.obj)
 .mdebug        0x00000000001f5320     0x19b8 E:/nightly/rwsdk.sky/rwsdk/lib/sky2/librwcore.a(texcache.obj)
 .mdebug        0x00000000001f6cd8      0xdc8 E:/nightly/rwsdk.sky/rwsdk/lib/sky2/librwcore.a(imrascnv.obj)
 .mdebug        0x00000000001f7aa0      0x8c4 E:/nightly/rwsdk.sky/rwsdk/lib/sky2/librwcore.a(palquant.obj)
 .mdebug        0x00000000001f8364      0x2b0 E:/nightly/rwsdk.sky/rwsdk/lib/sky2/librwcore.a(osintf.obj)
 .mdebug        0x00000000001f8614      0x3a0 E:/nightly/rwsdk.sky/rwsdk/lib/sky2/librwcore.a(babbox.obj)
 .mdebug        0x00000000001f89b4     0x120c E:/nightly/rwsdk.sky/rwsdk/lib/sky2/librwcore.a(babintex.obj)
 .mdebug        0x00000000001f9bc0      0x2bc E:/nightly/rwsdk.sky/rwsdk/lib/sky2/librwcore.a(bacolor.obj)
 .mdebug        0x00000000001f9e7c      0x628 E:/nightly/rwsdk.sky/rwsdk/lib/sky2/librwcore.a(batkbin.obj)
 .mdebug        0x00000000001fa4a4     0x1c4c E:/nightly/rwsdk.sky/rwsdk/lib/sky2/librwcore.a(badma.obj)
 .mdebug        0x00000000001fc0f0      0x25c E:/nightly/rwsdk.sky/rwsdk/lib/sky2/librwcore.a(baevent.obj)
 .mdebug        0x00000000001fc34c      0x6f4 E:/nightly/rwsdk.sky/rwsdk/lib/sky2/librwcore.a(dmaalloc.obj)
 .mdebug        0x00000000001fca40      0x320 E:/usr/local/sce/ee/lib/libgraph.a(graph001.o)
 .mdebug        0x00000000001fcd60      0x208 E:/usr/local/sce/ee/lib/libgraph.a(graph002.o)
 .mdebug        0x00000000001fcf68      0x210 E:/usr/local/sce/ee/lib/libgraph.a(graph011.o)
 .mdebug        0x00000000001fd178      0x1e4 E:/usr/local/sce/ee/lib/libgraph.a(graph012.o)
 .mdebug        0x00000000001fd35c      0x1dc E:/usr/local/sce/ee/lib/libgraph.a(graph016.o)
 .mdebug        0x00000000001fd538      0x250 E:/usr/local/sce/ee/lib/libgraph.a(graph018.o)
 .mdebug        0x00000000001fd788      0x1d4 E:/usr/local/sce/ee/lib/libgraph.a(graph021.o)
 .mdebug        0x00000000001fd95c      0x1d4 E:/usr/local/sce/ee/lib/libgraph.a(graph026.o)
 .mdebug        0x00000000001fdb30      0x29c E:/usr/local/sce/ee/lib/libgraph.a(graph027.o)
 .mdebug        0x00000000001fddcc      0x214 E:/usr/local/sce/ee/lib/libgraph.a(graph028.o)
 .mdebug        0x00000000001fdfe0      0x20c E:/usr/local/sce/ee/lib/libgraph.a(graph003.o)
 .mdebug        0x00000000001fe1ec      0x1ec E:/usr/local/sce/ee/lib/libgraph.a(graph004.o)
 .mdebug        0x00000000001fe3d8      0x1ec E:/usr/local/sce/ee/lib/libgraph.a(graph005.o)
 .mdebug        0x00000000001fe5c4      0x1f4 E:/usr/local/sce/ee/lib/libgraph.a(graph006.o)
 .mdebug        0x00000000001fe7b8      0x1d4 E:/usr/local/sce/ee/lib/libgraph.a(graph007.o)
 .mdebug        0x00000000001fe98c      0x1e4 E:/usr/local/sce/ee/lib/libgraph.a(graph008.o)
 .mdebug        0x00000000001feb70      0x1f4 E:/usr/local/sce/ee/lib/libgraph.a(graph022.o)
 .mdebug        0x00000000001fed64      0xadc E:/usr/local/sce/ee/lib/libdma.a(libdma.o)
 .mdebug        0x00000000001ff840     0x139c E:/usr/local/sce/ee/lib/libpad.a(libpad.o)
 .mdebug        0x0000000000200bdc     0x118c E:/usr/local/sce/ee/gcc/lib/gcc-lib/ee\2.95.2\../../../../ee\lib\libm.a(sf_ceil.o)
 .mdebug        0x0000000000201d68     0x1174 E:/usr/local/sce/ee/gcc/lib/gcc-lib/ee\2.95.2\../../../../ee\lib\libm.a(sf_cos.o)
 .mdebug        0x0000000000202edc     0x113c E:/usr/local/sce/ee/gcc/lib/gcc-lib/ee\2.95.2\../../../../ee\lib\libm.a(sf_sin.o)
 .mdebug        0x0000000000204018     0x1880 E:/usr/local/sce/ee/gcc/lib/gcc-lib/ee\2.95.2\../../../../ee\lib\libm.a(w_pow.o)
 .mdebug        0x0000000000205898     0x1244 E:/usr/local/sce/ee/gcc/lib/gcc-lib/ee\2.95.2\../../../../ee\lib\libm.a(wf_acos.o)
 .mdebug        0x0000000000206adc     0x1254 E:/usr/local/sce/ee/gcc/lib/gcc-lib/ee\2.95.2\../../../../ee\lib\libm.a(wf_atan2.o)
 .mdebug        0x0000000000207d30     0x194c E:/usr/local/sce/ee/gcc/lib/gcc-lib/ee\2.95.2\../../../../ee\lib\libm.a(wf_pow.o)
 .mdebug        0x000000000020967c     0x28ac E:/usr/local/sce/ee/gcc/lib/gcc-lib/ee\2.95.2\../../../../ee\lib\libm.a(e_pow.o)
 .mdebug        0x000000000020bf28     0x1810 E:/usr/local/sce/ee/gcc/lib/gcc-lib/ee\2.95.2\../../../../ee\lib\libm.a(e_sqrt.o)
 .mdebug        0x000000000020d738     0x1b90 E:/usr/local/sce/ee/gcc/lib/gcc-lib/ee\2.95.2\../../../../ee\lib\libm.a(ef_acos.o)
 .mdebug        0x000000000020f2c8     0x153c E:/usr/local/sce/ee/gcc/lib/gcc-lib/ee\2.95.2\../../../../ee\lib\libm.a(ef_atan2.o)
 .mdebug        0x0000000000210804     0x2ac0 E:/usr/local/sce/ee/gcc/lib/gcc-lib/ee\2.95.2\../../../../ee\lib\libm.a(ef_pow.o)
 .mdebug        0x00000000002132c4     0x1bf8 E:/usr/local/sce/ee/gcc/lib/gcc-lib/ee\2.95.2\../../../../ee\lib\libm.a(ef_rem_pio2.o)
 .mdebug        0x0000000000214ebc     0x1394 E:/usr/local/sce/ee/gcc/lib/gcc-lib/ee\2.95.2\../../../../ee\lib\libm.a(ef_sqrt.o)
 .mdebug        0x0000000000216250     0x1400 E:/usr/local/sce/ee/gcc/lib/gcc-lib/ee\2.95.2\../../../../ee\lib\libm.a(kf_cos.o)
 .mdebug        0x0000000000217650     0x1e44 E:/usr/local/sce/ee/gcc/lib/gcc-lib/ee\2.95.2\../../../../ee\lib\libm.a(kf_rem_pio2.o)
 .mdebug        0x0000000000219494     0x12ac E:/usr/local/sce/ee/gcc/lib/gcc-lib/ee\2.95.2\../../../../ee\lib\libm.a(kf_sin.o)
 .mdebug        0x000000000021a740     0x1070 E:/usr/local/sce/ee/gcc/lib/gcc-lib/ee\2.95.2\../../../../ee\lib\libm.a(s_fabs.o)
 .mdebug        0x000000000021b7b0     0x102c E:/usr/local/sce/ee/gcc/lib/gcc-lib/ee\2.95.2\../../../../ee\lib\libm.a(s_finite.o)
 .mdebug        0x000000000021c7dc      0xefc E:/usr/local/sce/ee/gcc/lib/gcc-lib/ee\2.95.2\../../../../ee\lib\libm.a(s_infconst.o)
 .mdebug        0x000000000021d6d8     0x10d8 E:/usr/local/sce/ee/gcc/lib/gcc-lib/ee\2.95.2\../../../../ee\lib\libm.a(s_isnan.o)
 .mdebug        0x000000000021e7b0      0xf08 E:/usr/local/sce/ee/gcc/lib/gcc-lib/ee\2.95.2\../../../../ee\lib\libm.a(s_lib_ver.o)
 .mdebug        0x000000000021f6b8     0x1000 E:/usr/local/sce/ee/gcc/lib/gcc-lib/ee\2.95.2\../../../../ee\lib\libm.a(s_matherr.o)
 .mdebug        0x00000000002206b8     0x13ec E:/usr/local/sce/ee/gcc/lib/gcc-lib/ee\2.95.2\../../../../ee\lib\libm.a(s_rint.o)
 .mdebug        0x0000000000221aa4     0x1390 E:/usr/local/sce/ee/gcc/lib/gcc-lib/ee\2.95.2\../../../../ee\lib\libm.a(s_scalbn.o)
 .mdebug        0x0000000000222e34     0x1554 E:/usr/local/sce/ee/gcc/lib/gcc-lib/ee\2.95.2\../../../../ee\lib\libm.a(sf_atan.o)
 .mdebug        0x0000000000224388     0x1038 E:/usr/local/sce/ee/gcc/lib/gcc-lib/ee\2.95.2\../../../../ee\lib\libm.a(sf_fabs.o)
 .mdebug        0x00000000002253c0     0x101c E:/usr/local/sce/ee/gcc/lib/gcc-lib/ee\2.95.2\../../../../ee\lib\libm.a(sf_finite.o)
 .mdebug        0x00000000002263dc     0x11a4 E:/usr/local/sce/ee/gcc/lib/gcc-lib/ee\2.95.2\../../../../ee\lib\libm.a(sf_floor.o)
 .mdebug        0x0000000000227580     0x1058 E:/usr/local/sce/ee/gcc/lib/gcc-lib/ee\2.95.2\../../../../ee\lib\libm.a(sf_isnan.o)
 .mdebug        0x00000000002285d8     0x1344 E:/usr/local/sce/ee/gcc/lib/gcc-lib/ee\2.95.2\../../../../ee\lib\libm.a(sf_scalbn.o)
 .mdebug        0x000000000022991c     0x10dc E:/usr/local/sce/ee/gcc/lib/gcc-lib/ee\2.95.2\../../../../ee\lib\libm.a(s_copysign.o)
 .mdebug        0x000000000022a9f8     0x10a4 E:/usr/local/sce/ee/gcc/lib/gcc-lib/ee\2.95.2\../../../../ee\lib\libm.a(sf_copysign.o)
 .mdebug        0x000000000022ba9c     0x12ac E:/usr/local/sce/ee/gcc/lib/gcc-lib/ee\2.95.2\libgcc.a(__main.o)
 .mdebug        0x000000000022cd48     0x106c E:/usr/local/sce/ee/gcc/lib/gcc-lib/ee\2.95.2\libgcc.a(_ctors.o)
 .mdebug        0x000000000022ddb4     0x10cc E:/usr/local/sce/ee/gcc/lib/gcc-lib/ee\2.95.2\libgcc.a(_fixdfdi.o)
 .mdebug        0x000000000022ee80     0x1114 E:/usr/local/sce/ee/gcc/lib/gcc-lib/ee\2.95.2\libgcc.a(_fixunsdfdi.o)
 .mdebug        0x000000000022ff94     0x10cc E:/usr/local/sce/ee/gcc/lib/gcc-lib/ee\2.95.2\libgcc.a(_floatdidf.o)
 .mdebug        0x0000000000231060     0x10e4 E:/usr/local/sce/ee/gcc/lib/gcc-lib/ee\2.95.2\libgcc.a(_floatdisf.o)
 .mdebug        0x0000000000232144     0x1094 E:/usr/local/sce/ee/gcc/lib/gcc-lib/ee\2.95.2\libgcc.a(_muldi3.o)
 .mdebug        0x00000000002331d8     0x10e8 E:/usr/local/sce/ee/gcc/lib/gcc-lib/ee\2.95.2\libgcc.a(_udivdi3.o)
 .mdebug        0x00000000002342c0     0x10e8 E:/usr/local/sce/ee/gcc/lib/gcc-lib/ee\2.95.2\libgcc.a(_umoddi3.o)
 .mdebug        0x00000000002353a8     0x1424 E:/usr/local/sce/ee/gcc/lib/gcc-lib/ee\2.95.2\libgcc.a(dp-bit.o)
 .mdebug        0x00000000002367cc     0x13fc E:/usr/local/sce/ee/gcc/lib/gcc-lib/ee\2.95.2\libgcc.a(fp-bit.o)
 .mdebug        0x0000000000237bc8      0xeec E:/usr/local/sce/ee/gcc/lib/gcc-lib/ee\2.95.2\../../../../ee\lib\libc.a(calloc.o)
 .mdebug        0x0000000000238ab4     0x13ec E:/usr/local/sce/ee/gcc/lib/gcc-lib/ee\2.95.2\../../../../ee\lib\libc.a(callocr.o)
 .mdebug        0x0000000000239ea0      0x624 E:/usr/local/sce/ee/gcc/lib/gcc-lib/ee\2.95.2\../../../../ee\lib\libc.a(ctype_.o)
 .mdebug        0x000000000023a4c4      0xe18 E:/usr/local/sce/ee/gcc/lib/gcc-lib/ee\2.95.2\../../../../ee\lib\libc.a(errno.o)
 .mdebug        0x000000000023b2dc     0x14d4 E:/usr/local/sce/ee/gcc/lib/gcc-lib/ee\2.95.2\../../../../ee\lib\libc.a(fclose.o)
 .mdebug        0x000000000023c7b0      0xe28 E:/usr/local/sce/ee/gcc/lib/gcc-lib/ee\2.95.2\../../../../ee\lib\libc.a(feof.o)
 .mdebug        0x000000000023d5d8     0x1500 E:/usr/local/sce/ee/gcc/lib/gcc-lib/ee\2.95.2\../../../../ee\lib\libc.a(fflush.o)
 .mdebug        0x000000000023ead8     0x1198 E:/usr/local/sce/ee/gcc/lib/gcc-lib/ee\2.95.2\../../../../ee\lib\libc.a(fgets.o)
 .mdebug        0x000000000023fc70     0x1e8c E:/usr/local/sce/ee/gcc/lib/gcc-lib/ee\2.95.2\../../../../ee\lib\libc.a(findfp.o)
 .mdebug        0x0000000000241afc     0x1758 E:/usr/local/sce/ee/gcc/lib/gcc-lib/ee\2.95.2\../../../../ee\lib\libc.a(fopen.o)
 .mdebug        0x0000000000243254     0x100c E:/usr/local/sce/ee/gcc/lib/gcc-lib/ee\2.95.2\../../../../ee\lib\libc.a(fputs.o)
 .mdebug        0x0000000000244260     0x15a8 E:/usr/local/sce/ee/gcc/lib/gcc-lib/ee\2.95.2\../../../../ee\lib\libc.a(fread.o)
 .mdebug        0x0000000000245808     0x1bcc E:/usr/local/sce/ee/gcc/lib/gcc-lib/ee\2.95.2\../../../../ee\lib\libc.a(freer.o)
 .mdebug        0x00000000002473d4     0x1f48 E:/usr/local/sce/ee/gcc/lib/gcc-lib/ee\2.95.2\../../../../ee\lib\libc.a(fseek.o)
 .mdebug        0x000000000024931c     0x1194 E:/usr/local/sce/ee/gcc/lib/gcc-lib/ee\2.95.2\../../../../ee\lib\libc.a(fstatr.o)
 .mdebug        0x000000000024a4b0     0x14b8 E:/usr/local/sce/ee/gcc/lib/gcc-lib/ee\2.95.2\../../../../ee\lib\libc.a(ftell.o)
 .mdebug        0x000000000024b968     0x1b84 E:/usr/local/sce/ee/gcc/lib/gcc-lib/ee\2.95.2\../../../../ee\lib\libc.a(fvwrite.o)
 .mdebug        0x000000000024d4ec     0x1494 E:/usr/local/sce/ee/gcc/lib/gcc-lib/ee\2.95.2\../../../../ee\lib\libc.a(fwalk.o)
 .mdebug        0x000000000024e980     0x1534 E:/usr/local/sce/ee/gcc/lib/gcc-lib/ee\2.95.2\../../../../ee\lib\libc.a(fwrite.o)
 .mdebug        0x000000000024feb4      0xdbc E:/usr/local/sce/ee/gcc/lib/gcc-lib/ee\2.95.2\../../../../ee\lib\libc.a(impure.o)
 .mdebug        0x0000000000250c70     0x185c E:/usr/local/sce/ee/gcc/lib/gcc-lib/ee\2.95.2\../../../../ee\lib\libc.a(makebuf.o)
 .mdebug        0x00000000002524cc     0x10bc E:/usr/local/sce/ee/gcc/lib/gcc-lib/ee\2.95.2\../../../../ee\lib\libc.a(malloc.o)
 .mdebug        0x0000000000253588     0x28c4 E:/usr/local/sce/ee/gcc/lib/gcc-lib/ee\2.95.2\../../../../ee\lib\libc.a(mallocr.o)
 .mdebug        0x0000000000255e4c      0x2dc E:/usr/local/sce/ee/gcc/lib/gcc-lib/ee\2.95.2\../../../../ee\lib\libc.a(memchr.o)
 .mdebug        0x0000000000256128      0x2a8 E:/usr/local/sce/ee/gcc/lib/gcc-lib/ee\2.95.2\../../../../ee\lib\libc.a(memcmp.o)
 .mdebug        0x00000000002563d0      0x2d4 E:/usr/local/sce/ee/gcc/lib/gcc-lib/ee\2.95.2\../../../../ee\lib\libc.a(memcpy.o)
 .mdebug        0x00000000002566a4      0x338 E:/usr/local/sce/ee/gcc/lib/gcc-lib/ee\2.95.2\../../../../ee\lib\libc.a(memmove.o)
 .mdebug        0x00000000002569dc      0x2d8 E:/usr/local/sce/ee/gcc/lib/gcc-lib/ee\2.95.2\../../../../ee\lib\libc.a(memset.o)
 .mdebug        0x0000000000256cb4      0xf98 E:/usr/local/sce/ee/gcc/lib/gcc-lib/ee\2.95.2\../../../../ee\lib\libc.a(mlock.o)
 .mdebug        0x0000000000257c4c     0x11a8 E:/usr/local/sce/ee/gcc/lib/gcc-lib/ee\2.95.2\../../../../ee\lib\libc.a(openr.o)
 .mdebug        0x0000000000258df4     0x12a0 E:/usr/local/sce/ee/gcc/lib/gcc-lib/ee\2.95.2\../../../../ee\lib\libc.a(printf.o)
 .mdebug        0x000000000025a094     0x2644 E:/usr/local/sce/ee/gcc/lib/gcc-lib/ee\2.95.2\../../../../ee\lib\libc.a(qsort.o)
 .mdebug        0x000000000025c6d8      0xfe8 E:/usr/local/sce/ee/gcc/lib/gcc-lib/ee\2.95.2\../../../../ee\lib\libc.a(realloc.o)
 .mdebug        0x000000000025d6c0     0x1da0 E:/usr/local/sce/ee/gcc/lib/gcc-lib/ee\2.95.2\../../../../ee\lib\libc.a(reallocr.o)
 .mdebug        0x000000000025f460     0x1774 E:/usr/local/sce/ee/gcc/lib/gcc-lib/ee\2.95.2\../../../../ee\lib\libc.a(refill.o)
 .mdebug        0x0000000000260bd4     0x1174 E:/usr/local/sce/ee/gcc/lib/gcc-lib/ee\2.95.2\../../../../ee\lib\libc.a(sbrkr.o)
 .mdebug        0x0000000000261d48      0x258 E:/usr/local/sce/ee/gcc/lib/gcc-lib/ee\2.95.2\../../../../ee\lib\libc.a(setjmp.o)
 .mdebug        0x0000000000261fa0     0x1700 E:/usr/local/sce/ee/gcc/lib/gcc-lib/ee\2.95.2\../../../../ee\lib\libc.a(sprintf.o)
 .mdebug        0x00000000002636a0     0x15e4 E:/usr/local/sce/ee/gcc/lib/gcc-lib/ee\2.95.2\../../../../ee\lib\libc.a(sscanf.o)
 .mdebug        0x0000000000264c84     0x1aa0 E:/usr/local/sce/ee/gcc/lib/gcc-lib/ee\2.95.2\../../../../ee\lib\libc.a(stdio.o)
 .mdebug        0x0000000000266724      0x300 E:/usr/local/sce/ee/gcc/lib/gcc-lib/ee\2.95.2\../../../../ee\lib\libc.a(strcat.o)
 .mdebug        0x0000000000266a24      0x328 E:/usr/local/sce/ee/gcc/lib/gcc-lib/ee\2.95.2\../../../../ee\lib\libc.a(strchr.o)
 .mdebug        0x0000000000266d4c      0x368 E:/usr/local/sce/ee/gcc/lib/gcc-lib/ee\2.95.2\../../../../ee\lib\libc.a(strcmp.o)
 .mdebug        0x00000000002670b4      0x2bc E:/usr/local/sce/ee/gcc/lib/gcc-lib/ee\2.95.2\../../../../ee\lib\libc.a(strcpy.o)
 .mdebug        0x0000000000267370      0xf10 E:/usr/local/sce/ee/gcc/lib/gcc-lib/ee\2.95.2\../../../../ee\lib\libc.a(strdup.o)
 .mdebug        0x0000000000268280      0xfa4 E:/usr/local/sce/ee/gcc/lib/gcc-lib/ee\2.95.2\../../../../ee\lib\libc.a(strdup_r.o)
 .mdebug        0x0000000000269224      0x2c0 E:/usr/local/sce/ee/gcc/lib/gcc-lib/ee\2.95.2\../../../../ee\lib\libc.a(strlen.o)
 .mdebug        0x00000000002694e4      0x3c0 E:/usr/local/sce/ee/gcc/lib/gcc-lib/ee\2.95.2\../../../../ee\lib\libc.a(strncat.o)
 .mdebug        0x00000000002698a4      0x37c E:/usr/local/sce/ee/gcc/lib/gcc-lib/ee\2.95.2\../../../../ee\lib\libc.a(strncpy.o)
 .mdebug        0x0000000000269c20      0xef4 E:/usr/local/sce/ee/gcc/lib/gcc-lib/ee\2.95.2\../../../../ee\lib\libc.a(strrchr.o)
 .mdebug        0x000000000026ab14      0xf44 E:/usr/local/sce/ee/gcc/lib/gcc-lib/ee\2.95.2\../../../../ee\lib\libc.a(strstr.o)
 .mdebug        0x000000000026ba58     0x2ef8 E:/usr/local/sce/ee/gcc/lib/gcc-lib/ee\2.95.2\../../../../ee\lib\libc.a(strtod.o)
 .mdebug        0x000000000026e950      0xe54 E:/usr/local/sce/ee/gcc/lib/gcc-lib/ee\2.95.2\../../../../ee\lib\libc.a(strtok.o)
 .mdebug        0x000000000026f7a4      0xfe4 E:/usr/local/sce/ee/gcc/lib/gcc-lib/ee\2.95.2\../../../../ee\lib\libc.a(strtok_r.o)
 .mdebug        0x0000000000270788     0x4110 E:/usr/local/sce/ee/gcc/lib/gcc-lib/ee\2.95.2\../../../../ee\lib\libc.a(vfprintf.o)
 .mdebug        0x0000000000274898     0x32e4 E:/usr/local/sce/ee/gcc/lib/gcc-lib/ee\2.95.2\../../../../ee\lib\libc.a(vfscanf.o)
 .mdebug        0x0000000000277b7c     0x11fc E:/usr/local/sce/ee/gcc/lib/gcc-lib/ee\2.95.2\../../../../ee\lib\libc.a(vsprintf.o)
 .mdebug        0x0000000000278d78     0x11b0 E:/usr/local/sce/ee/gcc/lib/gcc-lib/ee\2.95.2\../../../../ee\lib\libc.a(writer.o)
 .mdebug        0x0000000000279f28     0x1550 E:/usr/local/sce/ee/gcc/lib/gcc-lib/ee\2.95.2\../../../../ee\lib\libc.a(wsetup.o)
 .mdebug        0x000000000027b478      0xe6c E:/usr/local/sce/ee/gcc/lib/gcc-lib/ee\2.95.2\../../../../ee\lib\libc.a(atof.o)
 .mdebug        0x000000000027c2e4     0x1164 E:/usr/local/sce/ee/gcc/lib/gcc-lib/ee\2.95.2\../../../../ee\lib\libc.a(closer.o)
 .mdebug        0x000000000027d448     0x3d3c E:/usr/local/sce/ee/gcc/lib/gcc-lib/ee\2.95.2\../../../../ee\lib\libc.a(dtoa.o)
 .mdebug        0x0000000000281184     0x14d4 E:/usr/local/sce/ee/gcc/lib/gcc-lib/ee\2.95.2\../../../../ee\lib\libc.a(flags.o)
 .mdebug        0x0000000000282658     0x14f8 E:/usr/local/sce/ee/gcc/lib/gcc-lib/ee\2.95.2\../../../../ee\lib\libc.a(locale.o)
 .mdebug        0x0000000000283b50     0x11b0 E:/usr/local/sce/ee/gcc/lib/gcc-lib/ee\2.95.2\../../../../ee\lib\libc.a(lseekr.o)
 .mdebug        0x0000000000284d00     0x1128 E:/usr/local/sce/ee/gcc/lib/gcc-lib/ee\2.95.2\../../../../ee\lib\libc.a(mbtowc_r.o)
 .mdebug        0x0000000000285e28     0x4890 E:/usr/local/sce/ee/gcc/lib/gcc-lib/ee\2.95.2\../../../../ee\lib\libc.a(mprec.o)
 .mdebug        0x000000000028a6b8     0x11a8 E:/usr/local/sce/ee/gcc/lib/gcc-lib/ee\2.95.2\../../../../ee\lib\libc.a(readr.o)
 .mdebug        0x000000000028b860     0x10d8 E:/usr/local/sce/ee/gcc/lib/gcc-lib/ee\2.95.2\../../../../ee\lib\libc.a(s_isinf.o)
 .mdebug        0x000000000028c938     0x1480 E:/usr/local/sce/ee/gcc/lib/gcc-lib/ee\2.95.2\../../../../ee\lib\libc.a(strtol.o)
 .mdebug        0x000000000028ddb8     0x1460 E:/usr/local/sce/ee/gcc/lib/gcc-lib/ee\2.95.2\../../../../ee\lib\libc.a(strtoul.o)
 .mdebug        0x000000000028f218     0x19fc E:/usr/local/sce/ee/gcc/lib/gcc-lib/ee\2.95.2\../../../../ee\lib\libc.a(ungetc.o)
 .mdebug        0x0000000000290c14     0x499c E:/usr/local/sce/ee/lib\libkernl.a(klib.o)
 .mdebug        0x00000000002955b0      0x984 E:/usr/local/sce/ee/lib\libkernl.a(glue.o)
 .mdebug        0x0000000000295f34      0x454 E:/usr/local/sce/ee/lib\libkernl.a(cache.o)
 .mdebug        0x0000000000296388      0x924 E:/usr/local/sce/ee/lib\libkernl.a(intr.o)
 .mdebug        0x0000000000296cac      0x650 E:/usr/local/sce/ee/lib\libkernl.a(tty.o)
 .mdebug        0x00000000002972fc      0x690 E:/usr/local/sce/ee/lib\libkernl.a(kprintf.o)
 .mdebug        0x000000000029798c      0xfd8 E:/usr/local/sce/ee/lib\libkernl.a(sifrpc.o)
 .mdebug        0x0000000000298964     0x1790 E:/usr/local/sce/ee/lib\libkernl.a(filestub.o)
 .mdebug        0x000000000029a0f4      0x58c E:/usr/local/sce/ee/lib\libkernl.a(iopheap.o)
 .mdebug        0x000000000029a680      0xcb4 E:/usr/local/sce/ee/lib\libkernl.a(eeloadfile.o)
 .mdebug        0x000000000029b334      0x224 E:/usr/local/sce/ee/lib\libkernl.a(diei.o)
 .mdebug        0x000000000029b558      0x2d0 E:/usr/local/sce/ee/lib\libkernl.a(initsys.o)
 .mdebug        0x000000000029b828      0x630 E:/usr/local/sce/ee/lib\libkernl.a(thread.o)
 .mdebug        0x000000000029be58      0x694 E:/usr/local/sce/ee/lib\libkernl.a(deci2.o)
 .mdebug        0x000000000029c4ec      0xd54 E:/usr/local/sce/ee/lib\libkernl.a(sifcmd.o)
 .mdebug        0x000000000029d240     0x10e8 E:/usr/local/sce/ee/gcc/lib/gcc-lib/ee\2.95.2\libgcc.a(_divdi3.o)
 .mdebug        0x000000000029e328     0x10e8 E:/usr/local/sce/ee/gcc/lib/gcc-lib/ee\2.95.2\libgcc.a(_moddi3.o)

.DVP.ovlytab    0x00000000001b2b00       0xc0
 .DVP.ovlytab   0x00000000001b2b00       0x48 E:/nightly/rwsdk.sky/rwsdk/lib/sky2/librwcore.a(GenericPRS.obj)
 .DVP.ovlytab   0x00000000001b2b48       0x24 E:/nightly/rwsdk.sky/rwsdk/lib/sky2/librwcore.a(SegmentsPRL.obj)
 .DVP.ovlytab   0x00000000001b2b6c       0x24 E:/nightly/rwsdk.sky/rwsdk/lib/sky2/librwcore.a(SegmentsPRS.obj)
 .DVP.ovlytab   0x00000000001b2b90        0xc E:/nightly/rwsdk.sky/rwsdk/lib/sky2/librwcore.a(baim2dll.obj)
 .DVP.ovlytab   0x00000000001b2b9c        0xc E:/nightly/rwsdk.sky/rwsdk/lib/sky2/librwcore.a(baim2dtl.obj)
 .DVP.ovlytab   0x00000000001b2ba8        0xc E:/nightly/rwsdk.sky/rwsdk/lib/sky2/librwcore.a(banfim2dll.obj)
 .DVP.ovlytab   0x00000000001b2bb4        0xc E:/nightly/rwsdk.sky/rwsdk/lib/sky2/librwcore.a(banfim2dtl.obj)

.DVP.ovlystrtab
                0x00000000001b2b00      0x24b
 .DVP.ovlystrtab
                0x00000000001b2b00       0xe4 E:/nightly/rwsdk.sky/rwsdk/lib/sky2/librwcore.a(GenericPRS.obj)
 .DVP.ovlystrtab
                0x00000000001b2be4       0x70 E:/nightly/rwsdk.sky/rwsdk/lib/sky2/librwcore.a(SegmentsPRL.obj)
 .DVP.ovlystrtab
                0x00000000001b2c54       0x70 E:/nightly/rwsdk.sky/rwsdk/lib/sky2/librwcore.a(SegmentsPRS.obj)
 .DVP.ovlystrtab
                0x00000000001b2cc4        0x1 E:/nightly/rwsdk.sky/rwsdk/lib/sky2/librwcore.a(baasm.obj)
 .DVP.ovlystrtab
                0x00000000001b2cc5       0x22 E:/nightly/rwsdk.sky/rwsdk/lib/sky2/librwcore.a(baim2dll.obj)
 .DVP.ovlystrtab
                0x00000000001b2ce7       0x22 E:/nightly/rwsdk.sky/rwsdk/lib/sky2/librwcore.a(baim2dtl.obj)
 .DVP.ovlystrtab
                0x00000000001b2d09       0x21 E:/nightly/rwsdk.sky/rwsdk/lib/sky2/librwcore.a(banfim2dll.obj)
 .DVP.ovlystrtab
                0x00000000001b2d2a       0x21 E:/nightly/rwsdk.sky/rwsdk/lib/sky2/librwcore.a(banfim2dtl.obj)

.DVP.overlay..0x0.411933251.16.0
                0x0000000000000000      0x800
 .DVP.overlay..0x0.411933251.16.0
                0x0000000000000000      0x800 E:/nightly/rwsdk.sky/rwsdk/lib/sky2/librwcore.a(GenericPRS.obj)

.DVP.overlay..unknvma.3756202193.312.1
                0x0000000000000000      0x800
 .DVP.overlay..unknvma.3756202193.312.1
                0x0000000000000000      0x800 E:/nightly/rwsdk.sky/rwsdk/lib/sky2/librwcore.a(GenericPRS.obj)

.DVP.overlay..unknvma.3756202193.611.2
                0x0000000000000000      0x800
 .DVP.overlay..unknvma.3756202193.611.2
                0x0000000000000000      0x800 E:/nightly/rwsdk.sky/rwsdk/lib/sky2/librwcore.a(GenericPRS.obj)

.DVP.overlay..unknvma.1669965945.131.3
                0x0000000000000000      0x800
 .DVP.overlay..unknvma.1669965945.131.3
                0x0000000000000000      0x800 E:/nightly/rwsdk.sky/rwsdk/lib/sky2/librwcore.a(GenericPRS.obj)

.DVP.overlay..unknvma.1670043769.71.4
                0x0000000000000000      0x800
 .DVP.overlay..unknvma.1670043769.71.4
                0x0000000000000000      0x800 E:/nightly/rwsdk.sky/rwsdk/lib/sky2/librwcore.a(GenericPRS.obj)

.DVP.overlay..unknvma.2864883833.309.5
                0x0000000000000000      0x468
 .DVP.overlay..unknvma.2864883833.309.5
                0x0000000000000000      0x468 E:/nightly/rwsdk.sky/rwsdk/lib/sky2/librwcore.a(GenericPRS.obj)

.DVP.overlay..0x0.824048851.16.0
                0x0000000000000000      0x800
 .DVP.overlay..0x0.824048851.16.0
                0x0000000000000000      0x800 E:/nightly/rwsdk.sky/rwsdk/lib/sky2/librwcore.a(SegmentsPRL.obj)

.DVP.overlay..unknvma.3756202193.328.1
                0x0000000000000000      0x800
 .DVP.overlay..unknvma.3756202193.328.1
                0x0000000000000000      0x800 E:/nightly/rwsdk.sky/rwsdk/lib/sky2/librwcore.a(SegmentsPRL.obj)

.DVP.overlay..unknvma.3756202193.637.2
                0x0000000000000000      0x528
 .DVP.overlay..unknvma.3756202193.637.2
                0x0000000000000000      0x528 E:/nightly/rwsdk.sky/rwsdk/lib/sky2/librwcore.a(SegmentsPRL.obj)

.DVP.overlay..0x0.824048963.16.0
                0x0000000000000000      0x800
 .DVP.overlay..0x0.824048963.16.0
                0x0000000000000000      0x800 E:/nightly/rwsdk.sky/rwsdk/lib/sky2/librwcore.a(SegmentsPRS.obj)

.DVP.overlay..unknvma.3756202193.322.1
                0x0000000000000000      0x800
 .DVP.overlay..unknvma.3756202193.322.1
                0x0000000000000000      0x800 E:/nightly/rwsdk.sky/rwsdk/lib/sky2/librwcore.a(SegmentsPRS.obj)

.DVP.overlay..unknvma.3756202193.631.2
                0x0000000000000000      0x7d8
 .DVP.overlay..unknvma.3756202193.631.2
                0x0000000000000000      0x7d8 E:/nightly/rwsdk.sky/rwsdk/lib/sky2/librwcore.a(SegmentsPRS.obj)

.DVP.overlay..0x0.2250509715.6.0
                0x0000000000000000      0x1f0
 .DVP.overlay..0x0.2250509715.6.0
                0x0000000000000000      0x1f0 E:/nightly/rwsdk.sky/rwsdk/lib/sky2/librwcore.a(baim2dll.obj)

.DVP.overlay..0x0.2250509971.6.0
                0x0000000000000000      0x260
 .DVP.overlay..0x0.2250509971.6.0
                0x0000000000000000      0x260 E:/nightly/rwsdk.sky/rwsdk/lib/sky2/librwcore.a(baim2dtl.obj)

.DVP.overlay..0x0.412131731.6.0
                0x0000000000000000      0x148
 .DVP.overlay..0x0.412131731.6.0
                0x0000000000000000      0x148 E:/nightly/rwsdk.sky/rwsdk/lib/sky2/librwcore.a(banfim2dll.obj)

.DVP.overlay..0x0.412131987.6.0
                0x0000000000000000      0x178
 .DVP.overlay..0x0.412131987.6.0
                0x0000000000000000      0x178 E:/nightly/rwsdk.sky/rwsdk/lib/sky2/librwcore.a(banfim2dtl.obj)
